:020000040800F2
:1000000008FC002061020008215700089B4A0008F4
:100010001D570008E30600088D630008000000007B
:10002000000000000000000000000000A101000826
:100030009308000800000000FD010008695800084E
:100040007B0200087B0200087B0200087B0200089C
:100050007B0200087B0200087B020008150F0008E5
:100060007B0200081F0F00087B020008E906000859
:10007000F906000809070008190700082907000801
:1000800039070008490700087B0200087B020008C6
:100090007B0200087B0200087B020008290F000891
:1000A0007B0200087B0200087B0200087B0200083C
:1000B0007B0200087B020008615900087B020008EF
:1000C0007B0200087B0200087B0200087B0200081C
:1000D0007B0200085D6300086D6300087D63000813
:1000E0007B0200087B0200087B0200087B020008FC
:1000F0007B0200087B0200087B0200085907000809
:100100007B0200087B0200087B0200087B020008DB
:100110009D5C0008AD5C00087B0200087B020008C3
:100120007B0200087B020008690700087B020008C8
:100130007B020008A10900087B0200087B0200087E
:100140007B0200087B0200087B0200087B0200089B
:100150007B0200087B020008790700087B02000888
:100160007B0200087B0200087B0200087B0200087B
:100170007B0200087B0200087B02000800000000F0
:100180007B0200087B020008DFF810D000F06CFA58
:1001900000480047119D0008AFF3008008FC0020D4
:1001A0002C4B19680868B0E8F04F80F30988BFF35A
:1001B0006F8F4FF0000080F311887047000000003F
:1001C00008480068006880F308884FF0000080F35A
:1001D000148862B661B6BFF34F8FBFF36F8F00DF35
:1001E00000BF00BF08ED00E0DFF80C00016841F43B
:1001F00070010160704700BF88ED00E0EFF30980F7
:10020000BFF36F8F134B1A681EF0100F08BF20ED5D
:10021000108A20E9F04F106009B44FF0500080F3CD
:100220001188BFF34F8FBFF36F8F15F039FC4FF07C
:10023000000080F3118809BC19680868B0E8F04F25
:100240001EF0100F08BFB0EC108A80F30988BFF3CE
:100250006F8F704778000020EFF305807047000033
:100260000648804706480047FEE7FEE7FEE7FEE750
:10027000FEE7FEE7FEE7FEE7FEE7FEE74D59000872
:10028000890100082DE9F05F0546002092469B4653
:1002900088460646814640241BE02846414647469C
:1002A000224600F03DF953465A46C01A914110D3F8
:1002B00011461846224600F024F92D1A67EB010872
:1002C0004F4622460120002100F01BF917EB0009E0
:1002D0004E41201EA4F10104DFDC484631462A4687
:1002E0004346BDE8F09F00000649074A08685043AE
:1002F00043F2390210440860400870470149086021
:1003000070470000640600206D4EC64110B5431AC8
:10031000934209D28318881803E010F8011D03F8EE
:10032000011D521EF9D210BD40EA01039B0703D004
:1003300009E008C9121F08C0042AFAD203E011F824
:10034000013B00F8013B521EF9D210BDD2B201E0D0
:1003500000F8012B491EFBD270470022F6E710B5CA
:1003600013460A4604461946FFF7F0FF204610BD23
:10037000421C10F8011B0029FBD1801A704730B5D0
:1003800004460020034600E05B1C934203D2E05C7D
:10039000CD5C401BF8D030BD2DE9FE4F81EA03044F
:1003A00004F0004421F0004100944FF0000B23F0D2
:1003B000004350EA01045ED052EA03045BD0C3F369
:1003C0000A54C1F30A552C44A4F2F3340194A0FB5F
:1003D0000254C1F3130141F48011C3F3130343F436
:1003E000801301FB024400FB034E840A970A44EA8F
:1003F000815447EA8357A4FB076802958D0A05FBE1
:1004000007854FEA932C04FB0C542705029D4FEA05
:10041000065847EA1637B5EB08056EEB070C870E52
:10042000920E47EA811742EA8312A7FB0201B6EB5C
:100430000B0164EB00042B0D43EA0C335E1844EB14
:100440001C50DA465146E7FB0201C5F313044FEA9C
:100450000B3343EA14534FEA0432019C43EA060388
:10046000A4F10C040294009CCDE900B400F0AEF8B5
:1004700003B0BDE8F08F00200146F9E70EB5C10FCB
:1004800080EAE0700844CA07002140F233438DE857
:100490000E000A460B4600F099F803B000BD01F0CB
:1004A000004330B421F0004150EA010206D00A0DA9
:1004B000A2F56072C1F31301002A02DC30BC0020F7
:1004C0007047440F44EAC104C100E01830BC00EB9F
:1004D000C25000F035B830B50B460146002020224E
:1004E000012409E021FA02F59D4205D303FA02F541
:1004F000491B04FA02F52844151EA2F10102F1DCA1
:1005000030BD202A04DB203A00FA02F100207047B7
:100510009140C2F1200320FA03F319439040704741
:10052000202A04DB203A21FA02F00021704721FA48
:1005300002F3D040C2F120029140084319467047AF
:100540000029A8BF7047401C490008BF20F00100E7
:10055000704710B4B0FA80FC00FA0CF050EA0104C5
:1005600004BF10BC704749B1CCF1200421FA04F457
:1005700011FA0CF118BF012121430843A3EB0C0130
:10058000CB1D4FEA00614FEA102042BF002010BC93
:10059000704700EBC35010440029A4BF10BC704743
:1005A000401C490008BF20F0010010BC704710B586
:1005B000141E73F1000408DA401C41F10001921886
:1005C0005B411A4301D120F0010010BD2DE9F04D2F
:1005D00092469B4611B1B1FA81F202E0B0FA80F284
:1005E00020329046FFF78DFF04460F4640EA0A008E
:1005F00041EA0B0153465A46084313D0114653EAC9
:10060000010019D0C8F140025046FFF789FF0546A6
:100610000E46504659464246FFF773FF084305D041
:10062000012004E020463946BDE8F08D0020054356
:1006300046EAE0762C4337430A986305E40AA0EBC8
:1006400008000022FD0A44EA47540A3002D500207F
:100650000146E9E7010510196941DDE9084500197E
:100660006941BDE8F04DA2E7064C074D06E0E068A1
:1006700040F0010394E8070098471034AC42F6D3E9
:10068000FFF786FD5C7101087C71010870B58C185C
:1006900010F8015B15F0070301D110F8013B2A1196
:1006A00006D110F8012B03E010F8016B01F8016B83
:1006B0005B1EF9D12B0705D40023521E0DD401F87F
:1006C000013BFAE710F8013BCB1A921C03E013F848
:1006D000015B01F8015B521EF9D5A142D8D300207D
:1006E00070BD00BFFEE7000010B5024800F0E6FD57
:1006F00010BD0000C030002010B5024800F0DEFD43
:1007000010BD0000A032002010B5024800F0D6FD58
:1007100010BD0000A02F002010B5024800F0CEFD53
:1007200010BD00000033002010B5024800F0C6FDE7
:1007300010BD00000030002010B5024800F0BEFDE2
:1007400010BD0000E031002010B5024800F0B6FDF9
:1007500010BD00004032002010B5024800F0AEFD90
:1007600010BD00006030002010B5024800F0A6FD6A
:1007700010BD00002031002010B5024800F09EFDA1
:1007800010BD000080310020014608781038182381
:10079000B0FBF3F20848805CC865032A05D90868F5
:1007A0006FF30900001D886503E008686FF3090016
:1007B0008865886D70470000306E01080146002092
:1007C0008A6A8B69CBB932B1012A0DD0022A03D0D3
:1007D000032A10D10EE000BFCB6A03F08073B3F19F
:1007E000807F00D1012007E0CB6AB3F1C07F00D148
:1007F000012001E000E000BF34E08B69B3F5005F49
:100800001AD132B1012A07D0022A03D0032A11D10A
:100810000AE000BF01200EE0CB6A03F08073B3F161
:10082000807F00D1012006E0CB6AB3F1C07F00D108
:10083000012000E000BF15E032B1012A05D0022AF4
:1008400004D0032A0CD103E000BF00BF012008E060
:10085000CB6A03F08073B3F1807F00D1012000E008
:1008600000BF00BF704730B50468246824F48024BA
:1008700005682C60046863608468402C04D10468B7
:10088000A2600468E16003E00468A1600468E260BB
:1008900030BD704710B50146002226E002EB82040D
:1008A0000B6903EBC4000023036043608360C360F3
:1008B000036243624FF0004303604FF48C43436094
:1008C000436823F00043436001F1480343F82200EA
:1008D000032A07D202EB82040B6903EBC40328331B
:1008E000C36001E00B69C360521C042AD6D3002404
:1008F000CC650C668C66CC668C650B6803F5805302
:100900000C69DC6010BD10B50146002222E002EB4C
:100910008204CB6803EBC400002303604360836060
:10092000C36001F1180343F82200036843F4801305
:100930000360032A07D202EB8204CB6803EBC403F3
:100940002833C36001E0CB68C360036843F440030D
:100950000360521C042ADAD300248C620B6803F56E
:100960008053CC681C6110BD38B50446002000904F
:10097000206800F58050806940F48011206800F5FF
:1009800080508161206800F58050806900900120CE
:1009900000F074FE0099206800F58050816138BD38
:1009A00010B5044800F006FF4FF40051024801F072
:1009B00097FD10BD6C7E00200010024030B503464C
:1009C0001479557944EA0520084C0C442064D47805
:1009D0002406957844EA0544557844EA05241578B8
:1009E00044EA0500014C0C44606430BD00800240C4
:1009F00010B5A4B0044601208DF83C008DF83D00F0
:100A000000200D908DF84B0001208DF84A00002049
:100A10008DF8480001208DF8300000208DF84C0042
:100A20008DF83B0014908DF854001D908DF87800DF
:100A30001F908DF882008DF880004FF48040109058
:100A4000C010119000208DF881000BA9204600F005
:100A500095F901208DF80C008DF80D008DF81D0022
:100A60008DF80E00002005908DF81C008DF81E00FA
:100A7000089001208DF824008DF8040000040290F5
:100A8000800106904012049001208DF8250000207E
:100A90000A9000906946204600F010F924B010BD7D
:100AA0000020704710B501F02BFD10BD10B50248B5
:100AB00001F082F9002010BD6C7E002070B5044664
:100AC0000D46164633462A462146044801F0A6F84C
:100AD00010B14FF0FF3070BD0020FCE76C7E0020AD
:100AE00070B504460D46164633462A46214604484C
:100AF00001F0BFFA10B14FF0FF3070BD0020FCE7ED
:100B00006C7E00202DE9F04F80460C46164608F119
:100B100018031A69D3F810904FF0000C53F8221004
:100B2000A568E246086800F00040B0F1004F04D02C
:100B300003F1140050F8220010B10220BDE8F08F3C
:100B40000CF1010C2868886048686FF30C00D5F838
:100B500004B040EA0B004860207800F0010038B192
:100B6000086820F44000D4F814B040EA0B00086094
:100B7000207800F0200038B1086820F04060D4F8F8
:100B800010B040EA0B000860207800F0040018B1B3
:100B9000086840F080000860086840F080500860F5
:100BA00000BF00BF00BFBFF35F8F00BF00BF00BF2B
:100BB000086840F0004008605DE0086820F00050E0
:100BC000086026B1086840F08040086003E00868CB
:100BD00020F08040086000BF521C042A00D3121F7E
:100BE00000BF53F82210086820F0805008600868A1
:100BF00000F00040B0F1004F04D003F1140050F8B1
:100C00002200E8B14A4653F82210002714E000BF42
:100C100000BF00BFBFF35F8F00BF00BF00BF086809
:100C200020F00040086000BF521C042A00D3121FAD
:100C300000BF53F822107F1C6745E8D302207DE7F0
:100C40000CF1010CAD682868886048686FF30C00EF
:100C5000D5F804B040EA0B0048600AF1010A00BF71
:100C600000BF00BFBFF35F8F00BF00BF00BF0868B9
:100C700040F000400860A86800289ED126B10868AE
:100C800040F08040086003E0086820F08040086081
:100C9000086840F00050086003F11400D3F824B055
:100CA00040F822B01A6172B60AF10100D3F828B0F8
:100CB0005844986262B6002040E7000070B50546CF
:100CC0000C46286800F5805086692B480640207B3A
:100CD00008B9012000E000208006617B40EA416005
:100CE000617F09B9012100E0002140EA0150A17BA8
:100CF00040EA415061690843217F40EAC110A17F69
:100D000040EA8110216A084394F8241040EA8100E7
:100D10000643286800F580508661286800F58050F9
:100D20008669012000F0AAFC286800F580508661E1
:100D30002179A06840EA4160A1690843216908431C
:100D400094F8251040EAC110A16A40EA81002168A8
:100D5000084340F40001286800F5805001602868CD
:100D600000F580500668012000F088FC286800F536
:100D70008050066070BD0000233FDEF870B5054668
:100D80000C46286806683A480640207C08B90120CD
:100D900000E00020C005617C09B9012100E00021CC
:100DA00040EA8150A1680843E17F40EA014061695F
:100DB0000843A17F09B9012100E0002140EA413048
:100DC000217F40EA0130A1690843217940EA81206E
:100DD00094F8201009B9012100E0002140EA4120E7
:100DE000E17B40EAC110616A084394F8281040EAA8
:100DF000011006432868066028680668012000F094
:100E00003DFC28680660286886694FF641700640F8
:100E1000A06C000494F84C1009B9012100E00021F5
:100E200040EAC110216D084394F85510012900D102
:100E300000E0002140EAC10094F85610012900D1D9
:100E400000E0002140EA810094F85410012900D10B
:100E500000E0002140EA41000643286886612868D6
:100E60008669012000F00AFC2868866170BD0000D8
:100E70000F8120FF2DE9F8430446002000904FF039
:100E80000108A66E04F1480050F82650E76E2FE0E6
:100E9000286A58B9684600F033FF009810B94FF03F
:100EA000000803E0009828620098A860B8F1000FDD
:100EB0001ED0A06D10B91648686002E04FF48C4057
:100EC000686000BF00BF00BFBFF35F8F00BF00BFFF
:100ED00000BF286840F00040286000BF761C042E48
:100EE00000D3361F00BF04F1480050F826507F1E83
:100EF00017B1B8F1000FCBD1E06EB84206D0002197
:100F0000206800F580508160A666E766BDE8F8833A
:100F10000046008010B5022001F0D2F910BD10B5D6
:100F2000082001F0CDF910BD10B54FF4807001F02C
:100F3000C7F910BD7047000010B5002201B909E0E3
:100F4000012901D10A0205E0022901D10A0201E0CA
:100F50004FF440720E4B1B6823F440730C4C23601B
:100F600023461B681343236023461B6823F0F803C2
:100F7000236023461B68022444EAC0042343044C34
:100F8000236023461B6843F48033236010BD0000B8
:100F9000103C02401C48006800F40070B0B11A48D0
:100FA000006820F400701849086000BF0846006817
:100FB00040F4006008600846006820F400600860A3
:100FC00000BF0846006840F4007008600E480068E2
:100FD00000F48060B0B10C48006820F480600A49D9
:100FE000086000BF0846006840F48050086008466A
:100FF000006820F48050086000BF0846006840F494
:101000008060086070470000003C02400A4A126895
:1010100022F44072084B1A601A46126842F0040229
:101020001A601A4612684FF4803343EA00231A43C9
:10103000014B1A6070470000103C0240074A1268DA
:1010400022F44072054B1A601A4612681A601A465A
:10105000126842F001021A6001707047103C0240B1
:1010600010B50D49096821F440710B4C21602146EF
:10107000096841F4407121602146096841F001018D
:101080002160026000BF00BF00BFBFF36F8F00BFD1
:1010900000BF00BF436010BD103C0240084A126808
:1010A00022F44072064B1A601A46126842F48072AB
:1010B0001A601A46126842F001021A6001807047F5
:1010C000103C0240084A126822F44072064B1A6033
:1010D0001A46126842F400721A601A46126842F008
:1010E00001021A6001607047103C0240234800680A
:1010F00000F0100040B12248C06940F010002049C3
:10110000C86110201D4908601C48006800F02000DC
:1011100040B11B48C06940F008001949C86120204F
:10112000164908601548006800F0400040B11448B6
:10113000C06940F004001249C86140200F490860AE
:101140000E48006800F0800040B10D48C06940F0D2
:1011500002000B49C8618020084908600748006800
:1011600000F0020040B10648C06940F02000044988
:10117000C861022001490860704700000C3C024031
:10118000AC7F002070B50446002500201449C861DA
:1011900001F0B6F9054609E0601C38B124B101F050
:1011A000AFF9401BA04201D9032070BD0D48006873
:1011B00000F480300028EFD10A48006800F00100F8
:1011C00010B10120074908600648006800F0F200ED
:1011D00018B1FFF78BFF0120E7E70020E5E70000EB
:1011E000AC7F00200C3C024070B50446A56D01F0B8
:1011F00087F9064694F83500022808D080206065FB
:1012000000BF002084F8340000BF012070BD2068BA
:10121000006820F01600216808602068406920F00E
:10122000800021684861206C08B9A06C28B1206852
:10123000006820F00800216808602068006820F03D
:1012400001002168086010E001F05AF9801B0528B0
:101250000BD920206065032084F8350000BF0020F2
:1012600084F8340000BF0320D0E72068006800F055
:1012700001000028E8D194F85C103F208840A86065
:10128000012084F8350000BF002084F8340000BF3E
:1012900000BFBBE7014691F83500022803D080204B
:1012A000486501207047052081F83500086800680E
:1012B00020F001000A6810600020F3E7F8B504464A
:1012C000002000908C4800684FF41651B0FBF1F7F5
:1012D000A56D2E6894F85C1008208840304098B1C5
:1012E0002068006800F0040070B12068006820F0F9
:1012F00004002168086094F85C1008208840A86009
:10130000606D40F00100606594F85C100120884039
:10131000304068B12068406900F0800040B194F826
:101320005C1001208840A860606D40F0020060659C
:1013300094F85C1004208840304068B12068006850
:1013400000F0020040B194F85C1004208840A860CE
:10135000606D40F00400606594F85C1010208840D7
:10136000304078B32068006800F0080050B394F86B
:101370005C1010208840A8602068006800F480207D
:1013800080B12068006800F4002028B9206CC8B142
:101390002046216C884715E0A06C98B12046A16CCE
:1013A00088470FE02068006800F4807028B9206842
:1013B000006820F0080021680860206C10B1204609
:1013C000216C884794F85C10202088403040002829
:1013D00065D02068006800F0100000285FD094F805
:1013E0005C1020208840A86094F83500052828D19A
:1013F0002068006820F016002168086020684069B5
:1014000020F0800021684861206C08B9A06C28B1E8
:101410002068006820F008002168086094F85C10DB
:101420003F208840A860012084F8350000BF0020DC
:1014300084F8340000BF206D10B12046216D88472C
:10144000F8BD2068006800F4802080B12068006842
:1014500000F4002028B9606C10B12046616C884708
:101460001DE0E06BD8B12046E16B884717E02068AB
:10147000006800F4807068B92068006820F01000EF
:1014800021680860012084F8350000BF002084F83E
:10149000340000BFE06B10B12046E16B8847606DFF
:1014A00038B3606D00F00100F0B1052084F835001C
:1014B0002068006820F001002168086000BF0098E3
:1014C000401C0090B84200D905E02068006800F098
:1014D00001000028F3D100BF012084F8350000BFCF
:1014E000002084F8340000BFE06C10B12046E16CAD
:1014F000884700BFA4E70000740000202DE9F041F8
:101500000446002500F0FCFF074614B90120BDE8A1
:10151000F081606A00B100BF022084F8350000BF8E
:10152000002084F8340000BF2068006820F001002B
:10153000216808600AE000F0E3FFC01B052805D918
:1015400020206065032084F83500E0E7206800680B
:1015500000F001000028EED1206805682148054010
:10156000D4E901010843E16808432169084361693E
:101570000843A1690843E1690843216A0843054318
:10158000606A042803D1D4E90B01084305432068AD
:1015900005602068456925F00705606A0543606AB3
:1015A00004280DD1A06A0543E06A48B12046FFF740
:1015B00005F928B140206065012084F83500A6E7D0
:1015C000206845612046FFF7DFF8064694F85C1076
:1015D0003F208840B06000206065012084F835001D
:1015E000002094E73F8010F02DE9F04704460D46B7
:1015F00016461F464FF00008D4F8589000BF94F8E4
:101600003400012802D10220BDE8F087012084F8CF
:10161000340000BF94F83500012825D1022084F859
:101620003500002060653B46324629462046FFF7DC
:101630001AF994F85C103F208840C9F80800206827
:10164000006840F0160021680860206C28B120680E
:10165000006840F00800216808602068006840F0D9
:1016600001002168086006E000BF002084F8340013
:1016700000BF4FF002084046C6E7000070B50446C0
:1016800000F03EFF06462546681C10B1044800786D
:10169000054400BF00F034FF801BA842FAD370BDA0
:1016A0007000002010B50446204600F00BF800F052
:1016B0008000802803D10248006809F0B7FF10BD00
:1016C000340000200146D1F88C007047024609B969
:1016D0000120704710680068C0F3001081F82800EE
:1016E0001068006800F06000486210680068C0F38D
:1016F000402080F0010081F8200010680068C0F3ED
:101700000040C87710680068C0F3403080F00100E6
:10171000887710680068C0F30030087710680068A8
:1017200000F4006088611068006800F4804048613F
:1017300010680068C0F3805080F0010048741068A1
:101740000068C0F3C05080F00100087410680068A1
:10175000C0F3C010C8731068006800F4602088608F
:1017600010680068C0F38020087110688069C0F3B9
:10177000400081F8540010688069C0F3C01080F008
:10178000010081F84C001068806900F030000865A5
:1017900010688069000C886410688069C0F380005C
:1017A00081F8560010688069C0F3C00081F85500C8
:1017B00000208EE710B50446206800F5805040698F
:1017C00000F0400040280FD1206800F58050C0692B
:1017D00000F04000402807D14249206800F58050C1
:1017E0004161204600F0B0FA206800F58050406961
:1017F00000F0010078B1206800F58050C06900F069
:10180000010040B14FF00111206800F580504161A6
:10181000204600F01DFC206800F58050406900F46F
:101820000040B0F5004F3DD1206800F58050C06900
:1018300000F40040B0F5004F34D1D4F8880040F0F7
:101840000800C4F88800206800F58050406900F462
:101850000050B0F5005F15D1206800F58050406958
:1018600021490840C4F88C00206800F58050C06908
:1018700020F4C031206800F58050C161E020C4F838
:1018800084000CE0206800F58050406948F28061D7
:101890000840C4F88C00206800F580504161204663
:1018A000FFF700FF2068806B00F0080008280BD1CC
:1018B0002068C06A00F06000C4F89400204600F080
:1018C0002BF90020C4F894000848006800F40020B8
:1018D00030B14FF4002005490860204600F0C8FBF5
:1018E00010BD00004000010000207E00143C0140BB
:1018F00038B504460CB9012038BDD4F8840028B9A5
:101900002320C4F88400204600F05CF800BF0020CB
:1019100000902A48006840F4804028490860084642
:10192000006800F48040009000BF00BF24480068B9
:1019300020F400002249086008460068A1680843B6
:101940001F49086008460068206800F5805000685C
:1019500040F00101206800F58050016000F0D0FDEA
:1019600005460DE000F0CCFD401BB0F5FA7F07D92D
:101970000420C4F88800E020C4F884000120BBE7FC
:10198000206800F58050006800F001000028E9D1CF
:101990002046FFF72DF82046FEF7B5FF2046FEF75C
:1019A00079FF002120466268FFF708F80020C4F89C
:1019B00088001020C4F8840000209DE744380240CD
:1019C0000438014010B586B00446142101A8FEF782
:1019D000C4FC4C49206888427ED100BF00BF002073
:1019E00000904948006840F0007047490860084688
:1019F000006800F00070009000BF00BF00BF002032
:101A000000900846006840F0806008600846006862
:101A100000F08060009000BF00BF00BF0020009079
:101A20000846006840F0006008600846006800F062
:101A30000060009000BF00BF00BF00BF002000900A
:101A40000846006840F0040008600846006800F09E
:101A50000400009000BF00BF00BF002000900846B7
:101A6000006840F0010008600846006800F00100CE
:101A7000009000BF00BF00BF002000900846006833
:101A800040F0020008600846006800F00200009084
:101A900000BF00BF3220019002200290002003907E
:101AA000032004900B20059001A9184800F016FCB3
:101AB00086200190022002900020039003200490D1
:101AC0000B20059001A9124800F008FC4FF460506B
:101AD00001900220029000E011E00020039003201A
:101AE00004900B20059001A90A4800F0F7FB0022A2
:101AF00005213D2000F0D4FD3D2000F0C1FD06B0E1
:101B000010BD000000800240303802400008024052
:101B1000000002400004024070472DE9F05F0446D7
:101B20000F464FF00008C34647B9D4F8880040F08C
:101B30000100C4F888000120BDE8F09FD4F88400BB
:101B4000232801D00120F7E7E66D04F1480050F8A2
:101B50002650E06EC0F1040942E0286800F480706D
:101B600018B1A969A167E9696167286800F4007084
:101B700008B9E06F40B3286800F4007010B100218C
:101B800021666166D4F814A0286800F4807040B122
:101B90002868C0F30D40A0F1040A296821674FF0BE
:101BA000010BA86828621FFA8AF304F18001081F5C
:101BB0002A6A00F0D3F8206E401C2066606E00EBAD
:101BC0000A0161660020286200BF761C042E00D343
:101BD000361F00BF04F1480050F8265008F10108F4
:101BE000286800F0004020B9C84502D2BBF1000FC0
:101BF000B3D0E06E00EB0801E166E06E10B1204664
:101C0000FFF738F9E665BBF1010F05D1E06F3860E9
:101C10000021E16700208FE701208DE72DE9F047E3
:101C200005460E46174698462868046904F01C04C9
:101C30004FF4784000EAC62004434FF4F86000EA0D
:101C40008710044324F0020444F00104286804616E
:101C500000F056FC81460BE000F052FCA0EB0900BE
:101C6000B0F5803F02D30120BDE8F0872868046901
:101C700004F001000028EFD12868406980B2C8F85C
:101C800000000020F0E72DE9F047064606F11804B1
:101C9000A76AE56A4FF001082AE04FF001097F1EAC
:101CA00004F1140050F8250020B9681C00F0030569
:101CB0004FF00009B9F1000F1AD005EB8501F0686B
:101CC00050F8310000F0004080B904F1140151F8DF
:101CD000250000F0C7F9002104F1140040F8251098
:101CE000681C00F00305A762E56201E04FF0000800
:101CF00017B1B8F1000FD0D10020BDE8F087000087
:101D00007CB504460D4808F0D5FD054685B105F1C2
:101D1000200020600A4828614FF4C06120682B46EB
:101D20004122CDE900010021084609F057FF04E0F7
:101D3000012004490870002020607CBDEC6D010882
:101D400055C300083000002010B504460248006862
:101D500009F06CFC10BD000034000020F0B5044612
:101D60000D4621462E460020A2F1200000270760E4
:101D7000078143810F680FB9086001E03768386058
:101D80003060086803E007891F4407810068002865
:101D9000F9D1F0BD70B504460D460DB9012070BDF6
:101DA000D4F88400102805D129462046FEF7E6FF26
:101DB0000020F4E70120F2E770B5064630680569B7
:101DC00025F01C0500F0A2FD04461348844205D30B
:101DD0001248844202D245F008051AE00F488442B6
:101DE00005D30F48844202D245F00C0511E00C489F
:101DF000844203D30B48844200D20AE0094884425B
:101E000005D30948844202D245F0040501E045F0BB
:101E100010053068056170BD002D3101C00E16023D
:101E20000087930300E1F50580D1F00870B5044602
:101E3000D4F8840010285FD12320C4F88400012145
:101E4000A1652068C06B40F402702168C8632068F7
:101E5000D0F80C01294908432168C1F80C01206819
:101E6000D0F8100140F403102168C1F810010421DA
:101E7000E1662046FEF7FEFF2068006840F008009B
:101E800021680860206805680120FFF7F7FB2068DB
:101E900005602068006840F0040021680860206840
:101EA00005680120FFF7EAFB206805602046FEF781
:101EB0005BFD206800F58050806940F40051206887
:101EC00000F580508161206800F58050806940F005
:101ED0000201206800F580508161206800F5805083
:101EE000C06907490843216801F58051C861232072
:101EF000C4F88400002070BD0120FCE760000200EF
:101F0000C1A001002DE9F0410446D4F88400232843
:101F100051D1C4F88400206800F58050C069274979
:101F20000840216801F58051C861206800F58050A3
:101F3000806920F40051206800F58050816120689C
:101F400000F58050806920F00201206800F5805083
:101F500081612068006820F0040021680860206822
:101F600007680120FFF78AFB206807602046FEF71C
:101F7000FBFC2068006820F00800216808602068E9
:101F800007680120FFF77AFB20680760002508E05A
:101F900004F1480050F82560706840F0004070601F
:101FA0006D1C042DF4D30021A1651020C4F8840019
:101FB0000020BDE8F0810120FBE700003E5FFEFF4E
:101FC00070B504460D463DB9D4F8880040F00100D4
:101FD000C4F88800012070BDD4F88400232835D1CE
:101FE000696BE163012229462046FEF78BFD38B17B
:101FF000D4F8880040F00200C4F888000120EAE725
:1020000000BF00BF00BFBFF34F8F00BF00BF00BFC6
:1020100000BFA06A401CA062A06A042802D3A06A84
:10202000001FA06200BF206800F58050406900F0EA
:10203000040048B10421206800F58050416100216E
:10204000206800F5805041600020C4E70120C2E70D
:1020500010B504460248006809F0E8FA10BD000017
:102060003800002010B5044620460AF09FF810BD45
:1020700070472DE9F04705460E46174698462868F2
:10208000046904F01C044FF4784000EAC6200443BD
:102090004FF4F86000EA8710044344F0020444F06F
:1020A00001041FFA88F0296848612868046100F07B
:1020B00027FA81460BE000F023FAA0EB0900B0F507
:1020C000803F02D30120BDE8F0872868046904F04E
:1020D00001000028EFD100BFF5E700002DE9F04135
:1020E00004460E460127002500BF2548007E012832
:1020F00002D10220BDE8F08101202149087600BF0D
:102100004CF25030FFF73EF80746002F31D1401E09
:102110003060206801280FD1207C6168FEF776FFCF
:102120004CF25030FFF72EF807461648006820F0B2
:102130000400144908601AE0A56812E0217C2846D2
:10214000FEF7FAFE4CF25030FFF71CF807460D4838
:10215000006820F0FA000B4908600FB1356005E017
:102160006D1CD4E902100844A842E7D800BFFEF76E
:1021700011FF00BF00200249087600BF3846B9E7CA
:10218000AC7F0020103C02400348006840F0004053
:102190000149086000207047103C02402DE9F041E1
:1021A00006460F4614461D464FF0010800BF1F4863
:1021B000007E012802D10220BDE8F08101201B49E8
:1021C000087600BF4CF25030FEF7DCFF8046B8F1D5
:1021D000000F23D126B9E1B23846FEF72FFF12E0F7
:1021E000012E04D1A1B23846FEF758FF0BE0022EB3
:1021F00004D121463846FEF765FF04E022462B460F
:102200003846FEF72DFF4CF25030FEF7BBFF8046FC
:102210000748006820F001000549086000BF002061
:102220000249087600BF4046C6E70000AC7F0020A8
:10223000103C024000200949096801F0004159B1F1
:102240000749064A0C3A11600649116003490968BA
:1022500001F0004101B1012070470000103C024034
:1022600023016745AB89EFCD10B50446B4F5807FF7
:1022700015D11148007818B901200F4908700EE0F7
:102280000D480078012803D102200B49087006E0B0
:1022900009480078022802D1032007490870082C59
:1022A00003D16102054800F01BF9022C03D1610340
:1022B000024800F015F910BDE0F6002000100240C1
:1022C00010B5044604480068204020B1024804606C
:1022D0002046FFF7C9FF10BD143C0140F8B5024687
:1022E0000B460025002400200021D6E0012606FA36
:1022F00001F51E6806EA0504AC4274D11E7906F0A9
:102300000306012E04D01E7906F00306022E13D117
:1023100090684F000326BE40B0434F00DE68BE40C9
:1023200030439060506801268E40B0431E79C6F35A
:1023300000168E40304350601E7906F00306032ECF
:1023400009D0D0684F000326BE40B0434F009E68BE
:10235000BE403043D0601E7906F00306022E13D132
:10236000CF0802F1200656F827004E07F70E0F2679
:10237000BE40B0434F07FF0E1E69BE403043CF083A
:1023800002F1200646F8270010684F000326BE40E1
:10239000B0431E7906F003064F00BE403043106084
:1023A0005E6806F44036002E76D000BF0026009608
:1023B0003C4E366846F480463A4F3E603E463668AC
:1023C00006F48046009600BF00BF374E8F0856F8CF
:1023D00027008E07370F0F26BE40B043334EB24260
:1023E00002D1002624E057E0314EB24201D101264D
:1023F0001EE0304EB24201D1022619E02E4EB2420A
:1024000001D1032614E02D4EB24201D104260FE083
:102410002B4EB24201D105260AE02A4EB24201D12A
:10242000062605E0284EB24201D1072600E0082624
:102430008F073F0FBE4030431B4E8F0846F82700E2
:10244000224E3068A0435E6806F4801606B1204331
:102450001E4E3060361D3068A0435E6806F40016DC
:1024600006B12043194E361D3060184E361F3068B5
:10247000A0435E6806F4003606B12043134E361FB3
:102480003060361F3068A0435E6806F4803606B1BF
:1024900020430E4E083E3060491C1029FFF426AF41
:1024A000F8BD0000443802400838014000000240F6
:1024B0000004024000080240000C024000100240EC
:1024C0000014024000180240001C0240083C014079
:1024D000024613690B400BB1012000E00020704759
:1024E00010B5426921EA020302EA010443EA044307
:1024F000836110BD0AB1816101E00B048361704703
:10250000014800687047000068000020014800682A
:1025100070470000107AFF1F0148006870470000F4
:10252000147AFF1F034800680349097808440149E9
:1025300008607047680000207000002010B50D484A
:10254000006840F400700B4908600846006840F4D9
:10255000806008600846006840F4807008600320CE
:1025600000F0DCF80F2000F007F800F05FF8002022
:1025700010BD0000003C02402DE9F04188B0044647
:102580000027B84600BF002001902348006840F0B3
:102590000400214908600846006800F0040001902A
:1025A00000BF00BF02A903A800F08EF9069F1FB963
:1025B00000F0B2F9054602E000F0AEF94500174818
:1025C000B5FBF0F0A0F1010815481649086040F28B
:1025D000E7311448C160C0F80480002101618160C6
:1025E000816100F079FE064696B90E4800F0D6FEED
:1025F00006466EB91E2000F043F8102C07D20022C8
:1026000021461E2000F04CF80748046000E0012637
:10261000304608B0BDE8F0814038024040420F002B
:1026200000080040603300206C00002008B500BFA7
:10263000002000901148006840F480400F49086075
:102640000846006800F48040009000BF00BF00BF53
:1026500000200090081F006840F08050091F0860AB
:102660000846006800F08050009000BF00BF0022C4
:102670000F21901E00F014F808BD000044380240FD
:1026800001460846002809DB00F01F0301229A409A
:1026900043099B0003F1E023C3F8002100BF70470A
:1026A0002DE9F05F80460D461646002703F080FEB8
:1026B000074639462A46334601F00700C0F1070AAB
:1026C000BAF1040F02D94FF0040A01E0C0F1070A81
:1026D000D14600F1040ABAF1070F02D24FF0000A06
:1026E00001E0A0F1030AD4464FF0010A0AFA09FA00
:1026F000AAF1010A0AEA020A0AFA0CFA4FF0010BDF
:102700000BFA0CFBABF1010B0BEA030B4AEA0B04CF
:102710002146404603F054FEBDE8F09F00BF00F0A4
:102720000702064B19684FF6FF031940044B0B4391
:1027300043EA0221014B196000BF70470CED00E035
:102740000000FA0570B504460D460CB9012070BDB5
:102750005848006800F00700A84209D255490D709A
:102760000846006800F00700A84201D00120EEE70B
:10277000207800F0020002281DD1207800F004002B
:10278000042805D14C48006840F4E0504A490860EC
:10279000207800F00800082805D14748006840F478
:1027A0006040454908604448006820F0F000A16896
:1027B000084341490860207800F00100A8B3606830
:1027C000012807D13C4808380068C0F34040B8B938
:1027D0000120BCE76068022802D06068032807D1A6
:1027E000354808380068C0F3406048B90120AEE7BA
:1027F000314808380068C0F3400008B90120A6E756
:102800002D48006820F00300616808432A490860E9
:10281000FFF776FE064609E0FFF772FE801B41F2E5
:102820008831884202D9032091E707E022480068F6
:1028300000F00C006168B0EB810FEDD11D4800681D
:1028400000F00700A84209D91A490D70084600682F
:1028500000F00700A84201D0012078E7207800F0BE
:102860000400042807D11448006820F4E050E1680F
:10287000084311490860207800F00800082808D1B2
:102880000D48006820F46040216940EAC1000A490F
:10289000086000F061F808490968C1F30311074AAC
:1028A000515CC8400649086006480068FFF764FEAE
:1028B00000204CE7003C024008380240386E010816
:1028C000740000206C0000200F2202600D4A126884
:1028D00002F0030242600B4A126802F0F0028260CA
:1028E000084A126802F4E052C260064A126802F412
:1028F0006042D2080261044A126802F007020A60CC
:102900007047000008380240003C0240014800685F
:10291000704700007400002000B5FFF7F7FF04497E
:102920000968C1F38221034A515CC84000BD000020
:1029300008380240486E010800B5FFF7E7FF044978
:102940000968C1F34231034A515CC84000BD000030
:1029500008380240486E01082DE9F04700240025A0
:102960000026A1462548006800F00C0020B104288C
:1029700005D008283AD105E0DFF8849039E0DFF887
:10298000849036E01D48001F006800F03F041B489B
:10299000001F006800F4800078B11A481749091F29
:1029A0000968C1F38811A0FB01700146224600238B
:1029B0003846FDF767FC05460EE011480F49091F30
:1029C0000968C1F38811A0FB01700146224600236B
:1029D0003846FDF757FC05460848001F0068C0F35D
:1029E0000140401C4600B5FBF6F902E0DFF810900C
:1029F00000BF00BF4846BDE8F0870000083802402D
:102A00000024F40000C0A800F8B504460CB9012069
:102A1000F8BD207800F00100002874D0F948006863
:102A200000F00C0004280DD0F648006800F00C00FF
:102A3000082813D1F348001F006800F48000B0F5A7
:102A4000800F0BD1EF4808380068C0F340400028E1
:102A500059D06068002856D10120D9E700BF6068CE
:102A6000B0F5803F08D1E7480838006840F480306E
:102A7000E449083908601EE06068B0F5A02F0DD168
:102A8000E0480838006840F48020DE4908390860D2
:102A90000846006840F4803008600CE0D9480838E7
:102AA000006820F48030D74908390860084600687B
:102AB00020F48020086000BF606890B1FFF720FD1F
:102AC000054606E0FFF71CFD401B642801D90320E2
:102AD0009EE7CC4808380068C0F340400028F1D099
:102AE00011E0FFF70DFD054606E0FFF709FD401B6D
:102AF000642801D903208BE7C24808380068C0F376
:102B000040400028F1D1207800F0020002285FD177
:102B1000BC48006800F00C0058B1BA48006800F0EA
:102B20000C0008281CD1B748001F006800F4800082
:102B3000B0B9B44808380068C0F3400020B1E0687C
:102B4000012801D0012063E7AE480838006820F072
:102B5000F800216940EAC100AA490839086037E055
:102B6000E06800B30120A8490860FFF7C9FC0546EA
:102B700006E0FFF7C5FC401B022801D9032047E708
:102B8000A04808380068C0F340000028F1D09D48F4
:102B90000838006820F0F800216940EAC10099492E
:102BA0000839086014E0002097490860FFF7A8FC86
:102BB000054606E0FFF7A4FC401B022801D90320CC
:102BC00026E7904808380068C0F340000028F1D19B
:102BD000207800F0080008282CD16069A8B10120F5
:102BE0008A490860FFF78CFC054606E0FFF788FC81
:102BF000401B022801D903200AE782486C30006894
:102C0000C0F340000028F1D014E000207F490860A4
:102C1000FFF776FC054606E0FFF772FC401B022832
:102C200001D90320F4E677486C300068C0F3400017
:102C30000028F1D1207800F00400042870D100278A
:102C400070483830006800F0805090B900BF002014
:102C500000906C483830006840F080506949383145
:102C600008600846006800F08050009000BF00BF78
:102C700001276748006800F48070B0B964480068B4
:102C800040F4807062490860FFF73AFC054606E0B0
:102C9000FFF736FC401B022801D90320B8E65C4848
:102CA000006800F480700028F2D000BFA0680128FE
:102CB00008D154486830006840F00100514968313B
:102CC00008601DE0A06805280DD14E4868300068F6
:102CD00040F004004B49683108600846006840F045
:102CE000010008600CE047486830006820F00100EF
:102CF0004449683108600846006820F00400086014
:102D000000BFA068A8B1FFF7FBFB054609E0FFF78D
:102D1000F7FB401B41F28831884202D9032077E655
:102D200026E0384868300068C0F340000028EED044
:102D300013E0FFF7E5FB054608E0FFF7E1FB401B6A
:102D400041F28831884201D9032061E62D4868307C
:102D50000068C0F340000028EFD1012F07D12948B7
:102D60003830006820F0805026493831086000BFB4
:102D7000A069002845D02348006800F00C0008280E
:102D80005DD0A069022845D100201F490866FFF7E1
:102D9000B7FB054606E0FFF7B3FB401B022801D94D
:102DA000032035E6174808380068C0F34060002863
:102DB000F1D1D4E907010843616A40EA8111012297
:102DC000A06AC2EB500041EA00412C20005D41EABC
:102DD00000600C49091F086001200B490866FFF7D5
:102DE0008FFB054606E0FFF78BFB401B022801D94D
:102DF00003200DE6034808380068C0F3406000284F
:102E0000F1D049E00838024000004742800E4742B6
:102E100000700040002021490866FFF771FB05465D
:102E200006E0FFF76DFB401B022801D90320EFE508
:102E30001B480068C0F340600028F2D12CE0A06974
:102E4000012800D1E4E51648001D0668A0690128A4
:102E500020D006F48001E06981421BD106F03F01D9
:102E6000206A814216D147F6C0703040616AB0EBEB
:102E7000811F0FD106F440310122A06AC2EB50003D
:102E8000B1EB004F06D106F070612C20005DB1EB74
:102E9000006F01D00120BBE50020B9E500004742EA
:102EA0000038024010B504460CB9012010BD606A1C
:102EB00038B96068B0F5827F00D105E00021E1619A
:102EC00002E00021216161610021A16294F85100BA
:102ED00028B9002084F85000204600F047F802206E
:102EE00084F851002068006820F0400021680860E4
:102EF000A08800F48270218901F404410843A1896B
:102F000001F400610843217C01F002010843217DA6
:102F100001F001010843218B01F400710843217F76
:102F200001F0380108432021095D01F080010843C8
:102F3000218D01F400510843216808600421A06933
:102F400001EA104094F8241001F0100108432168B0
:102F500048602068C06920F400602168C8610020D2
:102F60006065012084F8510000209FE710B586B00D
:102F70000446142101A8FDF7F0F91B492068884296
:102F80002FD100BF002000901848006840F4805006
:102F9000164908600846006800F48050009000BFA1
:102FA00000BF00BF0020009010481438006840F0B7
:102FB00002000E49143908600846006800F002005B
:102FC000009000BF00BF3820019002200290012035
:102FD0000390032004900520059001A90448FFF701
:102FE0007DF906B010BD00000030014044380240B9
:102FF000000402402DE9FF5F0446884691461D46C5
:103000000E9E012002900020019000BF94F8500015
:10301000012803D1022004B0BDE8F09F012084F80C
:10302000500000BFFFF76CFA074694F851B0606893
:103030000390AA46BBF1010F0BD00398B0F5827F35
:1030400004D1A06810B9BBF1040F02D00220019096
:10305000DBE0B8F1000F03D0B9F1000F00D015B9D3
:1030600001200190D1E094F85100042802D00520FD
:1030700084F8510000206065C4F83890E587A58782
:10308000C4F83080E586A586206460642068006806
:1030900000F04000402805D02068006840F0400063
:1030A00021680860E068B0F5006F4AD1606810B12F
:1030B000BAF1010F09D1206B00882168C860206B2C
:1030C000801C2063E08E401EE08633E0206880682C
:1030D00000F00200022810D1E08E70B102980128A1
:1030E0000BD1206B00882168C860206B801C206396
:1030F000E08E401EE086002002902068806800F08C
:10310000010068B1E08F58B12068C068A16B0880E9
:10311000A06B801CA063E08F401EE087012002901E
:10312000FFF7EEF9C01BB04204D3701C10B10320AE
:1031300001906AE0E08E0028C8D1E08F0028C5D158
:103140004AE0606810B1BAF1010F09D1206B007834
:1031500021680873206B401C2063E08E401EE086CF
:1031600034E02068806800F00200022810D1E08E70
:1031700070B1029801280BD1206B00782168087388
:10318000206B401C2063E08E401EE08600200290F1
:103190002068806800F0010068B1E08F58B12068B5
:1031A000C068A16B0870A06B401CA063E08F401E3C
:1031B000E08701200290FFF7A3F9C01BB04201D3C2
:1031C000701C00B916B9032001901EE0E08E0028A3
:1031D000C7D1E08F0028C4D13A463146204602F0DC
:1031E000A1FA20B101200190202060650DE0A068C7
:1031F00050B900BF002000902068C068009020688F
:103200008068009000BF00BF00BF012084F851001B
:1032100000BF002084F8500000BF0198FBE6704713
:103220007047000030B502460B4600BF92F83C00E4
:10323000012801D1022030BD012082F83C0000BFEE
:10324000022082F83D00106844681068816824F00C
:1032500070041868044310684460184D1068A84250
:103260001BD01068B0F1804F17D0154D1068A842E0
:1032700013D0144D1068A8420FD0134D1068A84207
:103280000BD0124D1068A84207D0114D1068A8420B
:1032900003D0104D1068A84205D121F08001586874
:1032A000014310688160012082F83D0000BF0020CA
:1032B00082F83C0000BF00BFBDE7000000000140F5
:1032C0000004004000080040000C004000040140E1
:1032D000004001400018004010B504460CB9012020
:1032E00010BD94F83D0028B9002084F83C00204629
:1032F00000F026F8022084F83D00211D206802F02D
:1033000037FB012084F8460000BF84F83E0001210D
:103310003F200155402001554120015500BF00BF0D
:10332000012084F8420043200155442001554520E6
:10333000015500BF012084F83D000020D0E70000C7
:1033400008B50168B1F1804F0FD100BF0021009195
:103350001049096841F001010E4A116011460968DF
:1033600001F00101009100BF13E00B4A0168914296
:103370000FD100BF002100910649096841F0020108
:10338000044A11601146096801F00201009100BF72
:1033900000BF08BD4038024000040040014691F8DB
:1033A0003D00012801D001207047022081F83D0036
:1033B0000868C06840F001000B68D8601A4B0868C4
:1033C00098421BD00868B0F1804F17D0174B08689F
:1033D000984213D0164B086898420FD0154B0868D6
:1033E00098420BD0144B0868984207D0134B0868DA
:1033F000984203D0124B086898420CD10868806844
:1034000000F00702062A0CD00868006840F00100AE
:103410000B68186005E00868006840F001000B6860
:1034200018600020C0E700000000014000040040D8
:1034300000080040000C0040000401400040014032
:10344000001800402DE9F04104460D46002700BF5A
:1034500094F83C00012802D10220BDE8F08101204F
:1034600084F83C0000BF022084F83D002068866894
:1034700026F0770626F47F46206886602868502864
:1034800033D00CDC202850D004DC00284BD010288E
:1034900051D149E0302849D040284CD139E060284A
:1034A0002DD0702807D0B0F5805F03D0B0F5005F55
:1034B00041D10DE041E0D5E902136A68206802F0CD
:1034C000D4FA2068866846F077062068866034E083
:1034D000D5E902136A68206802F0C7FA206880689C
:1034E00040F480402168886027E0EA6869682068C5
:1034F00002F0ACFB5021206802F0C2FA1DE0EA683D
:103500006968206802F0B5FB6021206802F0B8FA13
:1035100013E0EA686968206802F098FB402120689F
:1035200002F0AEFA09E000BF00BF00BF29682068C2
:1035300002F0A6FA01E0012700BF00BF012084F8D5
:103540003D0000BF002084F83C0000BF384684E7FF
:103550002DE9F04104460D4614B90120BDE8F08183
:1035600094F83D0028B9002084F83C00204600F083
:1035700053F8022084F83D002068806844F2070177
:10358000884321688860211D206802F0F1F92068D5
:10359000D0F80880206886692068076A286840EAB1
:1035A000080840F203308643A969A86840EA012070
:1035B000064340F60C4086434FF2F0008643E9692B
:1035C000E86840EA0120064328690001296A40EAC8
:1035D0000130064327F0220727F0880769696868E9
:1035E00040EA011007432068C0F80880206886611F
:1035F00020680762012084F8460084F83E0001211B
:103600003F200155012084F842004320015501204C
:1036100084F83D000020A1E710B586B004461421CF
:1036200001A8FCF79AFE35492068884231D100BFD5
:10363000002000903248006840F0010030490860E6
:103640000846006800F00100009000BF00BF00BF06
:10365000002000902A481438006840F010002849E3
:10366000143908600846006800F01000009000BFA0
:1036700000BF4FF4206001900220029001200390CF
:10368000002004900120059001A91E48FEF726FEA7
:1036900032E01D49206888422ED100BF00200090F2
:1036A0001748006840F002001549086008460068A5
:1036B00000F00200009000BF00BF00BF002000909B
:1036C0000F481438006840F004000D4914390860B0
:1036D0000846006800F00400009000BF00BFC02052
:1036E0000190022002900020039004900320059096
:1036F00001A90648FEF7F2FD06B010BD000001402A
:10370000443802400010024000040140000802401A
:103710002DE9F04304460D4694F83E603F20075DD6
:1037200094F84280432010F804906DB9012E02D124
:10373000B8F1010F02D00120BDE8F083022084F827
:103740003E0084F8420025E0042D0CD1012F02D167
:10375000B9F1010F01D00120EEE702213F20015510
:103760004320015516E0012E07D1012F05D1B8F1F4
:10377000010F02D1B9F1010F01D00120DCE70220D5
:1037800084F83E0002213F200155022084F84200C7
:103790004320015515B1042D0CD105E00122002173
:1037A000206802F051F910E001220421206802F0A3
:1037B0004BF90AE001220021206802F045F90122BC
:1037C0000421206802F040F900BF00BF20680068B3
:1037D00040F00100216808600020ADE7704710B597
:1037E000044620680069C0F34000D8B12068C06872
:1037F000C0F34000B0B16FF0020021680861012001
:1038000020772068806900F0030018B12046FFF798
:10381000E5FF05E0204600F005F9204600F0B9F983
:103820000020207720680069C0F38000D8B12068AC
:10383000C068C0F38000B0B16FF004002168086177
:10384000022020772068806900F4407018B120467B
:10385000FFF7C4FF05E0204600F0E4F8204600F042
:1038600098F90020207720680069C0F3C000D8B123
:103870002068C068C0F3C000B0B16FF008002168D4
:103880000861042020772068C06900F0030018B1A7
:103890002046FFF7A3FF05E0204600F0C3F82046CE
:1038A00000F077F90020207720680069C0F300104D
:1038B000D8B12068C068C0F30010B0B16FF010003C
:1038C00021680861082020772068C06900F44070F2
:1038D00018B12046FFF782FF05E0204600F0A2F86D
:1038E000204600F056F9002020772068006900F09B
:1038F000010058B12068C06800F0010030B16FF0DD
:10390000010021680861204600F01EFA2068006965
:10391000C0F3C01058B12068C068C0F3C01030B107
:103920006FF08000216808612046FFF778FC20686E
:103930000069C0F3801058B12068C068C0F38010DF
:1039400030B16FF0400021680861204600F008FAAD
:1039500020680069C0F3401058B12068C068C0F307
:10396000401030B16FF02000216808612046FFF759
:1039700057FC10BD10B586B00446142101A8FCF711
:10398000ECFC2068B0F1804F1FD100BF00200090F8
:103990002048006840F001001E49086008460068A1
:1039A00000F00100009000BF00BF4FF40040019004
:1039B0000220029000200390032004900120059033
:1039C00001A91548FEF78AFC21E0144920688842C5
:1039D0001DD100BF002000900E48006840F002009A
:1039E0000C4908600846006800F00200009000BF23
:1039F00000BF0120019002200290002003900320CC
:103A000004900220059001A90548FEF767FC06B066
:103A100010BD0000303802400000024000040040A9
:103A20000004024070472DE9F04104460D46164659
:103A3000002700BF94F83C00012802D10220BDE815
:103A4000F081012084F83C0000BF36B1042E1BD069
:103A5000082E31D00C2E5ED145E02946206802F0B8
:103A600019F82068806940F00800216888612068A2
:103A7000806920F0040021688861206880692969D4
:103A800008432168886148E02946206802F03AF836
:103A90002068806940F4006021688861206880693E
:103AA00020F480602168886120688069296940EA83
:103AB00001202168886130E02946206802F060F822
:103AC0002068C06940F008002168C8612068C069AA
:103AD00020F004002168C8612068C0692969084392
:103AE0002168C86119E02946206802F085F820683D
:103AF000C06940F400602168C8612068C06920F492
:103B000080602168C8612068C069296940EA012095
:103B10002168C86101E0012700BF00BF00BF00208D
:103B200084F83C0000BF384689E710B504460CB95C
:103B3000012010BD94F83D0028B9002084F83C0015
:103B4000204600F025F8022084F83D00211D206861
:103B500001F00EFF012084F8460000BF84F83E000B
:103B600001213F200155402001554120015500BF52
:103B700000BF012084F84200432001554420015534
:103B80004520015500BF012084F83D000020D0E70A
:103B90007047704770B504460D4615B994F83E005D
:103BA0000BE0042D02D13F20005D06E0082D02D17C
:103BB0004020005D01E04120005D012801D001208E
:103BC00070BD1DB9022084F83E000EE0042D03D123
:103BD00002213F20015508E0082D03D10221402099
:103BE000015502E0022141200155012229462068A9
:103BF00001F02AFF23492068884203D02249206827
:103C0000884201D1012000E0002028B12068406CEA
:103C100040F40040216848641A49206888421BD05B
:103C20002068B0F1804F17D018492068884213D01F
:103C30001749206888420FD01649206888420BD067
:103C400011492068884207D013492068884203D070
:103C50001249206888420CD12068806800F007066D
:103C6000062E0CD02068006840F001002168086032
:103C700005E02068006840F001002168086000202D
:103C80009EE70000000001400004014000040040E5
:103C900000080040000C00400040014000180040B7
:103CA00030B504460D4600222946206801F0CCFEBE
:103CB00023492068884203D022492068884201D1E4
:103CC000012000E0002090B100BF2068006A41F2AE
:103CD0001111084050B92068006A8910084028B9BD
:103CE0002068406C20F400402168486400BF00BF99
:103CF0002068006A41F21111084050B92068006A3A
:103D00008910084028B92068006820F00100216867
:103D1000086000BF1DB9012084F83E000EE0042DAC
:103D200003D101213F20015508E0082D03D10121D5
:103D30004020015502E0012141200155002030BD05
:103D4000000001400004014010B50446034920680A
:103D5000884201D1FEF7E6FB10BD000000080040DC
:103D60007047F8B504460E46174694F83E002028E2
:103D700036D106B10FB90120F8BD00BF94F83C0060
:103D8000012801D10220F7E7012084F83C0000BFA0
:103D900020633A463146204602F048FA0546EDB91E
:103DA000206B012819D100BF002000902068006816
:103DB000009020684068009000BF00BF00BF00BFB7
:103DC00021680C3151E8001F41F0100021680C31CE
:103DD00041E80002002AF3D100E001252846CBE7A4
:103DE0000220C9E770B504460D467F48844277D16A
:103DF00000BF002084F83C0000BF7C4805804FF4E1
:103E00000071801CFCF7A9FA2A467949A1F50070D7
:103E1000FCF77CFA4FF4007275497348FFF7A1FF75
:103E2000724890F802020106704890F8030241EAD5
:103E300000416E4890F8040241EA00206B4991F875
:103E4000051208430206694890F802020106674815
:103E500090F8030241EA0041644890F8040241EA04
:103E60000020624991F80512084300F47F4042EABD
:103E700000225E4890F8020201065C4890F80302B6
:103E800041EA0041594890F8040241EA00215748AC
:103E900090F80502014301F47F0042EA10225348E2
:103EA00090F802020106514890F8030241EA0041ED
:103EB0004E4890F8040241EA00204C4991F805125E
:103EC000084342EA10604B4908604B48096841606A
:103ED0002A464749494804F0E7F808B911F0ACF818
:103EE0004748844217D100BF002084F83C0000BF3F
:103EF000444805804FF40071801CFCF72EFA2A46D6
:103F00004149A1F50070FCF701FA4FF400723E49F7
:103F10003B48FFF726FF3D4884421DD100BF0020EB
:103F200084F83C0000BF3A4805804FF40071801CC3
:103F3000FCF713FA2A463749A1F50070FCF7E6F9B9
:103F400035480078012801D1344908704FF40072D7
:103F500030492E48FFF705FF3148844222D100BF87
:103F6000002084F83C0000BF2E4805804FF400710B
:103F7000801CFCF7F2F92A462B49A1F50070FCF7EA
:103F8000C5F92A480078012801D1294908704FF461
:103F9000007225492248FFF7E4FE4FF400712248E1
:103FA000FCF7DBF9234884421DD100BF002084F8D0
:103FB0003C0000BF204805804FF40071801CFCF7D6
:103FC000CCF92A461D49A1F50070FCF79FF91C4861
:103FD0000078012801D11B4908704FF4007217497D
:103FE0001448FFF7BEFE70BDD42E002076240020BA
:103FF0007826002050000020747F002000000E086A
:104000004C2E00206C0600206E0800205C2F002043
:1040100070120020721400200B00002011000020FC
:10402000902E0020741E0020762000200800002022
:104030000E000020182F002072180020741A002093
:10404000090000200F00002010B5044617488442E4
:1040500013D100BF002084F83C0000BF2068006836
:1040600000F00400042802D1C043216808604FF426
:1040700000720F490D48FFF774FE0E48844213D1B9
:1040800000BF002084F83C0000BF2068006800F0FA
:104090000400042802D1C043216808604FF4007274
:1040A00005490448FFF75DFE10BD0000902E00207A
:1040B00076200020182F0020741A00202DE9F84FD8
:1040C0000446206805682068C668206847694FF084
:1040D0000009CA4605F00F09B9F1000F0AD105F031
:1040E000200038B106F0200020B1204601F00CFF7E
:1040F000BDE8F88FB9F1000F7CD007F0010018B9C6
:1041000006F49070002875D005F0010030B106F477
:10411000807018B1206C40F00100206405F00400AC
:1041200030B107F0010018B1206C40F002002064AB
:1041300005F0020030B107F0010018B1206C40F02A
:104140000400206405F0080048B106F0200010B912
:1041500007F0010018B1206C40F008002064206CCA
:10416000002846D005F0200028B106F0200010B14C
:10417000204601F0C9FE20684069C0F3801A206C17
:1041800000F0080010B9BAF1000F2DD0204601F060
:1041900062FE2068406900F04000402820D100BF46
:1041A00000BF2168143151E8001F21F04000216850
:1041B000143141E80002002AF3D100BFA06B50B1D6
:1041C0007548A16B0865A06BFDF764F888B1A06B1A
:1041D000016D88470DE02046FFF736FF09E009E052
:1041E0002046FFF731FF04E02046FFF72DFF0020B7
:1041F00020647DE7206B012876D105F010000028AF
:1042000072D006F010000028FAD000BF0020009005
:1042100020680068009020684068009000BF00BFE0
:104220002068406900F0400040285ED1A06B006823
:1042300040681FFA80F8B8F1000F54D0A08D4045B7
:1042400051DDA4F82E80A06BC069B0F5807F43D00B
:1042500000BF00BF21680C3151E8001F21F48070BD
:1042600021680C3141E80002002AF3D100BF00BFF1
:1042700000BF2168143151E8001F21F001002168BE
:10428000143141E80002002AF3D100BF00BF00BF93
:104290002168143151E8001F21F0400021681431D9
:1042A00041E80002002AF3D100BF202084F83E003C
:1042B0000020206300BF00BF21680C3151E8001FBF
:1042C00021F0100021680C3141E80002002AF3D1EE
:1042D00000BFA06BFCF788FFA08DE28D801A81B231
:1042E0002046FFF77FFD03E740E0A08DE18D401AF7
:1042F0001FFA80F8E08DC0B3B8F1000F35D000BFD1
:1043000000BF21680C3151E8001F21F49070216832
:104310000C3141E80002002AF3D100BF00BF00BF0A
:104320002168143151E8001F21F001002168143187
:1043300041E80002002AF3D100BF202084F83E00AB
:104340000020206300BF00BF21680C3151E8001F2E
:1043500021F0100021680C3141E80002002AF3D15D
:1043600000BF41462046FFF73DFDC1E605F0800055
:1043700030B106F0800018B1204601F0BFFFB7E66B
:1043800005F0400030B106F0400018B1204601F0C1
:1043900098FDADE600BFABE6BD5C000810B5044675
:1043A0000CB9012010BDA06900B100E000BF94F875
:1043B0003D0028B9002084F83C00204600F028F891
:1043C000242084F83D002068C06820F40050216853
:1043D000C860204601F014FE2068006920F4904077
:1043E000216808612068406920F02A00216848613E
:1043F0002068C06840F400502168C8600020206434
:10440000202084F83D0084F83E000020CAE7000028
:1044100010B586B00446142101A8FBF79EFFFD49A4
:10442000206888427BD100BF00200090FA480068D5
:1044300040F40020F84908600846006800F40020B5
:10444000009000BF00BF00BF00200090F24810386D
:10445000006840F00400F049103908600846006820
:1044600000F00400009000BF00BF4FF440600190D6
:104470000220029000200390032004900820059061
:1044800001A9E648FDF72AFFE548E649086040052E
:1044900048600021E3488160C1604FF480610161A0
:1044A000002141618161C1614FF44031016200210D
:1044B0004162FDF723F808B1FCF73CFD00BFD94885
:1044C000A063846300BFD6483030D74908604FF0FE
:1044D000006048604021D44881600021C1604FF4F1
:1044E00080610161002141618161C1614FF440310E
:1044F000016200214162FDF701F808B1FCF71AFDE5
:1045000000BFC9486063846300BF002205213420D6
:10451000FEF7C6F83420FEF7B3F83AE2FFE7C349E6
:10452000206888427ED100BF00200090BA48006811
:1045300040F48010B84908600846006800F4801014
:10454000009000BF00BF00BF00200090B2481038AC
:10455000006840F00400B04910390860084600685F
:1045600000F00400009000BF00BF00BF00200090DA
:104570000846006840F0080008600846006800F03F
:104580000800009000BF00BF881401900220029034
:1045900000200390032004900820059001A99F4863
:1045A000FDF79CFE04200190022002900020039061
:1045B000032004900820059001A99D48FDF78EFE78
:1045C000974878309B4908604FF000604860402170
:1045D000984881600021C1604FF480610161002131
:1045E00041618161C1614FF440310162002141624A
:1045F000FCF784FF08B1FCF79DFC00BF8D486063A9
:10460000846300BF864830388B490860C005486025
:10461000002189488160C1604FF4806101610021FF
:10462000416100E019E08161C1614FF440310162F4
:1046300000214162FCF762FF08B1FCF77BFC00BF80
:104640007D48A063846300BF002205213520FEF76A
:1046500027F83520FEF714F89BE178492068884256
:1046600078D100BF002000906B48001D006840F02A
:1046700010006949091D08600846006800F0100034
:10468000009000BF00BF00BF0020009062481038BB
:10469000006840F001006049103908600846006871
:1046A00000F00100009000BF00BF4FF4C060019017
:1046B0000220029000200390032004900720059020
:1046C00001A95F48FDF70AFE5E485F4908604FF0A8
:1046D0000060486000215C488160C1604FF48061E7
:1046E0000161002141618161C16101624162FCF7A8
:1046F00005FF08B1FCF71EFC00BF5348A0638463AC
:1047000000BF50487830514908604FF00060486061
:1047100040214E4881600021C1604FF480610161F9
:10472000002141618161C16101624162FCF7E6FEE5
:1047300008B1FCF7FFFB00BF44486063846300BF1F
:10474000002205212520FDF7ABFF2520FDF798FF6E
:104750001FE1FFE73E49206888427FD100BF00206B
:1047600000902D48006840F400302B49086008464E
:10477000006800F40030009000BF00BF00BF0020C0
:10478000009025481038006840F008002249103990
:1047900008600846006800F00800009000BF00BFF5
:1047A00060200190022002900020039003200490DA
:1047B0000720059001A91E48FDF790FD18484830D4
:1047C000244908604FF00060486000212148816062
:1047D000C1604FF480610161002141618161C1616B
:1047E0004FF44031016200214162FCF787FE08B1BD
:1047F000FCF7A0FB00BF1748A063846300BF084814
:104800006030154908604FF0006048604021124850
:10481000816024E0004C0040403802400008024023
:1048200040600240A02F00200030002000500040D7
:10483000000C024060300020C03000200010014019
:1048400000000240406402402031002080310020FE
:1048500000440040E03100204032002020E00021F0
:10486000C1604FF480610161002141618161C161DA
:104870004FF44031016200214162FCF73FFE08B174
:10488000FCF758FB00BF44486063846300BF00220C
:1048900005212620FDF704FF2620FDF7F1FE78E034
:1048A0003E492068884274D100BF002000903C48F7
:1048B000006840F480203A4908600846006800F427
:1048C0008020009000BF00BF00BF0020009034484F
:1048D0001038006840F00800314910390860084677
:1048E000006800F00800009000BF00BF4FF4407067
:1048F00001900220029001200390032004900720E1
:10490000059001A92748FDF7E9FC274827490860D9
:104910004FF000604860002124488160C1604FF47E
:1049200080610161002141618161C1610162416277
:10493000FCF7E4FD08B1FCF7FDFA00BF1B48A063DB
:10494000846300BF18483030194908604FF0006098
:1049500048604021164881600021C1604FF48061A9
:104960000161002141618161C16101624162FCF725
:10497000C5FD08B1FCF7DEFA00BF0D486063846333
:1049800000BF002205212720FDF78AFE2720FDF722
:1049900077FE06B010BD0000403200200048004005
:1049A00040380240000C024028600240A032002043
:1049B0000033002070477047F7B50446154694F859
:1049C0003D00202846D1019800B10DB90120FEBD5F
:1049D00000BF94F83C00012801D10220F7E7012034
:1049E00084F83C0000BF01982062A584E584002083
:1049F0002064212084F83D001748616BC863174884
:104A0000616B08641648616BC8640020616B0865BF
:104A100001AE23681A1D31682B46606BFCF7E4FD7C
:104A20006FF040002168086000BF002084F83C005F
:104A300000BF00BF00BF2168143151E8001F41F0E2
:104A400080002168143141E80002002AF3D100BF40
:104A50000020BCE70220BAE7F15D0008495E0008CB
:104A6000D15C000810B504460848844204D10122F4
:104A700011460748FDF73EFD0648844204D1012255
:104A800010210348FDF736FD10BD0000902E0020D8
:104A9000000C0240182F0020704700BFFEE738B519
:104AA0000446002000906A46012163692068984707
:104AB000002802DA6FF0040038BD6A4601216369FC
:104AC00020689847002802DA6FF00400F4E70098A5
:104AD00000F0040008B90120EEE76A46002163698E
:104AE00020689847002802DA6FF00400E4E7009895
:104AF00000F48050B0F5805F1FD0009800F40050A3
:104B0000B0F5005F07D1009800F48070B0F5807FA9
:104B100001D10220D0E7009800F40050B0F5005F0A
:104B200001D10320C8E7009800F48070B0F5807FC1
:104B300001D10420C0E70520BEE76A461F21636952
:104B400020689847002802DA6FF00400B4E7009864
:104B500000F4805008B90620AEE7009800F01C0071
:104B6000182801D10220A7E7009800F01C000828AF
:104B700001D10320A0E7009800F01C00142801D107
:104B8000042099E7052097E7F8B5044600270020A0
:104B90000090002500266068002855D1A06808B163
:104BA000A068804720202060002513E06A4612217B
:104BB000284663699847002802DA6FF0040608E087
:104BC000009800F01F00A84202D12560002603E0F3
:104BD00000BF6D1C1F2DE9D900BF20681F2801D917
:104BE0006FF0020656BB4FF4004200212369206893
:104BF0009847002826DB6A460021636920689847A9
:104C000000281CDBA0698047074612E0A0698047A6
:104C1000C01BB0F5FA7F09D86A4600216369206895
:104C20009847002805DA6FF0040607E06FF00106E8
:104C300004E0009800F400400028E7D104E06FF0A1
:104C4000040601E06FF003065EB9A06980470746DD
:104C500000BFA0698047C01BB0F5FA6FF9D90120E9
:104C600060603046F8BD02462AB1C86818B188684D
:104C700008B1086910B94FF0FF30704708689060BC
:104C80004B68D360CB6853618B6813610B69936188
:104C90000020F2E708B500BF002000903648006809
:104CA00040F40010344908600846006800F4001021
:104CB000009000BF00BF00BF0020009008460068C1
:104CC00040F4800008600846006800F4800000900E
:104CD00000BF00BF002205210B20FDF7E1FC0B20E7
:104CE000FDF7CEFC002205210C20FDF7D9FC0C209D
:104CF000FDF7C6FC002205210D20FDF7D1FC0D209B
:104D0000FDF7BEFC002205210E20FDF7C9FC0E2098
:104D1000FDF7B6FC002205210F20FDF7C1FC0F2096
:104D2000FDF7AEFC002205211020FDF7B9FC102094
:104D3000FDF7A6FC002205211120FDF7B1FC112092
:104D4000FDF79EFC002205212F20FDF7A9FC2F2056
:104D5000FDF796FC002205213A20FDF7A1FC3A2040
:104D6000FDF78EFC002205214620FDF799FC462028
:104D7000FDF786FC08BD00003038024000B5ABB03E
:104D80001C22244924A8FBF7C1FA002124A806F01C
:104D9000A9FC214908601C221E491C311DA8FBF7F3
:104DA000B5FA00211DA806F09DFC1C4908601C22D4
:104DB0001849383116A8FBF7A9FA002116A806F001
:104DC00091FC174908601C22124954310FA8FBF7C7
:104DD0009DFA00210FA806F085FC124908601C22EC
:104DE0000C49703108A8FBF791FA002108A806F0D9
:104DF00079FC0D4908601C2206498C3101A8FBF79B
:104E000085FA002101A806F06DFC084908602BB066
:104E100000BD0000446D01081400002018000020AF
:104E20001C0000202000002024000020280000207A
:104E300000B587B0142102A8FBF78FFA00BF00204D
:104E400001909E48006840F010009C4908600846A8
:104E5000006800F01000019000BF00BF00BF0020FC
:104E600001900846006840F080000860084600682D
:104E700000F08000019000BF00BF00BF0020019043
:104E80000846006840F0040008600846006800F02A
:104E90000400019000BF00BF00BF00200190084641
:104EA000006840F0010008600846006800F001005A
:104EB000019000BF00BF00BF0020019008460068BD
:104EC00040F0020008600846006800F0020001900F
:104ED00000BF00BF00BF002001900846006840F0FE
:104EE000080008600846006800F00800019000BF54
:104EF00000BF012211467248FDF7FCFA0122C621CB
:104F00007048FDF7F7FA012247F283016E48FDF77A
:104F1000F1FA00224FF4F1416C48FDF7EBFA01225F
:104F200048F211016948FDF7E5FA012211026848CB
:104F3000FDF7E0FA0C20029000200390012004907D
:104F400002A96148FDF7CAF90120029003900020F0
:104F500004900120059002A95948FDF7BFF90620E9
:104F60000290012003900490059002A95548FDF796
:104F7000B5F94FF4E14002900120039004900590B0
:104F800002A95148FDF7AAF94FF4807002904FF43E
:104F9000041003900120049002A94B48FDF79EF9EC
:104FA0004FF4804002904FF4881003900120049049
:104FB00002A94448FDF792F94FF4F0400290012015
:104FC0000390002004900320059002A93F48FDF7BC
:104FD00085F948F29100029001200390049003208B
:104FE000059002A93948FDF779F94FF44070029015
:104FF000002003900120049002A93148FDF76EF9CA
:105000004FF48070029001200390049003200590DB
:1050100002A92F48FDF762F94FF4C050029000201A
:1050200003900120049002A92948FDF757F90A20AE
:1050300002904FF4041003900120049002A9234829
:10504000FDF74CF9C020029001200390049003204A
:10505000059002A91B48FDF741F901200290039039
:1050600004900320059002A91748FDF737F90220A4
:10507000029001200390022004900320059002A9D1
:105080001148FDF72BF9002205210720FDF708FB49
:105090000720FDF7F5FA002205210920FDF700FBA6
:1050A0000920FDF7EDFA002205211720FDF7F8FA97
:1050B0001720FDF7E5FA07B000BD000030380240C8
:1050C000000802400004024000100240000C0240B0
:1050D0000000024000B58BB0C02097490870A8209E
:1050E0004870012088705820C870FF2093490870CC
:1050F000487088700020C870C02091490870A820AE
:105100004870012088701D20C87000200A90042279
:105110000AA98C4802F0BEFF9DF82800C0280CD1D7
:105120009DF82800844908709DF8290048709DF872
:105130002A0088709DF82B00C870002108460FF0E7
:105140005BFC7D48007800067B49497840EA0140D5
:105150007949897840EA01207749C97808430206ED
:105160007548007800067449497840EA0140724960
:10517000897840EA01207049C978084300F47F40EB
:1051800042EA00226C48007800066B49497840EA00
:1051900001416948807841EA00206749C97808439D
:1051A00000F47F0042EA102263480078010662485A
:1051B000407841EA00416048807841EA00205E4939
:1051C000C978084342EA10605F4908605B4800788C
:1051D00000065A49497840EA01405849897840EA2E
:1051E00001205649C9780843020654480078000651
:1051F0005249497840EA01405049897840EA012003
:105200004E49C978084300F47F4042EA00224B48E7
:10521000007800064949497840EA014147488078CA
:1052200041EA00204549C978084300F47F0042EA7A
:1052300010224248007801064048407841EA004187
:105240003E48807841EA00203C49C978084342EA58
:1052500010603E4908603A480078000638494978AD
:1052600040EA01403649897840EA01203449C9784A
:10527000084302063248007800063149497840EA7E
:1052800001402F49897840EA01202D49C978084317
:1052900000F47F4042EA00222948007800062849AD
:1052A000497840EA01412648807841EA00202449B3
:1052B000C978084300F47F0042EA102220480078B1
:1052C00001061F48407841EA00411D48807841EAC4
:1052D00000201B49C978084342EA10601C49086055
:1052E0001C481D4900221A4BCDE900210290174AA3
:1052F00015491A4805F02AFB184805F0AFFE174873
:1053000090F83100C0F3800018B1144806F008F896
:1053100002E0124805F0A8FE1149104805F018FFF8
:105320001C22104903A8FAF7F1FF0C4903A806F064
:10533000D9F90BB000BD00005C0000206000002027
:105340006400002000000E085000002054000020DF
:1053500058000020F14B0108BD7F0008747F002039
:10536000E17D0008146E010810B50F480F49086070
:105370004FF48270486000210C488160C1600221B6
:10538000016101214161490281613821C16100212E
:105390000162416281620A21C162FDF783FD08B1A9
:1053A000FBF7C8FD10BD000000300140D42C0020E8
:1053B00000B58BB0242102A8FAF7CFFF002000909F
:1053C00001901848184908600020486000211648DC
:1053D00081604FF6FF71C16000210161416181610F
:1053E00003200290002003900120049000200590EB
:1053F0000690079001200890002009900A9002A9C9
:105400000948FEF7A5F808B1FBF794FD00200090CD
:10541000019069460448FDF705FF08B1FBF78AFDD6
:105420000BB000BD000001402C2D002000B58DB058
:10543000002009900A900B900C90079008901C2176
:105440006846FAF78AFF4FF080401F490860002045
:10545000486000211C4881607721C1600021016102
:105460008161FDF739FF08B1FBF764FD4FF480500F
:10547000099009A91448FDF7E5FF08B1FBF75AFDAB
:105480001148FEF752FB08B1FBF754FD00200790CE
:10549000089007A90C48FDF7C5FE08B1FBF74AFDC7
:1054A000602000903C200190002002900490002297
:1054B00069460548FEF7B7FA08B1FBF73BFD02481D
:1054C000FEF758FA0DB000BD742D002000B58DB068
:1054D000002009900A900B900C90079008901C21D6
:1054E0006846FAF73AFF22482249086036204860A9
:1054F0000021204881604FF4B971C1600021016131
:105500008161FDF7E9FE08B1FBF714FD4FF480500F
:10551000099009A91748FDF795FF08B1FBF70AFDA7
:105520001448FEF702FB08B1FBF704FD00200790CA
:10553000089007A90F48FDF775FE08B1FBF7FAFCC4
:10554000602000905C2001900020029004900822CE
:1055500069460848FEF767FA08B1FBF7EBFC054817
:10556000FDF71CFF0348FEF705FA0DB000BD000073
:1055700000040040BC2D002000B58BB0242102A8FF
:10558000FAF7EBFE002000900190184818490860D7
:10559000002048600021164881604FF6FF71C1600D
:1055A000002101614161816103200290002003908C
:1055B000012004900020059006900790012008909B
:1055C000002009900A9002A90948FDF7C1FF08B11F
:1055D000FBF7B0FC00200090019069460448FDF7FD
:1055E00021FE08B1FBF7A6FC0BB000BD0004014092
:1055F000042E002010B50B480B4908604FF4E13031
:105600004860002108488160C16001610C2141614E
:1056100000218161C161FEF7C1FE08B1FBF78AFC80
:1056200010BD0000004C00404C2E002010B50D486D
:105630000D4908604FF4966048604FF480510A4865
:1056400081600021C1604FF4C06101610C214161A2
:1056500000218161C161FEF7A1FE08B1FBF76AFC80
:1056600010BD000000500040902E002010B50B48E7
:105670000B4908604FF4E130486000210848816020
:10568000C16001610C21416100218161C161FEF7AE
:1056900085FE08B1FBF74EFC10BD00000010014074
:1056A000D42E002010B50D480D4908604FF49660C7
:1056B00048604FF480510A4881600021C1604FF476
:1056C000C06101610C21416100218161C161FEF76E
:1056D00065FE08B1FBF72EFC10BD00000044004041
:1056E000182F002010B50B480B4908604FF4E1302B
:1056F0004860002108488160C16001610C2141615E
:1057000000218161C161FEF749FE08B1FBF712FC7F
:1057100010BD0000004800405C2F002000BFFEE7E5
:1057200000BFFEE77CB504460D46164616480068E5
:105730001821B0FBF1F01549B0FBF1F04FF47A718C
:10574000484301906068B0F5827F0DD12B4600225E
:1057500080212046009600F01BF898B1606D40F063
:105760002000606503207CBD00BF019800B908E0FF
:105770000198401E019020688068C0F3C010002886
:10578000F3D100BF0020EEE77400002040420F007C
:105790002DE9F84F04460D4690461E46DDF8289048
:1057A000FCF7AEFEA0EB0900371AFCF7A9FE824613
:1057B0002C480068C0F3CB307843009045E0701C63
:1057C000002842D0FCF79CFEA0EB0A00B84200D2B1
:1057D000A7BB2068406820F0E0002168486060684E
:1057E000B0F5827F0DD1A068B0F5004F03D0A0685E
:1057F000B0F5806F05D12068006820F04000216876
:105800000860A06AB0F5005F0DD100BF2068006895
:1058100020F40050216808602068006840F40050BF
:105820002168086000BF012084F8510000BF0020FB
:1058300084F8500000BF0320BDE8F88FFFE7009810
:1058400000B900270098401E00902068806828401A
:10585000A84201D1012000E000204045AFD1002046
:10586000EAE700007400002010B500BF502080F36C
:105870001188BFF34F8FBFF36F8F00BF10F0C8FFC9
:1058800018B14FF080500449086000BF002080F339
:10589000118800BF10BD000004ED00E000B593B01A
:1058A000302107A8FAF759FD142102A8FAF755FD8F
:1058B00000BF002001902348006840F0805021493B
:1058C00008600846006800F08050019000BF00BFEB
:1058D00000BF002001901C48006840F480401A4935
:1058E00008600846006800F48040019000BF00BFD7
:1058F000012007900004089002200D9041050E91B0
:105900000A210F91C82110910221119104211291B5
:1059100007A8FDF779F808B1FBF70CFB0F20029000
:1059200002200390002004904FF4A05005900690B0
:10593000032102A8FCF706FF08B1FBF7FBFA13B03E
:1059400000BD00004038024000700040034800687D
:1059500040F47000014908607047000088ED00E0E5
:1059600010B50248FDF73BFF10BD0000603300207A
:1059700010B50268294B98420ED0B0F1804F0BD081
:10598000274B984208D0274B984205D0264B984287
:1059900002D0264B984203D122F070024B681A4382
:1059A0001E4B984220D0B0F1804F1DD01C4B984226
:1059B0001AD01C4B984217D01B4B984214D01B4B4B
:1059C000984211D01A4B98420ED01A4B98420BD0E5
:1059D000194B984208D0194B984205D0184B984261
:1059E00002D0184B984203D122F44072CB681A437C
:1059F00022F080034C6943EA040202608B68C362B0
:105A00000B688362054B984202D0084B984201D143
:105A10000B6903630123436110BD000000000140D6
:105A20000004004000080040000C00400004014059
:105A3000004001400044014000480140001800407F
:105A4000001C00400020004030B501F01F0501247B
:105A500004FA05F3046A9C430462046A01F01F051A
:105A600002FA05F52C43046230BD30B50C4681685E
:105A700021F47F4142EA032525432943816030BD5B
:105A80000A46816821F0700142F0070319438160E2
:105A90007047000030B5056A25F001050562026A0D
:105AA0004368846924F0700424F003040D682C43D7
:105AB00022F002028D682A43104DA84200D103E073
:105AC0000F4DA84206D100BF22F00802CD682A433C
:105AD00022F00402094DA84202D0094DA84207D184
:105AE00023F4807323F400734D692B438D692B439A
:105AF000436084614D684563026230BD000001402F
:105B00000004014030B5056A25F010050562026AFF
:105B10004368846924F4E04424F440740D6844EA42
:105B2000052422F020028D6842EA0512124DA84297
:105B300000D103E0114DA84207D100BF22F080023E
:105B4000CD6842EA051222F040020B4DA84202D075
:105B50000A4DA84209D123F4806323F400634D6900
:105B600043EA85038D6943EA8503436084614D6898
:105B70008563026230BD0000000001400004014066
:105B800030B5056A25F480750562026A4368C46908
:105B900024F0700424F003040D682C4322F40072F6
:105BA0008D6842EA0522124DA84200D103E0114D52
:105BB000A84207D100BF22F40062CD6842EA052264
:105BC00022F480620A4DA84202D00A4DA84209D1AF
:105BD00023F4805323F400534D6943EA05138D6980
:105BE00043EA05134360C4614D68C563026230BD7A
:105BF000000001400004014030B5056A25F48055DD
:105C00000562036A4468C26922F4E04222F44072E9
:105C10000D6842EA052223F400538D6843EA0533F8
:105C2000084DA84202D0084DA84204D124F4804473
:105C30004D6944EA85144460C2614D68056403629D
:105C400030BD0000000001400004014030B50B46AB
:105C50001446026A056A25F001050562816921F092
:105C6000F00141EA041122F00A021A438161026242
:105C700030BD30B50B461446056A25F010050562A7
:105C80008169026A21F4704141EA043122F0A002E4
:105C900042EA03128161026230BD000010B5024881
:105CA000FEF70CFA10BD00004C2E002010B5024883
:105CB000FEF704FA10BD0000902E002070B50546D6
:105CC000AC6B0020E085E0842046FEF7BDF970BD96
:105CD00070B506460025B46B20684069C0F3C01556
:105CE00094F83D00212805D125B10020E08420460C
:105CF00000F0F7F820684069C0F3801594F83E0082
:105D0000222805D125B10020E085204600F0A3F827
:105D1000206C40F0100020642046FEF795F970BD1D
:105D200070B50546AC6B2868006800F480700028E8
:105D300042D1E08500BF00BF21680C3151E8001F4F
:105D400021F4807021680C3141E80002002AF3D16F
:105D500000BF00BF00BF2168143151E8001F21F0CF
:105D600001002168143141E80002002AF3D100BF8C
:105D700000BF00BF2168143151E8001F21F040002E
:105D80002168143141E80002002AF3D100BF20202D
:105D900084F83E00206B01280ED100BF00BF2168AF
:105DA0000C3151E8001F21F0100021680C3141E84E
:105DB0000002002AF3D100BF206B012804D1A18D7D
:105DC0002046FEF70FF802E02046FEF7F3FD70BD17
:105DD00070B50546AC6B206B012805D1A08D41083C
:105DE0002046FDF7FFFF02E02046FEF7E4FD70BD10
:105DF00070B50546AC6B2868006800F48070F8B98F
:105E00000020E08400BF00BF2168143151E8001F6A
:105E100021F080002168143141E80002002AF3D10A
:105E200000BF00BF00BF21680C3151E8001F41F0E6
:105E3000400021680C3141E80002002AF3D102E061
:105E40002046FEF70FFE70BD70B50446A56B2846D0
:105E5000FEF722FE70BD00BF00BF02680C3252E8A0
:105E6000002F22F4907102680C3242E80013002BDC
:105E7000F3D100BF00BF00BF0268143252E8002F08
:105E800022F001010268143242E80013002BF3D122
:105E900000BF016B01290ED100BF00BF02680C32A8
:105EA00052E8002F22F0100102680C3242E8001381
:105EB000002BF3D100BF202180F83E1000210163A8
:105EC000704710B504462068C06820F04000216883
:105ED000C860202084F83D002046FEF7C3FD002066
:105EE00010BD00BF00BF02680C3252E8002F22F044
:105EF000C00102680C3242E80013002BF3D100BF4E
:105F0000202180F83D107047F8B5044694F83E0013
:105F1000222873D1A068B0F5805F0CD1206950B9F8
:105F20000025A66A20684068C0F308003080A06A97
:105F3000801CA06215E0A56A0026A068B0F5805F0D
:105F400003D0A06828B9206918B920684068287073
:105F500004E02068406800F07F002870A06A401CC0
:105F6000A062E08D401E80B2E085002844D1206808
:105F7000C06820F020002168C8602068C06820F454
:105F800080702168C8602068406920F001002168A5
:105F90004861202084F83E00206B012826D1002093
:105FA000206300BF00BF21680C3151E8001F21F0C1
:105FB000100021680C3141E80002002AF3D100BF33
:105FC0002068006800F0100010280AD100BF0020EF
:105FD000009020680068009020684068009000BF32
:105FE00000BFA18D2046FDF7FDFE02E02046FEF732
:105FF000E1FC0020F8BD01E00020FBE70220F9E70A
:106000002DE9F84F04462068006920F44050E1680B
:106010000843216808612169A06808436169084351
:10602000E169084300902068C06849F20C61884328
:10603000009908432168C8602068406920F44070D6
:10604000A16908432168486176492068884203D0E5
:1060500075492068884203D1FCF76EFC814602E056
:10606000FCF75AFC8146E069B0F5004F6CD1022084
:106070006168A0FB015003461920A9FB007001468E
:106080002A463846FAF7FEF86421B0FBF1F04FEAF1
:10609000001A02206168A0FB01510B461920A9FBE0
:1060A00000712A463846FAF7EDF883460220616807
:1060B000A0FB015003461920A9FB00712A4638466F
:1060C000FAF7E0F86421B0FBF1F000EBC00101EB5E
:1060D0000010ABEB8000322101EBC0006421B0FB6B
:1060E000F1F000F0F8000AEB400A02206168A0FB22
:1060F000015003461920A9FB007001462A46384684
:10610000FAF7C0F8834602206168A0FB01500346FD
:106110001920A9FB00712A463846FAF7B3F8642122
:10612000B0FBF1F000EBC00101EB0010ABEB800025
:10613000322101EBC0006421B0FBF1F000F0070058
:106140005044216888606AE004206168A0FB015027
:1061500003461920A9FB007001462A463846FAF783
:1061600091F8824604206168A0FB01500346192083
:10617000A9FB007001462A463846FAF783F86421E5
:10618000B0FBF1F000EBC00101EB0010AAEB8000C6
:10619000322101EB00106421B0FBF1F000F0F00AB5
:1061A00004206168A0FB017003461920A9FB00517F
:1061B0003A462846FAF766F86421B0FBF1F00AEB9C
:1061C000001A04206168A0FB01510B461920A9FBAD
:1061D00000712A463846FAF755F88346042061686C
:1061E000A0FB015003461920A9FB007001462A4676
:1061F0003846FAF747F86421B0FBF1F000EBC00134
:1062000001EB0010ABEB8000322101EB00106421A8
:10621000B0FBF1F000F00F00504421688860BDE849
:10622000F88F0000001001400014014077B581B0E4
:10623000044615460298A062A5850020206422200D
:1062400084F83E002A48A16BC8632A48A16B086401
:106250002948A16BC8640020A16B086502AE3268B2
:106260002368191D2B46A06BFBF7BEF900BF002069
:10627000009020680068009020684068009000BF8F
:1062800000BF00BF002084F83C0000BF206970B14F
:1062900000BF00BF21680C3151E8001F41F480703D
:1062A00021680C3141E80002002AF3D100BF00BF91
:1062B00000BF2168143151E8001F41F0010021683E
:1062C000143141E80002002AF3D100BF00BF00BF33
:1062D0002168143151E8001F41F040002168143159
:1062E00041E80002002AF3D100BF002004B070BDD5
:1062F000215D0008D15D0008D15C0008014691F8DD
:106300003D00212828D18868B0F5805F0BD108694D
:1063100048B90A6A1088C0F308000B685860086A18
:10632000801C086205E00B6A581C086218780B682C
:106330005860C88C401E80B2C88458B90868C068CC
:1063400020F080000B68D8600868C06840F040000A
:106350000B68D860002070470220FCE710B50248A7
:10636000FDF7ACFE10BD0000D42E002010B5024891
:10637000FDF7A4FE10BD0000182F002010B5024844
:10638000FDF79CFE10BD00005C2F002000BFFEE763
:106390000FB4054B10B503A9044A029800F034F875
:1063A00010BC5DF814FB0000158100086806002091
:1063B00002480068C0F30220704700000CED00E0C6
:1063C00010B5002804DB0A07130E054A135406E033
:1063D0000A07140E034A00F00F031B1FD45410BD0C
:1063E00000E400E018ED00E002E008C8121F08C158
:1063F000002AFAD170477047002001E001C1121F46
:10640000002AFBD1704700002DE9FF4F8BB09A4660
:106410000F460546002606E025280BD052460D996A
:1064200090476D1C761C28780028F5D10FB03046B7
:10643000BDE8F08F0024A0460122604900E004433B
:1064400015F8013F203B02FA03F00842F7D1287803
:106450002E2817D115F8010F44F004042A280ED075
:106460006FF02F022878A0F1300109290AD808EB33
:10647000880102EB410100EB01086D1CF2E757F8BF
:10648000048B6D1C287869283ED006DC0028CDD00E
:1064900063280BD0642804D136E0732810D0752807
:1064A0004BD052460D999047761C85E017F8040BA7
:1064B0008DF8000000208DF80100E946012003E07E
:1064C00057F8049B4FF0FF3061074FF0000401D4F0
:1064D0000AE0641C44450DDA8442FADB19F8041022
:1064E0000029F6D106E0641C8442FCDB19F8041094
:1064F0000029F8D1264404E019F8010B52460D9901
:106500009047641EF8D257E001CF4FF00A0B0028E5
:1065100002DA40422D2102E0210504D52B218DF81D
:106520002410012103E0E10705D02021F7E70DF158
:10653000200908910CE00021F9E701CF4FF00A0B88
:10654000F9E75946F9F7C7FF01F1300209F8012DC3
:106550000028F6D1ADEB090000F1200B600701D453
:106560004FF00108D84502DDA8EB0B0000E0002049
:106570008046002406E009A85246005D0D99904728
:10658000641C761C08988442F5DB04E030205246F7
:106590000D999047761CB8F10001A8F10108F5DCCF
:1065A00005E019F8010B52460D999047761CBBF196
:1065B0000001ABF1010BF4DC6D1C34E7092801008C
:1065C00010B5012240210748FBF794FF01228021EA
:1065D0000448FBF78FFF012211460348FBF78AFFAF
:1065E00010BD0000000402400010024010B501225E
:1065F00040210748FBF77EFF012280210448FBF77A
:1066000079FF002201210348FBF774FF10BD000051
:10661000000402400010024070B50446254800EB1B
:10662000041041682448C0F89410903000F0C4F978
:1066300000BF42F2107000F063F90028F9D11F4842
:1066400000EB0410047000F0ABF805461B4800EBAB
:106650000410456000EE105AB8EEC00AF0EE040ACD
:1066600060EE200AB7EE001A80EE810ADFED140A10
:1066700080EE201A114800EB041080ED021A0F483A
:1066800000EB0410D0ED020A9FED0E1A80EE810A95
:10669000DFED0D0A20EE200A084800EB041080ED23
:1066A000030A00210448C0F89410903000F084F9E7
:1066B00070BD000060050020D001002040F60020E1
:1066C000FFFF7F4B0000C84200007A442DE9FC41E7
:1066D0000446002600200090019000250027207825
:1066E00000F03F0040F040008DF8000020680228D4
:1066F00005D11748808A00F4806000B10127207A14
:10670000401C3844C1B2684600F072F80646002EBC
:1067100002DA3046BDE8FC812FB1A068401C1DF8AC
:1067200000000B49486000206060012509E06068B6
:10673000000260601DF80510606808446060681C15
:10674000C5B2A068401CA842F1DC3046E2E7000078
:10675000D00100202DE9FC4104460027002600203E
:10676000009001900025207800F03F008DF8000097
:10677000666800BF07E0F0B2A168491B0DF8010090
:106780003612681CC5B2A068A842F4DC207A401C0E
:10679000C1B2684600F02CF807463846BDE8FC81D7
:1067A00010B5044800F008F802482038446A204632
:1067B00010BD0000F001002070B5054628680628CD
:1067C0000ED00A4890F8740000F0400040B142F248
:1067D000107000F0B3F80446002C01DA204670BDBA
:1067E0002846FFF773FF04462046F8E7D001002053
:1067F00070B504460D46002000F02AF9002000F094
:106800000EF92A462146044806F0B6FC064600204A
:1068100000F0ECF8304670BDD42C00201CB50024EC
:1068200007A103C9CDE9000108216846FFF7E0FF91
:10683000044642F2107000F09FF8044620461CBD4A
:10684000FFFFFFFFFFFFFFFF70B5FFF7E7FF054604
:10685000002D01DA284670BD0A20FAF70FFF144810
:10686000FFF7AAFF002419E01148503800EB04108C
:10687000C068012810D10E49503901EB041000F016
:106880009BF805460A49503901EB0410FFF794FFC5
:106890000546002D00DA03E0601CC4B2292CE3DBBE
:1068A00000BF012202210348FBF724FE2846D2E75D
:1068B000200200200010024010B50F480F49086068
:1068C0004FF48270486000210C488160C160022151
:1068D000016101214161490281612021C1610021E1
:1068E0000162416281620A21C162FCF7DBFA08B1F0
:1068F000FAF720FB10BD000000300140D42C00202E
:1069000070B5044600260CE00B48FFF755FF05461E
:10691000002D01DA284670BD07484068012121EAB0
:10692000D01616B9601E041EEED10CB10020F2E79D
:106930006FF00200EFE70000D001002070B50446C0
:1069400000260DE00B48FFF737FF0546002D01DA62
:10695000284670BD07486038406E012121EA901634
:1069600016B9601E041EEDD10CB10020F1E76FF0E6
:106970000200EEE73002002070B5044600260CE06D
:106980000C48FFF719FF0546002D01DA284670BDB7
:1069900008484068012121EA10161EB9201EA4F102
:1069A0000104EDD104B90EB10020F0E76FF0020050
:1069B000EDE70000D001002070B505460A4890F8C8
:1069C000740000F0400040B142F21070FFF7B6FFD3
:1069D0000446002C01DA204670BD2846FFF7BAFEB7
:1069E00004462046F8E70000D001002010B5044618
:1069F00024B1012C05D0022C0BD106E0FFF7E0FDFD
:106A00000BE0012000F058F807E0022000F054F8F5
:106A100003E0022000F050F800BF00BF10BD10B529
:106A2000044624B1012C05D0022C0BD106E0FFF75F
:106A3000DDFD0BE0012000F06DF807E0022000F022
:106A400069F803E0022000F065F800BF00BF10BD48
:106A500010B5044624B1012C05D0022C09D105E063
:106A6000FFF72AFF08E000F0D1F805E000F0CEF8CB
:106A700002E000F0CBF800BF00BF10BD10B50A481F
:106A800090F83E00202804D1020108490648FDF78D
:106A900068F9074890F83E00202804D10201054912
:106AA0000348FDF75EF910BD902E002076200020EF
:106AB000182F0020741A002010B50446012C02D0B3
:106AC000022C20D10FE0012240211048FBF712FDDB
:106AD000012280210D48FBF70DFD012211460C48D3
:106AE000FBF708FD10E0012240210848FBF702FDFA
:106AF000012280210548FBF7FDFC012211460448D4
:106B0000FBF7F8FC00E000BF00BF10BD000402402E
:106B10000010024010B50446012C02D0022C20D1F6
:106B20000FE0002240211048FBF7E4FC0122802105
:106B30000D48FBF7DFFC012211460C48FBF7DAFC9D
:106B400010E0002280210848FBF7D4FC01224021FC
:106B50000548FBF7CFFC012211460448FBF7CAFCAD
:106B600000E000BF00BF10BD000402400010024062
:106B700010B54FF6FF720621012000F069F840F2CF
:106B80000E720521012000F063F84FF6FF72062116
:106B9000022000F05DF840F20E720521022000F0A4
:106BA00057F810BD30B52DED028B81B00546B0EE23
:106BB000408A9FED140A28EE000AF3EE080A80EEE0
:106BC000201ABCEEC10A10EE104A002000900420EA
:106BD0008DF80000200A8DF80100E0B28DF8020067
:106BE0002846FFF735FF2846FFF719FF03226946BD
:106BF000054806F0C1FA2846FFF7F8FE01B0BDECE3
:106C0000028B30BD00FF7F47D42C002010B50E480A
:106C10000E4908604FF48270486000210B48816083
:106C2000C160016141614FF4007181612021C16146
:106C300000210162416281620A21C162FCF732F9DE
:106C400008B1FAF777F910BD00300140D42C0020CC
:106C5000F8B506460D461446002000908DF8005009
:106C600020128DF80100E0B28DF802003046FFF7E7
:106C7000EFFE3046FFF7D3FE03226946034806F0D5
:106C80007BFA3046FFF7B2FEF8BD0000D42C00209E
:106C900070B504460D461646324629462046FDF795
:106CA0008BFE08B1FAF746F970BD00002DE9F041FE
:106CB00004460D4600BF05F00300002808D000BFC1
:106CC0000BA34FF4B67216A11DA0FFF761FB00BF26
:106CD00000BF2E4606F064FB0746A06800683060DF
:106CE000A0680660384606F067FBBDE8F08100004A
:106CF0002E2E2F4D6964646C6577617265732F5415
:106D0000686972645F50617274792F4C7749502FB3
:106D10007372632F636F72652F6D656D702E6300E4
:106D20006D656D705F667265653A206D656D20708A
:106D3000726F7065726C7920616C69676E65640052
:106D4000417373657274696F6E2022257322206609
:106D500061696C6564206174206C696E65202564CE
:106D600020696E2025730A0070B5054606F018FBF1
:106D70000646A8680468002C16D02068A968086038
:106D800000BF04F00300002808D000BF09A34FF49F
:106D90008C7214A11CA0FFF7FBFA00BF00BF3046A5
:106DA00006F00AFB204670BD304606F005FB0020C9
:106DB000F9E700002E2E2F4D6964646C65776172CF
:106DC00065732F54686972645F50617274792F4CD7
:106DD0007749502F7372632F636F72652F6D656DE6
:106DE000702E63006D656D705F6D616C6C6F633AE2
:106DF000206D656D702070726F7065726C792061A6
:106E00006C69676E65640000417373657274696FC5
:106E10006E2022257322206661696C65642061748E
:106E2000206C696E6520256420696E2025730A0038
:106E300070B50546002411E004EB4400094901EB5C
:106E4000C000067D4EB104EB440001EBC000806839
:106E5000A84202D1204600F087F9641C0A2CEBDB23
:106E600070BD000034F500202DE9FF5F064689461D
:106E700017464FF00A0AD346D04600240A20039052
:106E8000002002900190009000BF73E004EB4400EA
:106E9000764901EBC000057DB8F10A0F02D10DB9AA
:106EA000A04665E0002D63D000BF012D0AD0022D61
:106EB00008DA00BF6EA340F223127BA18AA0FFF77D
:106EC00067FA00BF00BFAEB104EB4401674A02EBB2
:106ED000C1013068496888420CD13FB104EB4400DD
:106EE000114601EBC0008068B84203D1204604B0CF
:106EF000BDE8F09F012D28D104EB44005B4951F817
:106F0000300080B104EB440001EBC000418A0298DC
:106F100081422DDB039404EB4400544901EBC00093
:106F2000408A029024E004EB4400504901EBC00089
:106F3000418A019881421BDBA24604EB44004B4985
:106F400001EBC000408A019012E0022D10DB04EB3F
:106F50004400464901EBC000418A0098814207DBAA
:106F6000A34604EB4400414901EBC000408A009075
:106F7000601C04B20A2C89DB09F0020028B9B8F1C0
:106F80000A0F05D109F0010010B94FF0FF30AEE74C
:106F9000B8F10A0F01DA444631E0BBF10A0F11DA09
:106FA0005C4600BF04EB4400304951F8300040B16A
:106FB00000BF2FA340F26D1255A14BA0FFF7E8F9D7
:106FC00000BF0CE0BAF10A0F01DA544607E003985B
:106FD0000A2801DA039C02E04FF0FF3087E700BF88
:106FE0000A2C08DB00BF22A340F27F124EA13EA074
:106FF000FFF7CEF900BF00BF204600F0B5F800BF94
:107000000A2C08DB00BF1AA340F2831246A136A067
:10701000FFF7BEF900BF00BF00BF04EB44001349F7
:1070200001EBC000007D40B100BF11A34FF4C2725C
:1070300042A12DA0FFF7ACF900BF00BF36B104EBB1
:1070400044010A4A02EBC10130684860002004EBA9
:107050004401064A02EBC101488204EB4400114698
:1070600001EBC0008760204641E7000034F50020B6
:107070002E2E2F4D6964646C6577617265732F5491
:10708000686972645F50617274792F4C7749502F30
:107090007372632F636F72652F697076342F657416
:1070A000686172702E6300007374617465203D3DE9
:1070B000204554484152505F53544154455F504518
:1070C0004E44494E47207C7C207374617465203E99
:1070D0003D204554484152505F53544154455F53FD
:1070E0005441424C45000000417373657274696FEE
:1070F0006E2022257322206661696C6564206174AC
:10710000206C696E6520256420696E2025730A0055
:107110006172705F7461626C655B695D2E71203DA8
:107120003D204E554C4C000069203C204152505FA0
:107130005441424C455F53495A4500006172705FAB
:107140007461626C655B695D2E7374617465203D6A
:107150003D204554484152505F53544154455F458A
:107160004D5054590000000010B5044604EB440093
:107170000C4951F8300060B104EB4401094A52F85F
:10718000310005F013F8002004EB4401054A42F8F1
:107190003100002004EB4401024A02EBC1010875F2
:1071A00010BD000034F50020F0B587B007460D464D
:1071B00000BF002D0AD100BF2EA340F28A223BA1BE
:1071C0003EA0FFF7E5F800BF07B0F0BD00BF7C6848
:1071D0002088B0F5807F08D12079062805D1607914
:1071E000042802D16088082803D0384604F0DEFF66
:1071F000EAE7D4F80E000690A0690590686808B91F
:10720000002607E005986968884201D1012000E066
:10721000002006460EB1012000E00220034604F1E2
:10722000080206A9284600F0CBFCE088B0F5807F74
:1072300003D0B0F5007F15D113E086B1022206AB72
:1072400004F10800291DCDE90232CDE9001005F155
:107250002A0302462631284600F05CFB00E000BF0E
:1072600001E000E000BF00BF384604F09FFF00BF10
:10727000AAE700002E2E2F4D6964646C6577617259
:1072800065732F54686972645F50617274792F4C12
:107290007749502F7372632F636F72652F69707611
:1072A000342F6574686172702E6300006E657469B6
:1072B0006620213D204E554C4C0000004173736503
:1072C0007274696F6E2022257322206661696C6575
:1072D00064206174206C696E6520256420696E20CD
:1072E00025730A002DE9FE4304460F461546A946BC
:1072F00000BF002C08D100BF5DA340F21E326AA17E
:107300006DA0FFF745F800BF00BF00BF47B900BF41
:1073100057A340F21F3272A167A0FFF739F800BFF0
:1073200000BF00BF002D08D100BF51A34FF4487229
:107330006EA161A0FFF72CF800BF00BF21462868AE
:1073400001F037F910B1DFF8B48186E0287800F059
:10735000F000E02816D101208DF8040000208DF8FF
:1073600005005E208DF80600687800F07F008DF83B
:107370000700A8788DF80800E8788DF809000DF16D
:10738000040869E02868A1680840D4E901121140A6
:1073900088420ED0288880B24FF6A961884208D072
:1073A000E06810B104F10C0903E06FF00300BDE8E0
:1073B000FE835348007800EB4000524901EBC000C7
:1073C000007D02281BDB4E48007800EB400001EBFB
:1073D000C0008068A04212D14949097801EB4101FF
:1073E000484A02EBC101D9F800004968884206D139
:1073F000434802783946204600F086F8D7E7002651
:1074000022E006EB46003F4901EBC000007D022868
:1074100018DB06EB460001EBC0008068A04211D1EA
:1074200006EB4601374A02EBC101D9F80000496872
:10743000884207D13248067032463946204600F06D
:1074400063F8B4E7701CC6B20A2EDADB3A46494646
:10745000204600F00DF9AAE700BF4FF40060434654
:1074600004F12A0239460090204600F025FD9EE7EF
:107470002E2E2F4D6964646C6577617265732F548D
:10748000686972645F50617274792F4C7749502F2C
:107490007372632F636F72652F697076342F657412
:1074A000686172702E6300006E6574696620213D0C
:1074B000204E554C4C000000417373657274696F27
:1074C0006E2022257322206661696C6564206174D8
:1074D000206C696E6520256420696E2025730A0082
:1074E0007120213D204E554C4C00000069706164B4
:1074F000647220213D204E554C4C0000506E010816
:107500009401002034F50020F8B505460E461446D7
:1075100000BF04EB4400314901EBC000007D0228AC
:1075200008DA00BF2EA340F2EE223BA146A0FEF7F0
:107530002FFF00BF00BF04EB4400284901EBC0004F
:10754000007D022839D104EB440001EBC000408AE1
:10755000B0F58E7F11DD04EB44000A4602EBC0005B
:10756000011D284600F09CFA38BB032004EB4401BF
:107570001A4A02EBC10108751FE004EB44001749E9
:1075800001EBC000408AB0F5877F16DB04EB4400B6
:107590000B4603EBC00000F10C0204EB440003EBCC
:1075A000C000011D284600F087FA30B9032004EB23
:1075B00044010A4A02EBC10108754FF400600090D3
:1075C00004EB4400054901EBC00000F10C0305F198
:1075D0002A023146284600F06FFCF8BD34F5002041
:1075E0002E2E2F4D6964646C6577617265732F541C
:1075F000686972645F50617274792F4C7749502FBB
:107600007372632F636F72652F697076342F6574A0
:10761000686172702E6300006172705F7461626CE9
:10762000655B6172705F6964785D2E737461746507
:10763000203E3D204554484152505F5354415445EB
:107640005F535441424C4500417373657274696FD6
:107650006E2022257322206661696C656420617446
:10766000206C696E6520256420696E2025730A00F0
:107670002DE9FE4F81460F46164609F12A0A4FF0C2
:10768000FF300290002001904946386800F091FFD9
:1076900038B9387800F0F000E02802D00FB138682F
:1076A00018B96FF00F00BDE8FE8F4A460121384639
:1076B000FFF7DAFB8046B8F1000F02DA4FFA88F0E4
:1076C000F1E700BFB8F17F0F08D300BF5FA340F21E
:1076D000C1326CA16FA0FEF75BFE00BF00BF08F0D7
:1076E000FF0404EB4400754901EBC000007D70B954
:1076F0000120019004EB4401704A02EBC1010875BE
:1077000004EB4400114601EBC000C0F8089000BF34
:1077100004EB4400694901EBC000007D01280FD053
:1077200004EB440001EBC000007D022808DA00BF32
:1077300046A340F2CD3262A156A0FEF729FE00BF5B
:1077400000BF019800B93EB93946484600F0A8F993
:1077500002900EB90298A6E700BF46B900BF3BA34E
:1077600040F2E13260A14BA0FEF712FE00BF00BF65
:1077700004EB4400514901EBC000007D022811DBFD
:107780005C4804704FF40060009004EB440001EB8F
:10779000C00000F10C0352463146484600F08CFB15
:1077A000029050E004EB4400444901EBC000007D2E
:1077B000012848D14FF0000B354618E000BF68891A
:1077C000298988420AD1286840B100BF1FA340F22E
:1077D000F13249A12FA0FEF7DBFD00BF00BF287BDF
:1077E00000F0400010B14FF0010B02E02D68002DB9
:1077F000E4D100BFBBF1000F07D032464FF4207137
:107800000E2004F0C7FA054603E03546284604F08A
:10781000DDFEA5B104EB4400284951F8300030B139
:1078200004EB4401254A52F8310004F0BFFC04EB9C
:107830004400224941F830500020029002E04FF00D
:10784000FF30029000BF02982DE700002E2E2F4D32
:107850006964646C6577617265732F5468697264DA
:107860005F50617274792F4C7749502F7372632F78
:10787000636F72652F697076342F657468617270FA
:107880002E63000074797065206F766572666C6F88
:1078900077000000417373657274696F6E20222552
:1078A0007322206661696C6564206174206C696E66
:1078B0006520256420696E2025730A0034F50020B8
:1078C0006172705F7461626C655B695D2E73746177
:1078D0007465203D3D2050454E44494E47206F720F
:1078E00020535441424C45007120213D204E554CBF
:1078F0004C000000940100206E6F207061636B6586
:10790000742071756575657320616C6C6F77656443
:10791000210000002DE9FC5F06460F46904699467F
:10792000DDE90CAB0020019000BF002E08D100BFA4
:1079300031A340F257423EA141A0FEF729FD00BF0E
:1079400000BF4FF420721C210E2003F099FF054662
:107950001DB94FF0FF30BDE8FC9F00BF68891C28AF
:1079600008DA00BF24A340F262423FA134A0FEF730
:107970000FFD00BF00BF6C680F9802F074F9E08043
:1079800000BF96F83000062808D000BF1AA340F2C6
:10799000694242492AA0FEF7FBFC00BF00BFD9F8AC
:1079A0000000A060B9F80400A081DBF80000C4F872
:1079B0001200BBF80400E082DAF80000C4F80E0000
:1079C0000E980068A0614FF48070208008206080CD
:1079D000062020710420607140F6060043463A46B6
:1079E00029460090304600F067FA284604F0DEFB96
:1079F00000250198AFE700002E2E2F4D6964646CBE
:107A00006577617265732F54686972645F50617243
:107A100074792F4C7749502F7372632F636F72659F
:107A20002F697076342F6574686172702E63000060
:107A30006E6574696620213D204E554C4C00000057
:107A4000417373657274696F6E20222573222066FC
:107A500061696C6564206174206C696E65202564C1
:107A600020696E2025730A00636865636B20746863
:107A70006174206669727374207062756620636138
:107A80006E20686F6C642073747275637420657403
:107A9000686172705F68647200000000187101080C
:107AA00070B504460D46034A2946204600F004F806
:107AB00070BD0000506E01087FB504460D461646A5
:107AC0000121074A201D04F12A038DE825000391B6
:107AD000324619462046FFF71DFF04B070BD000076
:107AE000566E010870B5002464E004EB440033498D
:107AF00001EBC000057D002D5BD004EB440001EBE1
:107B0000C000408A401C04EB44012C4A02EBC10136
:107B1000488204EB4400114601EBC000408AB0F5F6
:107B2000967F0DDA04EB440001EBC000007D0128D4
:107B30000AD104EB440001EBC000408A052803DBB6
:107B40002046FFF711FB34E004EB44001B4901EB36
:107B5000C000007D032807D1042004EB4401174A2C
:107B600002EBC101087524E004EB4400134901EB6A
:107B7000C000007D042807D1022004EB44010F4A15
:107B800002EBC101087514E004EB44000B4901EB62
:107B9000C000007D01280CD104EB44020B4603EB2E
:107BA000C202111D04EB440203EBC2029068FFF70E
:107BB00077FF641C0A2C98DB70BD000034F50020B0
:107BC0002DE9F84305460E461746984600BF95F83E
:107BD0003000062808D000BF2EA340F2A9123BA116
:107BE00043A0FEF7D5FB00BF00BF5EB1306848B1CF
:107BF0002946306800F0DDFC20B9307800F0F00054
:107C0000E02803D16FF00F00BDE8F8832A46414613
:107C10003046FFF729F90446002C01DA60B2F3E799
:107C2000022004EB44013C4A02EBC101087504EB5D
:107C30004400114601EBC000856004EB440001EBF9
:107C4000C0003968C160B9880182002004EB44019A
:107C500002EBC101488204EB4400114651F83000A8
:107C6000B0B104EB440051F83090002004EB440123
:107C700042F831004FF400603B4605F12A024946C4
:107C80000090284600F018F9484604F08FFA00BF2B
:107C90000020B9E72E2E2F4D6964646C6577617200
:107CA00065732F54686972645F50617274792F4CE8
:107CB0007749502F7372632F636F72652F697076E7
:107CC000342F6574686172702E6300006E6574698C
:107CD000662D3E6877616464725F6C656E203D3D21
:107CE000204554485F4857414444525F4C454E003C
:107CF000417373657274696F6E202225732220664A
:107D000061696C6564206174206C696E652025640E
:107D100020696E2025730A0034F500202DE9F0411A
:107D200004460E464FF00E0860890E2800DC4FE036
:107D3000E07B18B996F83400401CE0736568AF89A1
:107D4000287800F00100B0B12878012809D16878BE
:107D500088B9A8785E280ED1607B40F0100060736F
:107D600009E006221D492846F8F709FB18B9607B8F
:107D700040F008006073082F03D0B7F5C16F22D11F
:107D800010E096F8310000F0080000B920E041460C
:107D9000204604F06FFC00B11AE03146204600F0A6
:107DA00095FD11E096F8310000F0080000B90FE0F1
:107DB0004146204604F05EFC00B109E03146204611
:107DC000FFF7F2F900E003E000BF0020BDE8F0811A
:107DD000204604F0EBF90020F8E70000506E01089F
:107DE000704700009AB00646642101A8F8F7B5FA7A
:107DF00000240027A046A146354600BF2C48FCF7CA
:107E00004EFE044695F83100C0F3800058B1012CB5
:107E100009DC2848FAF776F8284603F025F92846C1
:107E200003F09AF93FE095F83100C0F38000002894
:107E300039D1012C37DD022C06D0032C0AD0042CBA
:107E40000ED0052C17D111E04FF400694FF4804893
:107E5000012711E04FF000094FF4804801270BE0A3
:107E60004FF400694FF00008012705E04FF00009CA
:107E7000C846012700E000BF00BFA7B101A90D4817
:107E8000F9F724FCCDF81C90CDF8188001A9094819
:107E9000F9F780FF0748F9F7C9FF284603F040FAD1
:107EA000284603F0C9F9642003F0A8FAA6E7000009
:107EB000547F00206C7E00202DE9F04705460E46D9
:107EC00017469846DDF82090484601F0CCFE8246E1
:107ED0000E21304603F057FC00B122E07468A4F88C
:107EE0000CA0D8F800002060B8F80400A080386822
:107EF000C4F80600B888608100BF95F830000628F5
:107F000008D000BF08A34FF4997215A121A0FEF775
:107F10003FFA00BF00BF31462846AA699047BDE836
:107F2000F0876FF00100FAE72E2E2F4D6964646C24
:107F30006577617265732F54686972645F5061720E
:107F400074792F4C7749502F7372632F6E65746963
:107F5000662F65746865726E65742E63000000009C
:107F60006E657469662D3E6877616464725F6C65E6
:107F70006E206D757374206265203620666F7220E6
:107F800065746865726E65745F6F75747075742161
:107F900000000000417373657274696F6E202225C2
:107FA0007322206661696C6564206174206C696E5F
:107FB0006520256420696E2025730A0010B50446EB
:107FC00000BF44B900BF0CA34FF4F07211A115A07B
:107FD000FEF7DEF900BF00BF732084F83200742181
:107FE00033200155194860611948A061204601F00D
:107FF0009DFC002010BD00002E2E2F4C5749502F05
:108000005461726765742F65746865726E65746912
:10801000662E63006E6574696620213D204E554CC6
:108020004C000000417373657274696F6E202225E5
:108030007322206661696C6564206174206C696ECE
:108040006520256420696E2025730A00E57200080A
:108050003D9B000806460024354600BF4FF0FF3127
:108060000B48006803F00AFB0028F7D100BF284640
:1080700001F052FD04463CB1294620462A6990474A
:1080800010B1204604F092F8002CF0D1E6E7000091
:108090003400002070B504460D461646324621468F
:1080A0002846F8F733F970BD2DE9F04786B005464C
:1080B0000E4617464FF0000AA846FAF7BBF8002014
:1080C00001900B2003900120049002200590694646
:1080D00001A8FAF703F810B14FF0010A14E00024E8
:1080E0000EE056F804904A46002341460220FAF773
:1080F00055F810B14FF0010A04E008F10408241DFE
:10810000BC42EED300BF00BFFAF73EF8504606B0BF
:10811000BDE8F08738B504468DF8000069460320B5
:10812000ABBE204638BD000070B50546062D2CD2EA
:10813000DFE805F0030A11181F254FF48071154878
:10814000FAF7C6F9044622E04FF400711148FAF735
:10815000BFF904461BE04FF400610F48FAF7B8F985
:10816000044614E04FF480510B48FAF7B1F9044685
:108170000DE004210948FAF7ABF9044607E00821AD
:108180000648FAF7A5F9044601E0002400BF00BF45
:10819000204670BD0008024000000240001002406E
:1081A00010B500224FF480710F48FAF7A3F90022AE
:1081B00080210E48FAF79EF90A20F9F75FFA0122AA
:1081C00011020948FAF796F9012280210748FAF7C7
:1081D00091F9012211460548FAF78CF90122102184
:1081E0000248FAF787F910BD00000240000C024077
:1081F00070B505460C4622460321284600F03AF9A0
:1082000070BD00002DE9FF5F05468A46654880681D
:108210000390039800780007860E142E00DAB7E06A
:108220006889042800D2B3E06868047814B1082C87
:1082300070D100E0A6E0DFF86C9109F1140959480B
:10824000007D00F0F000E02800D1A5E0554A11685B
:10825000506900F0AEF900B19EE02889082800D2EC
:1082600096E006F10E01284603F08DFA002840D072
:10827000288930441FFA80FB2889584500DD8BE0AF
:108280004FF4207259460E2003F0FAFA074607B958
:1082900082E0798906F10800814203D2384603F072
:1082A00085FF79E0324678680399F8F72FF8314670
:1082B000384604F0DFF900280DD000BF00BF3AA314
:1082C000B62247A154A0FEF763F800BF00BF3846AE
:1082D00003F06CFF60E02946384603F0B3FD18B1A7
:1082E000384603F063FF57E0284603F05FFF3D4642
:1082F00011E006F10E01284604F0BCF958B100BFA8
:1083000000BF29A3C7224EA143A0FEF741F800BF3A
:1083100000BF41E024E0D5F804803146284603F050
:1083200032FAE0B96F68D9F80000F8601D480069BA
:108330003861002088F80000A8F80200FF20387299
:108340000020788101200021FF230A46CDE9010A9F
:1083500000914946284600F099FB834600BF11E092
:10836000032C0ED00B2C0CD00C2C0AD0042C08D0D3
:10837000052C06D00D2C04D00E2C02D0112C00D0D0
:1083800000BF00BF00BF284603F010FFBDE8FF9FFD
:10839000284603F00BFFF9E7284603F007FF00BF6C
:1083A000F4E70000B0BE00202E2E2F4D6964646CEF
:1083B0006577617265732F54686972645F5061728A
:1083C00074792F4C7749502F7372632F636F7265E6
:1083D0002F697076342F69636D702E630000000082
:1083E00069636D705F696E7075743A206D6F766940
:1083F0006E6720722D3E7061796C6F616420746FBE
:108400002069636D702068656164657220666169CA
:108410006C65640A00000000417373657274696FD3
:108420006E2022257322206661696C656420617468
:10843000206C696E6520256420696E2025730A0012
:1084400069636D705F696E7075743A2072657374DC
:108450006F72696E67206F726967696E616C2070F8
:108460002D3E7061796C6F6164206661696C656432
:108470000A0000002DE9FF470746884691464FF461
:1084800020722421222003F0FBF905460DB9BDE836
:10849000FF8700BF6889242808D200BF19A34FF4C2
:1084A000B47226A130A0FDF773FF00BF00BFD7F85C
:1084B00004A06C6884F8008084F801900020A080FB
:1084C000E08079686A6802F108001C22F7F71EFF55
:1084D000DAF80C00039003A800F040FD06465EB1F8
:1084E0000020608001200021FF2303AACDE90106BE
:1084F0000091284600F0CAFA284603F057FE00BF54
:10850000C5E700002E2E2F4D6964646C657761729B
:1085100065732F54686972645F50617274792F4C6F
:108520007749502F7372632F636F72652F6970766E
:10853000342F69636D702E6300000000636865630B
:108540006B20746861742066697273742070627540
:10855000662063616E20686F6C642069636D7020B3
:108560006D65737361676500417373657274696FDC
:108570006E2022257322206661696C656420617417
:10858000206C696E6520256420696E2025730A00C1
:1085900070B505460C4622460B212846FFF76AFFB8
:1085A00070BD00BFEFF3058008B1012070470020C7
:1085B000FCE718B502460092D04300B10AB9012089
:1085C00018BD91F8310000F0020008B90020F7E76B
:1085D0004868904201D10020F2E700988B6818406B
:1085E000D1E901342340984208D1886822EA00008A
:1085F0008C68E343984201D10120E1E70020DFE7E6
:108600002DE9F74F8CB004460F464FF00008398D26
:10861000A1F11400C11700EB5171C1F3CF0A14206E
:10862000059060680990DDF8249099F8000000F04A
:108630000F001421B1EB800F04D06FF005000FB0D4
:10864000BDE8F08F00BF608914280BDA00BF72A369
:108650004FF43F727FA186A0FDF79AFE00BF6FF036
:108660000500ECE700BFB9F8060001F0FCFA049041
:108670000498C0F30C000790049800F40050039095
:10868000208914381FFA80FBBDE04FF6FF7000EA26
:10869000CA00584501DD584603E04FF6FF7000EA76
:1086A000CA0008904FF4207214210E2003F0E8F85D
:1086B000054605B9ADE000BF6889142808DA00BF97
:1086C00055A34FF4497274A169A0FDF761FE00BF84
:1086D00000BF142268680999F7F718FED5F80490CE
:1086E00008980A9054E061890598081A80B20290AF
:1086F00000BF61890598814208DA00BF46A340F2B5
:108700002D326DA15AA0FDF743FE00BF00BF0299B4
:108710000A98884201DA0A9800E002988046B8F187
:10872000000F03D100200590246831E000F0BEFC6A
:1087300006461EB9284603F039FD6AE061680598CF
:108740000844334641224146CDE90008002003F0A9
:1087500045FA0B900B9830B9304600F0ADFC284636
:1087600003F024FD55E0204603F030FF74615648C5
:10877000306128460B9903F05BFA0A98A0EB0800D9
:1087800080B20A900A9810B100200590246800BFBA
:108790000A980028A7D10598404480B20590388DEA
:1087A0001438584501DB012000E0002006900798AE
:1087B000C0F30C000490069808B1039818B104980F
:1087C00040F400500490049801F04DFAA9F8060016
:1087D0000899143188B201F046FAA9F80200002085
:1087E000A9F80A007B69294638460E9A9847284618
:1087F00003F0DCFC0898ABEB00001FFA80FB079845
:10880000504480B20790BBF1000F7FF43EAF0020D0
:1088100015E74FF0FF3012E72E2E2F4D6964646C80
:108820006577617265732F54686972645F50617215
:1088300074792F4C7749502F7372632F636F726571
:108840002F697076342F6970345F667261672E63AA
:10885000000000006970345F6672616728293A2061
:108860007062756620746F6F2073686F7274000099
:10887000417373657274696F6E20222573222066BE
:1088800061696C6564206174206C696E6520256483
:1088900020696E2025730A0074686973206E65650F
:1088A00064732061207062756620696E206F6E654A
:1088B0002070696563652100702D3E6C656E203EF9
:1088C0003D20706F66660000099800082DE9F047AA
:1088D00007460E467D6828780421B1EB201F05D09D
:1088E000384603F063FC0020BDE8F08728780007D5
:1088F0004FEA9068688801F0B6F9814639894945A0
:1089000003DD4946384603F0ADFD7889404505DB77
:108910003889484502DBB8F1140F04DA384603F011
:1089200045FC0020E0E7286949494861E86808619A
:108930000846007D00F0F000E0280AD196F83100EA
:1089400000F0010018B1706808B134461CE0002442
:108950001AE0304600F080F808B1344614E00024F4
:108960003B48007D7F280FD03A48046809E0B442B4
:1089700000D105E0204600F06FF800B103E000BF31
:108980002468002CF3D100BF314908693146FFF754
:1089900010FE28B92E48007C00F0F000E02804D139
:1089A000384603F003FC00209EE724B9384603F064
:1089B000FDFB002098E7E8884FF63F71084038B18A
:1089C000384600F04DF907460FB900208CE77D6866
:1089D0001F4804604660856028780007800E1C49A7
:1089E00088814146384603F045FE687A012806D062
:1089F000062809D13146384606F03AF81DE03146DE
:108A00003846FFF7FFFB18E0114948692146FFF798
:108A1000D0FD70B90E48007D00F0F000E02808D0CD
:108A20000FFA88F1384603F0D2FC02213846FFF7EE
:108A3000DFFB384603F0BAFB00BF00BF002004494B
:108A400008604860886088810861486100BF4BE722
:108A5000B0BE00203401002010B5044694F8310067
:108A600000F0010070B1606860B10748406961685A
:108A7000884205D0044948692146FFF79AFD08B1AC
:108A8000012010BD0020FCE7B0BE00202DE9FE4F04
:108A900007460C4615469846DDE90C9A0E9EA346FD
:108AA00025B10CB1206808B906F1040B43462A46EB
:108AB00059463846CDE9009A029600F003F8BDE821
:108AC000FE8F00002DE9F84F05460F4690469A4666
:108AD000DDF828B00C9E00BFA87B012808D000BF9D
:108AE00037A34FF4557243A145A0FDF751FC00BFD9
:108AF00000BFB8F1000F46D04FF0140914212846EA
:108B000002F041FE18B16FF00100BDE8F88F6C680B
:108B100000BF6889142808D200BF29A34FF46272ED
:108B200041A137A0FDF734FC00BF00BF84F808A0C6
:108B30000B986072D8F80000206148464FEAE9714E
:108B400009EB9171C1F3870141F04001217084F874
:108B500001B0288901F087F860800020E0803E485D
:108B6000008801F080F8A0803B480088401C3A490A
:108B700008801FB939480068E06001E03868E060AB
:108B80000020608109E06889142802DA6FF0010092
:108B9000BBE76C6820690090E846308D48B12889B1
:108BA000318D884205DD424631462846FFF728FDD3
:108BB000ABE742462946304673699847A5E700006F
:108BC0002E2E2F4D6964646C6577617265732F5426
:108BD000686972645F50617274792F4C7749502FC5
:108BE0007372632F636F72652F697076342F6970AB
:108BF000342E6300702D3E726566203D3D203100AD
:108C0000417373657274696F6E202225732220662A
:108C100061696C6564206174206C696E65202564EF
:108C200020696E2025730A00636865636B20746891
:108C30006174206669727374207062756620636166
:108C40006E20686F6C642073747275637420697031
:108C50005F6864720000000096010020886F0108C0
:108C60002DE9F14F84B004984568287800F00F0092
:108C70001421B1EB800F00D011E1E88800F0F3FF80
:108C8000C0F30C004FF6FF7101EAC00A688800F0DB
:108C9000EAFF074628780007810E02910299B9423F
:108CA00000DDFCE00298381A87B2049803F068F8F7
:108CB00006467D48018888190A280ADD314628467B
:108CC00000F044FD20B17848008830440A2800DDD7
:108CD000E5E07648046811E06069E968884209D1F6
:108CE000A0692969884205D1A089A988884201D153
:108CF000012000E0002000B102E02468002CEBD14C
:108D000000BF34B93146284600F006FC044694B949
:108D1000C5E0E88800F0A7FFC0F30C0058B9E0896F
:108D200000F0A1FFC0F30C0028B11422294604F181
:108D30000800F7F7EBFAE888012121EA50100190CA
:108D4000019850B10AEB070188B2504503DB4FF69A
:108D5000EB71884200DD80E000BF2046019A049953
:108D600000F0F6F983460BF1010000B975E04E48BA
:108D7000008830444C490880019840B10AEB070153
:108D800088B2A083A17F41F00101A17700BFBBF1B0
:108D9000010F60D1A08B143080B2009060684068F1
:108DA000D0F8009060684568142204F10801284654
:108DB000F7F7ACFA009800F056FF68800020E880D2
:108DC0006881606804900DE0D9F8040003901421D4
:108DD000484603F04FFC4946049802F029FF0398E7
:108DE000D0F80090B9F1000FEED13048006884420D
:108DF00002D14FF000080EE02C48D0F8008006E0C9
:108E0000D8F80000A04200D104E0D8F80080B8F102
:108E1000000FF5D100BF4146204600F01BFB04982F
:108E200002F0AEFF064600BF1F480088B04208DAD5
:108E300000BF1FA340F29B222CA133A0FDF7A8FA8C
:108E400000BF00BF18480088801B1749088004989D
:108E500005B0BDE8F08F0020FAE700BF44B900BFBD
:108E600013A34FF42A7232A127A0FDF791FA00BF95
:108E700000BF606890B900BF0C480068844208D009
:108E800000BF0BA340F2AB222CA11FA0FDF780FA7C
:108E900000BF00BF0021204600F0DCFA00BF0498AC
:108EA00003F084F90020D3E79C0100209801002002
:108EB0002E2E2F4D6964646C6577617265732F5433
:108EC000686972645F50617274792F4C7749502FD2
:108ED0007372632F636F72652F697076342F6970B8
:108EE000345F667261672E630000000069705F7214
:108EF000656173735F70627566636F756E74203E33
:108F00003D20636C656E0000417373657274696F18
:108F10006E2022257322206661696C65642061746D
:108F2000206C696E6520256420696E2025730A0017
:108F300069707220213D204E554C4C006E6F74209C
:108F40006669727374616C74686F756768206A759E
:108F5000737420656E7175657565640010B50246A1
:108F60002148016821E091F8310000F00100D8B1FA
:108F700091F83100C0F38000B0B14868A0B110682A
:108F80008B681840D1E901342340984201D108464A
:108F900010BD91F8310000F0020028B91068CB68CC
:108FA000984201D10846F3E709680029DBD10F4850
:108FB0000068A0B10D48006890F8310000F0010091
:108FC00068B10A48006890F83100C0F3800030B101
:108FD00006480068406810B110787F2801D1002051
:108FE000D6E702480068D3E73401002038010020AA
:108FF00010B5044610220249204600F003F810BDC7
:1090000024F600202DE9FC4706460B4614464FF097
:10901000000C30680190194601AA00273CE00025A9
:1090200000BF10784FF00A0990FBF9FA09FB1A000B
:1090300000F0FF08107890FBF9F0107008F1300094
:1090400000F0FF0A284605F1010909F0FF050DF8B7
:1090500000A010780028E4D10BE060460CF1010C70
:10906000A04202DB0020BDE8FC871DF8050001F8E6
:10907000010B281EA5F1010909F0FF05EDD160469D
:109080000CF1010CA04201DB0020ECE72E2001F8DE
:10909000010B521C781CC7B2042FC0DB4FF0000933
:1090A000481E014680F800901846DCE710B5042001
:1090B00001F0A8FB10BD000010B5044600BF002C55
:1090C00008D100BF06A34FF4317214A116A0FDF71A
:1090D0005FF900BF00BF2146042001F0C5FA10BDB2
:1090E0002E2E2F4D6964646C6577617265732F5401
:1090F000686972645F50617274792F4C7749502FA0
:109100007372632F636F72652F697076342F697085
:10911000345F667261672E63000000007020213D9D
:10912000204E554C4C000000417373657274696F9A
:109130006E2022257322206661696C65642061744B
:10914000206C696E6520256420696E2025730A00F5
:109150002DE9F74F84B0064688460025012001908E
:10916000D8F8040002900299488800F07CFD8346FC
:10917000029800780007800E03900398584503DD9D
:10918000681E07B0BDE8F08F0398ABEB00001FFA34
:1091900080FB0299C88800F066FDC0F30C004FF612
:1091A000FF7101EAC00A00BF00BFD8F804400020E8
:1091B0002060A4F804A00AEB0B00E080E088504592
:1091C00002DA4FF0FF30DCE7D6F804903EE0D9F841
:1091D0000470A088B988884220DAC4F800909DB154
:1091E000A088E988884203DBE088B988884202DDEC
:1091F0004FF0FF30C5E7C5F80080E888A1888842B5
:109200000BD00020019008E0E088B988884202DD98
:109210004FF0FF30B5E7C6F804801AE0A088B9889F
:10922000884202D14FF0FF30ABE7A088F98888422E
:1092300002DA4FF0FF30A4E72DB1E888B988884200
:1092400001D000200190D7F800903D46B9F1000F01
:10925000BDD100BFB9F1000F28D1002D17D000BF3C
:10926000E888A188884208DD00BF3EA34FF4DB7286
:109270004BA153A0FDF78CF800BF00BFC5F80080DC
:10928000E888A188884211D0002001900EE000BF3C
:10929000706840B100BF33A34FF4DF7252A148A001
:1092A000FDF776F800BF00BFC6F80480069820B925
:1092B000B07F00F00100002851D00198002848D06C
:1092C000706818B170684068808810B10020019003
:1092D0003FE02546D4F800900BE0D9F80440E88838
:1092E000A188884202D00020019005E02546D4F8EC
:1092F0000090B9F1000FF0D100BF0198002828D0EC
:1093000000BF706840B900BF16A340F2DF1244A14D
:109310002BA0FDF73DF800BF00BF00BF706840689C
:10932000A04208D100BF0FA34FF4F0723CA124A0CB
:10933000FDF72EF800BF00BF00BF206840B100BF9E
:1093400008A34FF4F1723AA11DA0FDF721F800BF68
:1093500000BF019808B1012013E7002011E70020A9
:109360000FE700002E2E2F4D6964646C65776172E3
:1093700065732F54686972645F50617274792F4C01
:109380007749502F7372632F636F72652F69707600
:10939000342F6970345F667261672E6300000000CD
:1093A000636865636B20667261676D656E747320B8
:1093B000646F6E2774206F7665726C6170000000B8
:1093C000417373657274696F6E2022257322206663
:1093D00061696C6564206174206C696E6520256428
:1093E00020696E2025730A006E6F207072657669A1
:1093F0006F757320667261676D656E742C2074687A
:109400006973206D757374206265207468652066C9
:109410006972737420667261676D656E74210000F5
:1094200073616E69747920636865636B0000000086
:1094300076616C69646174655F64617461677261AF
:109440006D3A6E6578745F70627566213D4E554C5D
:109450004C00000070B504460D460E480068A0425E
:1094600003D10C49206808600EE000BF002D08D130
:1094700000BF09A340F2451216A11DA0FCF788FF0A
:1094800000BF00BF206828602146032001F0ECF8EF
:1094900070BD0000980100202E2E2F4D6964646C71
:1094A0006577617265732F54686972645F50617289
:1094B00074792F4C7749502F7372632F636F7265E5
:1094C0002F697076342F6970345F667261672E631E
:1094D0000000000073616E69747920636865636BD6
:1094E000206C696E6B6564206C6973740000000009
:1094F000417373657274696F6E2022257322206632
:1095000061696C6564206174206C696E65202564F6
:1095100020696E2025730A0070B505460E460320AB
:1095200001F070F9044664B93146284600F00EF99E
:10953000B04203DB032001F065F904460CB90020BA
:1095400070BD20212046F6F708FF0F20E07706487F
:1095500000682060044804601422294604F10800D1
:10956000F6F7D4FE2046EBE7980100202DE9F047FE
:1095700004468846002500BFA04507D100BF40A390
:10958000AB224EA150A0FCF703FF00BF00BFB8F113
:10959000000F0DD000BFD8F80000A04207D000BFD8
:1095A00037A3AD2252A148A0FCF7F2FE00BF00BFD6
:1095B0006068D0F80490B9F80400002824D16768E6
:1095C000D9F800006060142204F108017868F6F709
:1095D0009DFE01213846FEF7DBFF384602F0D0FB46
:1095E000064600BFA819B0F5803F07DB00BF24A3E3
:1095F000BC2244A134A0FCF7CBFE00BF00BFA819D9
:1096000085B2384602F0D2FD67681CE0D7F80490B6
:10961000BA46D9F80070504602F0B2FB064600BFC9
:10962000A819B0F5803F07DB00BF15A3CC2235A1F8
:1096300025A0FCF7ADFE00BF00BFA81985B25046BB
:1096400002F0B4FD00BF002FE0D141462046FFF7F5
:1096500001FF00BF33480088A84207DA00BF08A313
:10966000D22231A118A0FCF793FE00BF00BF2D4805
:109670000088401B2B4908802846BDE8F087000081
:109680002E2E2F4D6964646C6577617265732F545B
:10969000686972645F50617274792F4C7749502FFA
:1096A0007372632F636F72652F697076342F6970E0
:1096B000345F667261672E63000000007072657629
:1096C00020213D2069707200417373657274696F67
:1096D0006E2022257322206661696C6564206174A6
:1096E000206C696E6520256420696E2025730A0050
:1096F000707265762D3E6E657874203D3D206970F0
:109700007200000070627566735F66726565642042
:109710002B20636C656E203C3D2030786666666663
:10972000000000009C01002069705F726561737326
:109730005F70627566636F756E74203E3D20706267
:109740007566735F66726565640000002DE9F84F09
:1097500005468946002700BF0026B246002000903B
:1097600083461B48046821E06069E968884207D1A4
:10977000A0692969884203D1A089A988884201D0BB
:10978000012000E0002068B10BF1010B1EB9264654
:10979000CDF800A006E0E07FF17F884202DC26469B
:1097A000CDF800A0206800B1A2462468002CDBD1CF
:1097B0002EB130460099FFF7D9FE804647444F4509
:1097C00002DABBF1010FC7DC3846BDE8F88F0000B4
:1097D0009801002070B500250A4804680FE0E07F7A
:1097E000002805DDE07F401EE0772546246806E07E
:1097F0002646246829463046FFF7B8FE00BF002CF5
:10980000EDD170BD9801002070B505462C4600BF13
:10981000002C08D100BF0FA340F2CE221CA11FA034
:10982000FCF7B6FD00BF00BF00BFAC4208D000BFD0
:1098300008A340F2CF2223A118A0FCF7A9FD00BF86
:1098400000BF606910B1606902F0B0FC2046FFF70C
:1098500033FC70BD2E2E2F4D6964646C6577617288
:1098600065732F54686972645F50617274792F4C0C
:109870007749502F7372632F636F72652F6970760B
:10988000342F6970345F667261672E6300000000D8
:1098900070637220213D204E554C4C00417373651E
:1098A0007274696F6E2022257322206661696C656F
:1098B00064206174206C696E6520256420696E20C7
:1098C00025730A00706372203D3D20700000000087
:1098D00010B52DED048B0020104908701048006869
:1098E0000068C0F3001048700D480068406A00B27C
:1098F00048604868F6F7C2FD41EC190B9FED090B73
:1099000053EC102BF6F748FD41EC180BF6F7C7FDAA
:1099100002498860BDEC048B10BD000034F60020C5
:10992000042E00207B14AE47E17A743F2DE9F0410C
:10993000A2B004460027B8460026642109A8F6F71D
:109940000CFD6A486A49086000208DF81C008020E0
:109950008DF81D00E1208DF81E0000208DF81F00FD
:109960008DF820008DF8210007A848604FF4000111
:109970005F4881605F49C1605F4901614FF4C06128
:109980004161F8F7C3FDC0B28DF81F00F8F7C4FDC0
:10999000C0B28DF820006068000E8DF8210007A885
:1099A000534948600846F7F7A3FF07463821534854
:1099B000F6F7D3FC2120514908604FF4400048617C
:1099C000002008614E4800F007FF062084F83000B0
:1099D00047484068007884F82A0045484068417844
:1099E0002B2001554248406881782C200155404881
:1099F0004068C1782D2001553D48406801792E20EE
:109A000001553B48406841792F20015540F2DC5018
:109A1000208594F8310040F00A0084F831000322D8
:109A2000002101200CF05CF9364908600322002176
:109A300001200CF055F9344908601C22334968466E
:109A4000F6F764FC2146684601F04CFE3049314887
:109A5000FBF709F92F48FBF797F8002F41D12D4864
:109A6000FBF71DF80646012E06DC204601F074FBCC
:109A7000204601F0F9FA36E0022E06D0032E09D076
:109A8000042E0BD0052E11D10DE04FF400654FF4DC
:109A9000804810E000254FF480480CE04FF400654A
:109AA0004FF0000807E00025A84604E04FF40065E9
:109AB0004FF4804800BF00BF09A90D48F7F706FE24
:109AC0000F95CDF8388009A90948F8F763F90848D7
:109AD000F8F7ACF9204601F023FC204601F0ACFB7E
:109AE00001E0F7F727FA22B0BDE8F08100800240DC
:109AF0006C7E0020CC7D00202C7D00201C7F00206F
:109B0000EC6D01083400002038000020F86D0108D9
:109B10003C000020547F002038B50446002000900F
:109B20000448007818B969460348F7F7F6FF00982B
:109B300038BD0000300000206C7E00202DE9F0418F
:109B40008CB080460D460024002600273021684650
:109B5000F6F703FC30216846F6F7FFFB2E4629E0B6
:109B6000042C04D36FF00B000CB0BDE8F08104EBC3
:109B7000440170684DF82100708904EB44016A4685
:109B800002EB8101486054B104EB4400694601EBEB
:109B90008001601E00EB400002EB800081603068B5
:109BA00030B9002004EB44016A4602EB8101886071
:109BB000641C3668002ED3D128890D494860C1F84D
:109BC00008D008464563284602F000FD08490948C8
:109BD000F8F7F6F900BF4FF0FF310748006801F0D1
:109BE0004DFD0028F7D10348F8F74DF83846BBE79C
:109BF0001C7F00206C7E0020380000202DE9F04101
:109C0000044625466868804703F062FC06460D4915
:109C1000286809684718B81BB0F1004F01D301202C
:109C200000E0002030B1296888192246064903F077
:109C3000D7FC04E022460449384603F0D1FCBDE8D5
:109C4000F08100008C010020FD9B00080146080601
:109C500001F47F4240EA022001F47F0240EA122030
:109C600040EA1160704701460806000C40EA1120E6
:109C70007047000008B50020009000BF6846804291
:109C800008D000BF0BA340F25112164916A0FCF7F2
:109C90007FFB00BF00BF00BF00BF03F0C1FB00F0AF
:109CA000AFF900F089FD01F0B7F804F0D5FE03F03C
:109CB00037FD08BD2E2E2F4D6964646C6577617287
:109CC00065732F54686972645F50617274792F4CA8
:109CD0007749502F7372632F636F72652F696E69B6
:109CE000742E630004700108417373657274696FA8
:109CF0006E2022257322206661696C656420617480
:109D0000206C696E6520256420696E2025730A0029
:109D1000F8F714FCFBF7C2FDFBF78AF8FAF7BAFF75
:109D2000FBF7D4FBFBF720FBFBF764FCFBF77EFBA8
:109D3000FBF77CFCFBF7B6FCFBF7D4FCFBF738FB2E
:109D4000FBF794FCFBF718FC4FF400721749184816
:109D5000FAF707F84FF4007216491748FAF701F8B6
:109D60004FF4007215491648F9F7FBFF4FF40072E3
:109D700014491548F9F7F5FF4FF4007213491448D8
:109D8000F9F7EFFFFEF70CFA00211248F9F702FF8E
:109D90003C211148F9F7BCFC3C211048F9F7B8FC0C
:109DA000FAF7ECFF01F036FB00BFFEE76E0800207B
:109DB0004C2E0020721400205C2F00207620002002
:109DC000902E0020741A0020182F002078260020E2
:109DD000D42E0020742D00202C2D0020042E0020D5
:109DE00001460020842901D0CA1C1044704700009D
:109DF00070B5054605B970BD05F00300002813D005
:109E000000BF00BF3DA340F2732248A150A0FCF761
:109E1000BFFA00BF00BF00BF03F0C2FA06463046DB
:109E200003F0CAFA00BFE6E7A5F10804524800684B
:109E3000844205D305F10C0050490968884213D9C2
:109E400000BF00BF2DA340F27F224DA140A0FCF730
:109E50009FFA00BF00BF00BF03F0A2FA06463046DB
:109E600003F0AAFA00BFC6E74C4803F013FB2079C1
:109E7000002816D100BF00BF20A34FF4237248A1D1
:109E800033A0FCF785FA00BF00BF444803F01AFB7B
:109E900000BF03F085FA0646304603F08DFA00BF96
:109EA000A9E7204600F026F9002816D100BF00BF20
:109EB00012A340F2952244A125A0FCF769FA00BF45
:109EC00000BF364803F0FEFA00BF03F069FA064609
:109ED000304603F071FA00BF8DE70020207147483B
:109EE0000068844201D245480460204602F03CFCF0
:109EF0002A4803F0E7FA00BF7DE700002E2E2F4D21
:109F00006964646C6577617265732F546869726403
:109F10005F50617274792F4C7749502F7372632FA1
:109F2000636F72652F6D656D2E6300006D656D5FEB
:109F3000667265653A2073616E697479206368653D
:109F4000636B20616C69676E6D656E740000000064
:109F5000417373657274696F6E20222573222066C7
:109F600061696C6564206174206C696E652025648C
:109F700020696E2025730A00F0000020F400002004
:109F80006D656D5F667265653A20696C6C656761C9
:109F90006C206D656D6F727900000000F800002084
:109FA0006D656D5F667265653A20696C6C656761A9
:109FB0006C206D656D6F72793A20646F75626C65A7
:109FC00020667265650000006D656D5F667265658F
:109FD0003A20696C6C6567616C206D656D6F727994
:109FE0003A206E6F6E2D6C696E6B65643A20646FFB
:109FF00075626C652066726565000000FC000020DB
:10A0000010B500BF00BF194820F0030018490860D0
:10A01000084604684FF4C8602080002060802071EA
:10A020004FF4C86002F0D4FF1249086001200968AB
:10A0300008714FF4C8600F49096808800D49096824
:10A0400048800B4800680C4908600C4803F02AFA65
:10A0500000280AD000BF00BF09A340F21F2214A1AC
:10A060001AA0FCF795F900BF00BF10BDCBBE0020C1
:10A07000F0000020F4000020FC000020F800002088
:10A080002E2E2F4D6964646C6577617265732F5451
:10A09000686972645F50617274792F4C7749502FF0
:10A0A0007372632F636F72652F6D656D2E63000091
:10A0B0006661696C656420746F20637265617465A4
:10A0C000206D656D5F6D7574657800004173736513
:10A0D0007274696F6E2022257322206661696C6537
:10A0E00064206174206C696E6520256420696E208F
:10A0F00025730A002DE9F0410446204600F084F95A
:10A100000546208802F064FF0646608802F060FF82
:10A1100007462088B0F5C86F10D86088B0F5C86FC2
:10A120000CD86088A84202D03888A84206D10648D8
:10A130000068864205D07088A84202D00020BDE8A1
:10A14000F0810120FBE70000F40000202DE9F0473A
:10A150008146B9F1000F02D10020BDE8F08709F176
:10A16000030020F0030085B20C2D00D20C25B5F5BC
:10A17000C86F01D84D4501DA0020EEE75C4803F0D6
:10A1800089F95C48006800F03FF90646A6E03046D1
:10A1900002F01EFF0446207900287CD1218806F1B8
:10A1A0000800081AA84276D3218806F10800091A87
:10A1B00005F11400814229D306F1080028441FFA52
:10A1C00080F800BFB8F5C86F08D100BF4AA340F2BD
:10A1D000873255A159A0FCF7DBF800BF00BF40460D
:10A1E00002F0F6FE074600213971218839807E8011
:10A1F000A4F80080012020713888B0F5C86F07D01E
:10A20000388802F0E5FEA0F8028001E0012020710C
:10A2100038480068844227D13648D0F800A004E0CE
:10A22000BAF8000002F0D4FE82469AF8040018B191
:10A230004C4800688245F3D12E48C0F800A000BF0A
:10A2400000684849096888420CD02A4800680079AB
:10A2500040B100BF28A340F2B53243A137A0FCF7BC
:10A2600097F800BF00BF00BF214803F02BF900BFE3
:10A2700004F1080028443B490968884208D900BF16
:10A280001DA340F2B9323FA12CA0FCF781F800BF1A
:10A2900000BF00BF00E01DE004F0030040B100BFBC
:10A2A00015A340F2BB3243A124A0FCF771F800BF14
:10A2B00000BF00BF04F0030040B100BF0EA340F296
:10A2C000BD3248A11DA0FCF763F800BF00BF04F138
:10A2D000080042E7304602F07BFE0688C5F5C860FC
:10A2E000B0423FF654AF024803F0ECF8002034E7E8
:10A2F000F8000020FC0000202E2E2F4D6964646CB5
:10A300006577617265732F54686972645F5061721A
:10A3100074792F4C7749502F7372632F636F726576
:10A320002F6D656D2E630000696E76616C69642027
:10A330006E6578742070747200000000417373655C
:10A340007274696F6E2022257322206661696C65C4
:10A3500064206174206C696E6520256420696E201C
:10A3600025730A00F40000206D656D5F6D616C6CF3
:10A370006F633A20216C667265652D3E7573656466
:10A38000000000006D656D5F6D616C6C6F633A205D
:10A39000616C6C6F6361746564206D656D6F72795B
:10A3A000206E6F742061626F76652072616D5F65EB
:10A3B0006E642E006D656D5F6D616C6C6F633A202D
:10A3C000616C6C6F6361746564206D656D6F72792B
:10A3D0002070726F7065726C7920616C69676E6550
:10A3E000642E00006D656D5F6D616C6C6F633A206B
:10A3F00073616E69747920636865636B20616C6951
:10A40000676E6D656E740000014602480088081A88
:10A4100080B27047F00000202DE9F84F81468B464E
:10A420000BF1030020F0030085B20C2D00D20C25A7
:10A43000B5F5C86F01D85D4502DA0020BDE8F88F98
:10A4400000BF5C480068814503D35B4800688145D4
:10A4500008D300BF59A340F2D12264A169A0FBF741
:10A4600097FF00BF00BF53480068814503D352489F
:10A470000068814509D300BF02F092FF0090009868
:10A4800002F09AFF00BF4846D8E7A9F10806304617
:10A49000FFF7BAFF07463188C81B08381FFA80FA51
:10A4A00000BF554508DD00BF44A34FF439725FA1DA
:10A4B00054A0FBF76DFF00BF00BF554501DD002034
:10A4C000BCE7554501D14846B8E7604802F0E2FFD5
:10A4D000308802F07DFD04462079002833D100BF8A
:10A4E0003088B0F5C86F08D100BF34A340F2F52220
:10A4F00057A144A0FBF74CFF00BF00BF208800908D
:10A5000007F1080028441FFA80F856480068A04266
:10A5100004D1404602F05CFD52490860404602F01A
:10A5200057FD044600202071009820806780A6F81F
:10A5300000802088B0F5C86F04D0208802F048FD64
:10A54000A0F8028031E005F1140050452DD807F144
:10A55000080028441FFA80F800BF3088B0F5C86FA3
:10A5600008D100BF15A340F2163239A125A0FBF790
:10A570000FFF00BF00BF404602F02AFD04463948E5
:10A580000068844201D2374804600020207130887E
:10A5900020806780A6F800802088B0F5C86F04D0BE
:10A5A000208802F015FDA0F80280284802F08AFFFA
:10A5B000484643E7F0000020F40000202E2E2F4DE7
:10A5C0006964646C6577617265732F54686972643D
:10A5D0005F50617274792F4C7749502F7372632FDB
:10A5E000636F72652F6D656D2E6300006D656D5F25
:10A5F0007472696D3A206C6567616C206D656D6F72
:10A6000072790000417373657274696F6E20222540
:10A610007322206661696C6564206174206C696EC8
:10A620006520256420696E2025730A006D656D5FC5
:10A630007472696D2063616E206F6E6C792073682F
:10A6400072696E6B206D656D6F727900F800002085
:10A65000696E76616C6964206E65787420707472BE
:10A6600000000000FC00002070B504460D4600BF4D
:10A670000C2C09DB00BF0AA34FF4D57214A11BA058
:10A68000FBF786FE00BF70BD00BF05B9FBE721499F
:10A6900051F824002946FCF709FB00BFF3E700004E
:10A6A0002E2E2F4D6964646C6577617265732F542B
:10A6B000686972645F50617274792F4C7749502FCA
:10A6C0007372632F636F72652F6D656D702E6300FB
:10A6D0006D656D705F667265653A2074797065208E
:10A6E0003C204D454D505F4D41580000417373650E
:10A6F0007274696F6E2022257322206661696C6511
:10A7000064206174206C696E6520256420696E2068
:10A7100025730A00EC6E010870B504460D4600BFB3
:10A72000002C08D100BF09A340F2951213A118A074
:10A73000FBF72EFE00BF00BF04B105B970BD29466E
:10A740002046FCF7B3FA00BFF8E700002E2E2F4D8D
:10A750006964646C6577617265732F5468697264AB
:10A760005F50617274792F4C7749502F7372632F49
:10A77000636F72652F6D656D702E6300696E766113
:10A780006C696420706F6F6C2064657363000000F7
:10A79000417373657274696F6E202225732220667F
:10A7A00061696C6564206174206C696E6520256444
:10A7B00020696E2025730A0010B5002406E00549C3
:10A7C00051F8240000F008F8601C84B20C2CF6D379
:10A7D00010BD0000EC6E010810B5002384682360F2
:10A7E0004368DB1C23F00301002207E083681B6839
:10A7F0000B608368196003881944521C4388934294
:10A80000F4DC10BD70B5044600BF0C2C0ADB00BFA1
:10A8100009A340F2571214A11BA0FBF7B9FD00BF1A
:10A82000002070BD00BF224951F82400FCF79CFABB
:10A8300005462846F5E700002E2E2F4D6964646C0E
:10A840006577617265732F54686972645F506172D5
:10A8500074792F4C7749502F7372632F636F726531
:10A860002F6D656D702E63006D656D705F6D616C31
:10A870006C6F633A2074797065203C204D454D50D3
:10A880005F4D415800000000417373657274696F39
:10A890006E2022257322206661696C6564206174D4
:10A8A000206C696E6520256420696E2025730A007E
:10A8B000EC6E010810B5044600BF002C08D100BFA3
:10A8C00007A34FF49E7212A116A0FBF761FD00BF13
:10A8D00000BF0CB9002010BD2046FCF745FAFAE78E
:10A8E0002E2E2F4D6964646C6577617265732F54E9
:10A8F000686972645F50617274792F4C7749502F88
:10A900007372632F636F72652F6D656D702E6300B8
:10A91000696E76616C696420706F6F6C206465731A
:10A9200063000000417373657274696F6E202225A5
:10A930007322206661696C6564206174206C696EA5
:10A940006520256420696E2025730A002DE9F05FDB
:10A9500004460E4617469846DDE90AB900BF002CAA
:10A960000BD100BF4CA340F2271258A15EA0FBF709
:10A970000FFD00BF0020BDE8F09F00BF00BFB9F190
:10A98000000F0AD100BF44A34FF4947260A156A0F7
:10A99000FBF7FEFC00BF0020EDE700BF06B9654EE7
:10A9A00007B9644FB8F1000F01D1DFF888810020AA
:10A9B0006060A060E060604860610020208584F8ED
:10A9C0003100E0612062C4F824B05C48007884F86B
:10A9D00034000C98206143463A463146204600F048
:10A9E000E9FA2046C84708B10020C4E700BF94F840
:10A9F0003400FF2802D1002084F834004FF0000A10
:10AA00004F48056829E000BFA54208D100BF22A336
:10AA100040F28B124BA134A0FBF7BAFC00BF00BF81
:10AA20000AF1010A00BFBAF1FF0F08DD00BF1AA347
:10AA300040F28D1248A12CA0FBF7AAFC00BF00BF7A
:10AA400095F8340094F83410884205D194F8340015
:10AA5000401C84F8340002E02D68002DD3D100BFE3
:10AA6000002DC4D194F83400FE2803D100203349CE
:10AA7000087004E094F83400401C304908703048F5
:10AA8000006820602E48046000220121204600F06A
:10AA9000C5F920466FE700002E2E2F4D6964646CC7
:10AAA0006577617265732F54686972645F50617273
:10AAB00074792F4C7749502F7372632F636F7265CF
:10AAC0002F6E657469662E63000000006E65746900
:10AAD000665F6164643A20696E76616C6964206EB9
:10AAE0006574696600000000417373657274696F74
:10AAF0006E2022257322206661696C656420617472
:10AB0000206C696E6520256420696E2025730A001B
:10AB10006E657469665F6164643A204E6F20696E89
:10AB200069742066756E6374696F6E2067697665F7
:10AB30006E000000886F0108ADAF00083C010020E6
:10AB4000340100206E6574696620616C7265616411
:10AB50007920616464656400746F6F206D616E7943
:10AB6000206E65746966732C206D61782E20737574
:10AB700070706F72746564206E756D6265722069A5
:10AB8000732032353500000070B504460D46294665
:10AB9000204604F065FF70BD70B504460D461646AC
:10ABA0002868E168884201D1012000E000200028E7
:10ABB00014D100BF46B900BF09A34FF4147215A108
:10ABC00018A0FBF7E5FB00BF00BFE06830600DB9DF
:10ABD000002000E02868E060012070BD0020FCE754
:10ABE0002E2E2F4D6964646C6577617265732F54E6
:10ABF000686972645F50617274792F4C7749502F85
:10AC00007372632F636F72652F6E657469662E634E
:10AC100000000000696E76616C696420706F696E77
:10AC200074657200417373657274696F6E202225BA
:10AC30007322206661696C6564206174206C696EA2
:10AC40006520256420696E2025730A00F8B5044646
:10AC50000D46164600BF002D08D100BF1CA340F2D0
:10AC6000CB1228A12BA0FBF793FB00BF00BF00BFB6
:10AC700046B900BF16A34FF4E67222A125A0FBF748
:10AC800087FB00BF00BF28686168884201D10120AE
:10AC900000E00020C8B9286800906068306069460C
:10ACA0003046FFF771FF0DB9002000E028686060B2
:10ACB0000121204600F00EF900BFE06910B12046E6
:10ACC000E169884700BF0120F8BD0020FCE70000D3
:10ACD0002E2E2F4D6964646C6577617265732F54F5
:10ACE000686972645F50617274792F4C7749502F94
:10ACF0007372632F636F72652F6E657469662E635E
:10AD000000000000696E76616C696420706F696E86
:10AD100074657200417373657274696F6E202225C9
:10AD20007322206661696C6564206174206C696EB1
:10AD30006520256420696E2025730A0070B50446DD
:10AD40000D4616462868A168884201D1012000E01E
:10AD50000020002814D100BF46B900BF09A34FF45A
:10AD6000047215A118A0FBF713FB00BF00BFA06879
:10AD700030600DB9002000E02868A060012070BD9F
:10AD80000020FCE72E2E2F4D6964646C657761729C
:10AD900065732F54686972645F50617274792F4CC7
:10ADA0007749502F7372632F636F72652F6E6574CE
:10ADB00069662E6300000000696E76616C6964202C
:10ADC000706F696E74657200417373657274696F38
:10ADD0006E2022257322206661696C65642061748F
:10ADE000206C696E6520256420696E2025730A0039
:10ADF00002466AB10748016808E091F83400401C37
:10AE0000C0B2904201D10846704709680029F4D1C8
:10AE10000020F9E734010020704700002DE9F041DF
:10AE200005460E4617460D48046800BF002D08D1A0
:10AE300000BF0BA340F2FC6216A11CA0FBF7A8FA0E
:10AE400000BF00BF05E03A463146284623689847D0
:10AE50006468002CF7D1BDE8F081000030010020CB
:10AE60002E2E2F4D6964646C6577617265732F5463
:10AE7000686972645F50617274792F4C7749502F02
:10AE80007372632F636F72652F6E657469662E63CC
:10AE9000000000006E65746966206D757374206231
:10AEA0006520213D204E554C4C00000041737365D8
:10AEB0007274696F6E2022257322206661696C6549
:10AEC00064206174206C696E6520256420696E20A1
:10AED00025730A0070B504460D4600BF002C08D14A
:10AEE00000BF12A340F26D321DA126A0FBF750FA5D
:10AEF00000BF00BF94F8310000F0040020B194F8C6
:10AF0000310000F0010000B970BD05F0010050B142
:10AF1000606840B194F8310000F0080018B1211DBC
:10AF20002046FCF7BDFD00BFEEE700002E2E2F4DA2
:10AF30006964646C6577617265732F5468697264C3
:10AF40005F50617274792F4C7749502F7372632F61
:10AF5000636F72652F6E657469662E630000000072
:10AF60006E657469665F69737375655F7265706F2E
:10AF70007274733A20696E76616C6964206E6574D0
:10AF800069660000417373657274696F6E202225D3
:10AF90007322206661696C6564206174206C696E3F
:10AFA0006520256420696E2025730A0003466FF032
:10AFB0000B0070472DE9F04F87B083460D461646CB
:10AFC0001F4600240DF10C080DF1080905B9224DAA
:10AFD00006B9214E07B9204F0DB1286808B90120E4
:10AFE00000E000208246BAF1000F09D001AA2946EC
:10AFF0005846FFF72BFE18B144F0100401A8049046
:10B00000424631465846FFF799FE18B144F04004D5
:10B01000CDF814804A4639465846FFF7BDFD18B1B1
:10B0200044F02004CDF81890BAF1000F09D101AA1C
:10B0300029465846FFF70AFE18B144F0100401A84B
:10B04000049034B144F0800404AA21465846FFF726
:10B05000E5FE07B0BDE8F08F886F01080149086080
:10B0600070470000380100203EB5044600BF002CA8
:10B0700009D100BF17A340F29B3223A12AA0FBF7FE
:10B0800087F900BF3EBD00BF94F8310000F0010019
:10B09000F0B100208DF800006A4608212046FFF735
:10B0A000BDFE00BF94F8310000F0FE0084F83100CE
:10B0B00000BF94F8310000F0080010B12046FBF703
:10B0C000B7FE00BFE06910B12046E169884700BFC4
:10B0D00000BFD7E72E2E2F4D6964646C65776172CF
:10B0E00065732F54686972645F50617274792F4C74
:10B0F0007749502F7372632F636F72652F6E65747B
:10B1000069662E63000000006E657469665F736592
:10B11000745F646F776E3A20696E76616C69642043
:10B120006E65746966000000417373657274696FBF
:10B130006E2022257322206661696C65642061742B
:10B14000206C696E6520256420696E2025730A00D5
:10B1500000B10162704700003EB5044600BF002CFC
:10B1600009D100BF14A340F2064220A128A0FBF79A
:10B170000FF900BF3EBD00BF94F8310000F004009D
:10B18000B8B100BF94F8310000F0FB0084F8310042
:10B1900000BF00BF206A10B12046216A884700BF67
:10B1A00000208DF800006A4604212046FFF736FE95
:10B1B00000BF00BFDEE700002E2E2F4D6964646CD7
:10B1C0006577617265732F54686972645F5061724C
:10B1D00074792F4C7749502F7372632F636F7265A8
:10B1E0002F6E657469662E63000000006E657469D9
:10B1F000665F7365745F6C696E6B5F646F776E3AE0
:10B2000020696E76616C6964206E65746966000001
:10B21000417373657274696F6E20222573222066F4
:10B2200061696C6564206174206C696E65202564B9
:10B2300020696E2025730A003EB5044600BF002C2D
:10B2400009D100BF16A34FF4787222A12AA0FBF700
:10B250009FF800BF3EBD00BF94F8310000F004002D
:10B26000D8B900BF94F8310040F0040084F83100F0
:10B2700000BF03212046FFF72DFE00BF206A10B15A
:10B280002046216A884700BF01208DF800006A46E9
:10B2900004212046FFF7C2FD00BF00BFDAE700002F
:10B2A0002E2E2F4D6964646C6577617265732F541F
:10B2B000686972645F50617274792F4C7749502FBE
:10B2C0007372632F636F72652F6E657469662E6388
:10B2D000000000006E657469665F7365745F6C6979
:10B2E0006E6B5F75703A20696E76616C6964206E72
:10B2F0006574696600000000417373657274696F5C
:10B300006E2022257322206661696C656420617459
:10B31000206C696E6520256420696E2025730A0003
:10B320003EB5044600BF002C09D100BF15A34FF461
:10B33000547221A127A0FBF72BF800BF3EBD00BF30
:10B3400094F8310000F00100D0B900BF94F831004A
:10B3500040F0010084F8310000BF00BFE06910B187
:10B360002046E169884700BF01208DF800006A4649
:10B3700008212046FFF752FD03212046FFF7AAFDD2
:10B3800000BFDBE72E2E2F4D6964646C6577617218
:10B3900065732F54686972645F50617274792F4CC1
:10B3A0007749502F7372632F636F72652F6E6574C8
:10B3B00069662E63000000006E657469665F7365E0
:10B3C000745F75703A20696E76616C6964206E6591
:10B3D00074696600417373657274696F6E2022250B
:10B3E0007322206661696C6564206174206C696EEB
:10B3F0006520256420696E2025730A0070B5044617
:10B4000025460DB1294600E0012108460AF058F909
:10B41000002070BD10B50AF069FA002010BD10B50B
:10B42000FDF7BFF810B10BF0E9F910BD0BF0E0F932
:10B43000FBE7F8B504460D46A06840B1E06830B1BE
:10B440000020009094E80F000AF077FCF8BD00227D
:10B45000D4E900010AF044FCF8E700002DE9FF41BF
:10B4600007460D4614460295002001903DB9802004
:10B4700000909DE8070087E80700BDE8FF810020F5
:10B4800003900026601C08B9761E03E014B126461E
:10B4900006B90126FDF785F8B0B103AA01A928462F
:10B4A0000AF07EFF012802D11020009001E0002068
:10B4B00000900398B8B14FF080500E490860BFF378
:10B4C0004F8FBFF36F8F0EE0324601A928460AF076
:10B4D000B3FE012802D11020009004E00EB9002034
:10B4E00000E0402000909DE8070087E8070000BFCB
:10B4F000C3E7000004ED00E077B581B006461446CE
:10B5000000200090254605B90125FDF74AF8A8B1AD
:10B5100000236A4602A930460AF0A0FD012802D0A5
:10B52000FF2004B070BD009890B14FF080500949E1
:10B530000860BFF34F8FBFF36F8F09E000232A46E7
:10B5400002A930460AF0B6FC012801D0FF20E8E746
:10B550000020E6E704ED00E010B50446606820B185
:10B56000012061680AF0A7FB10BD01200AF092FBE0
:10B57000FAE7000038B50446002500200090FDF7EA
:10B5800010F890B1694620460AF0E6FD012801D086
:10B59000FF2038BD009888B14FF0805008490860FE
:10B5A000BFF34F8FBFF36F8F08E000231A46194691
:10B5B00020460AF07FFC012800D0FF252846E8E756
:10B5C00004ED00E0F8B506460C46002000900EB9E8
:10B5D0008020F8BD0025601C08B96D1E03E014B181
:10B5E000254605B90125FCF7DCFF98B16A46002124
:10B5F00030460AF0D5FE012801D0FF20E9E7009887
:10B6000080B14FF0805008490860BFF34F8FBFF3FF
:10B610006F8F07E0294630460AF028FF012801D045
:10B62000FF20D6E70020D4E704ED00E038B504465B
:10B63000002500200090FCF7B4FF90B16946204639
:10B640000AF08AFD012801D0FF2038BD009888B19A
:10B650004FF0805008490860BFF34F8FBFF36F8FE2
:10B6600008E000231A46194620460AF023FC012868
:10B6700000D0FF252846E8E704ED00E0F8B50646CF
:10B680000C46002000900EB98020F8BD0025601CFB
:10B6900008B96D1E03E014B1254605B90125FCF774
:10B6A00080FF98B16A46002130460AF079FE0128F1
:10B6B00001D0FF20E9E7009880B14FF080500849A1
:10B6C0000860BFF34F8FBFF36F8F07E02946304606
:10B6D0000AF0CCFE012801D0FF20D6E70020D4E7F5
:10B6E00004ED00E07FB504460D46606998B1A0699D
:10B6F00088B1B4F90800FEF773FB0646D4E90510DB
:10B70000CDE9006102902B462269D4E900100BF0CC
:10B7100001F8039013E0B4F90800FEF761FB064658
:10B7200003A8CDE90060238A9AB22B46D4E9001021
:10B730000AF0BEFF012802D0002004B070BD0398BB
:10B74000FBE7000010B50446FCF72BFF60B1204674
:10B750000BF090FA01280AD1000706490860BFF3F0
:10B760004F8FBFF36F8F02E020460AF077F800207A
:10B7700010BD000004ED00E010B5044620460AF0BC
:10B780000DF9002010BD70B504460D460022294673
:10B79000204600F001F870BD2DE9F04704460D4643
:10B7A000904600BF44B900BF1CA340F2DF1227A19E
:10B7B00029A0FAF7EDFD00BF00BF14B1B5F5803F39
:10B7C00002D30120BDE8F0870DB90020FAE7AEB240
:10B7D0002089304480B2B04201DA0120F2E794F8C7
:10B7E0000C9009F0800038B16068471B04F110002C
:10B7F000874209D20120E5E7B8F1000F02D0606866
:10B80000471B01E00120DDE767606089304460810B
:10B810002089304420810020D4E700002E2E2F4DB7
:10B820006964646C6577617265732F5468697264CA
:10B830005F50617274792F4C7749502F7372632F68
:10B84000636F72652F706275662E63007020213DF4
:10B85000204E554C4C000000417373657274696F43
:10B860006E2022257322206661696C6564206174F4
:10B87000206C696E6520256420696E2025730A009E
:10B880002DE9FE4F82460E4690465746B8F1010F0D
:10B890000AD0B8F1410F06D0B8F5C17F0BD0B8F58A
:10B8A000207F7DD16AE000BF42463146002000F093
:10B8B00037F90446AEE0002400200290B14600BFF4
:10B8C0000B20FEF79FFF054645B900F0A9FD14B116
:10B8D000204600F06BFC0020BDE8FE8FF81C20F035
:10B8E0000300C0F5147080B2484501DD484605E00C
:10B8F000F81C20F00300C0F5147080B283460020CD
:10B90000CDE9008005F110003844C01C20F003018F
:10B910005B464A46284600F074FD00BF287900F0D7
:10B920000300002808D000BF3CA34FF4807247A159
:10B9300052A0FAF72DFD00BF00BF00BFF81C20F099
:10B940000300C0F51470002808D100BF33A34FF4E2
:10B95000817254A149A0FAF71BFD00BF00BF0CB9CA
:10B960002C4601E0029805600295A9EB0B001FFA36
:10B9700080F90027B9F1000FA2DC4BE0F81C20F0A1
:10B980000301F01C20F00300084485B205F110000B
:10B990001FFA80F9F01C20F00300A84206D800E04E
:10B9A0002BE0F01C20F00300484501D9002093E76C
:10B9B0004846FEF7CBFB04460CB900208CE700207C
:10B9C000CDE9008004F110003844C01C20F00301D0
:10B9D00033463246204600F014FD00BF207900F0C7
:10B9E000030040B100BF0DA34FF491723AA123A010
:10B9F000FAF7CEFC00BF00BF0CE000BF00BF07A3FA
:10BA000040F227123FA11DA0FAF7C2FC00BF00BF01
:10BA1000002061E700BF20465EE700002E2E2F4D7C
:10BA20006964646C6577617265732F5468697264C8
:10BA30005F50617274792F4C7749502F7372632F66
:10BA4000636F72652F706275662E63007062756633
:10BA50005F616C6C6F633A207062756620712D3E79
:10BA60007061796C6F61642070726F7065726C794F
:10BA700020616C69676E6564000000004173736546
:10BA80007274696F6E2022257322206661696C656D
:10BA900064206174206C696E6520256420696E20C5
:10BAA00025730A00504255465F504F4F4C5F425538
:10BAB0004653495A45206D7573742062652062694A
:10BAC00067676572207468616E204D454D5F414C1B
:10BAD00049474E4D454E5400706275665F616C6C0F
:10BAE0006F633A20706275662D3E7061796C6F618C
:10BAF000642070726F7065726C7920616C69676E1A
:10BB000065640000706275665F616C6C6F633A20FB
:10BB10006572726F6E656F75732074797065000061
:10BB20002DE9FC4107460D46144600BF412C0AD0C2
:10BB3000012C08D000BF0EA34FF4A57218A11DA0C0
:10BB4000FAF726FC00BF00BF0A20FEF75BFE0646A0
:10BB500016B90020BDE8FC8100202B462A46394654
:10BB6000CDE90040304600F04CFC3046F2E70000E2
:10BB70002E2E2F4D6964646C6577617265732F5446
:10BB8000686972645F50617274792F4C7749502FE5
:10BB90007372632F636F72652F706275662E630018
:10BBA000696E76616C696420706275665F74797025
:10BBB00065000000417373657274696F6E20222501
:10BBC0007322206661696C6564206174206C696E03
:10BBD0006520256420696E2025730A002DE9FC5F2D
:10BBE00005460C4617469846DDE90C9BAA460AF125
:10BBF000030020F003002044584502D90020BDE88E
:10BC0000FC9FB9F1000F06D00AF1030020F00300F9
:10BC100000EB090600E000260220234622463146BA
:10BC2000CDE90070404600F0ECFB4046E7E700003D
:10BC300070B506460D4600BF0EB1002D09D100BFFC
:10BC40001BA340F2593226A133A0FAF7A1FB00BF93
:10BC500070BD00BF344604E0208929890844208152
:10BC6000246820680028F7D100BF208961898842B4
:10BC700008D000BF0EA340F2623231A126A0FAF72D
:10BC800087FB00BF00BF00BF206840B100BF08A312
:10BC900040F2633236A120A0FAF77AFB00BF00BF62
:10BCA0002089298908442081256000BFD0E7000051
:10BCB0002E2E2F4D6964646C6577617265732F5405
:10BCC000686972645F50617274792F4C7749502FA4
:10BCD0007372632F636F72652F706275662E6300D7
:10BCE000286820213D204E554C4C2920262620280E
:10BCF0007420213D204E554C4C29202870726F67CE
:10BD000072616D6D65722076696F6C617465732008
:10BD10004150492900000000417373657274696FD6
:10BD20006E2022257322206661696C65642061742F
:10BD3000206C696E6520256420696E2025730A00D9
:10BD4000702D3E746F745F6C656E203D3D20702DCC
:10BD50003E6C656E20286F66206C61737420706283
:10BD6000756620696E20636861696E2900000000B5
:10BD7000702D3E6E657874203D3D204E554C4C0034
:10BD80000146002002E0421C90B209680029FAD165
:10BD9000704700002DE9F04180460E461446218987
:10BDA00032464046FFF76CFD074617B90020BDE854
:10BDB000F0812146384600F045F8054600BF45B100
:10BDC00000BF05A340F224520FA114A0FAF7E0FA35
:10BDD00000BF00BF3846EAE72E2E2F4D6964646C21
:10BDE0006577617265732F54686972645F50617220
:10BDF00074792F4C7749502F7372632F636F72657C
:10BE00002F706275662E6300706275665F636F7077
:10BE100079206661696C6564000000004173736598
:10BE20007274696F6E2022257322206661696C65C9
:10BE300064206174206C696E6520256420696E2021
:10BE400025730A002DE9F04105460C46002600271F
:10BE500000BF25B11CB12889218988420CDA00BFB6
:10BE600044A340F2C9324FA15AA0FAF791FA00BF99
:10BE70006FF00F00BDE8F08100BF00BF6889801B34
:10BE80006189C91B884203D36089A0EB070802E0DF
:10BE90006889A0EB06086268D1196A689019424661
:10BEA000F4F734FA4644474400BF6889B04208D2E8
:10BEB00000BF30A340F2D93250A146A0FAF768FA89
:10BEC00000BF00BF00BF6089B84208D200BF29A3ED
:10BED00040F2DA324FA13FA0FAF75AFA00BF00BF92
:10BEE0006089B84201D8002724686889B04211D11E
:10BEF00000262D6800BF65B95CB100BF1DA34FF4DB
:10BF000079724BA133A0FAF743FA00BF6FF00F002C
:10BF1000B0E700BF002C13D06089218988420FD17F
:10BF200000BF206858B100BF12A340F2E93244A11B
:10BF300028A0FAF72DFA00BF6FF005009AE700BFBE
:10BF4000002D13D06889298988420FD100BF286845
:10BF500058B100BF07A340F2EE3239A11DA0FAF795
:10BF600017FA00BF6FF0050084E700BF002C85D1F1
:10BF700000207FE72E2E2F4D6964646C6577617217
:10BF800065732F54686972645F50617274792F4CC5
:10BF90007749502F7372632F636F72652F706275CC
:10BFA000662E6300706275665F636F70793A207405
:10BFB0006172676574206E6F742062696720656EB8
:10BFC0006F75676820746F20686F6C6420736F757D
:10BFD00072636500417373657274696F6E20222508
:10BFE0007322206661696C6564206174206C696EDF
:10BFF0006520256420696E2025730A006F666673CC
:10C0000065745F746F203C3D20705F746F2D3E6CD3
:10C01000656E00006F66667365745F66726F6D2093
:10C020003C3D20705F66726F6D2D3E6C656E00004A
:10C03000705F746F20213D204E554C4C0000000075
:10C04000706275665F636F7079282920646F65730D
:10C05000206E6F7420616C6C6F77207061636B650C
:10C060007420717565756573210000002DE9F05F1E
:10C070008046894616461D464FF0000AD34600BF4B
:10C08000B8F1000F0BD100BF21A340F20A422CA14E
:10C0900033A0FAF77DF900BF0020BDE8F09F00BF94
:10C0A00000BFB9F1000F0AD100BF19A340F20B4243
:10C0B00035A12BA0FAF76CF900BF0020EDE700BF17
:10C0C000444620E035B16089A84203DC6089281A23
:10C0D00085B217E06089401B87B2B74200DD374662
:10C0E0006268511909EB0A003A46F4F70FF90BEBB5
:10C0F00007001FFA80FB0AEB07001FFA80FAF01B0B
:10C1000086B2002524680EB1002CDBD15846C4E766
:10C110002E2E2F4D6964646C6577617265732F54A0
:10C12000686972645F50617274792F4C7749502F3F
:10C130007372632F636F72652F706275662E630072
:10C14000706275665F636F70795F70617274696148
:10C150006C3A20696E76616C6964206275660000D5
:10C16000417373657274696F6E2022257322206695
:10C1700061696C6564206174206C696E652025645A
:10C1800020696E2025730A00706275665F636F70A8
:10C19000795F7061727469616C3A20696E76616C66
:10C1A0006964206461746170747200002DE9F04765
:10C1B0000446002C0ED100BF44B900BF38A34FF491
:10C1C000377243A145A0FAF7E3F800BF00BF002093
:10C1D000BDE8F08700265EE001F0E2F8824600BF8D
:10C1E000A07B002808DC00BF2DA340F2F12245A16E
:10C1F0003AA0FAF7CDF800BF00BFA07B401E00F0C8
:10C20000FF0884F80E80504601F0D6F8B8F1000F10
:10C210003FD12768207B00F00F05607B00F0020013
:10C22000002814D0A14600BFD9F81000002808D17A
:10C2300000BF1BA340F2FF2238A128A0FAF7A8F8FC
:10C2400000BF00BF2046D9F8101088471DE0022D1E
:10C2500004D121460B20FEF707FA16E0012D04D188
:10C2600021460A20FEF700FA0FE01DB92046FDF72F
:10C27000BFFD0AE000BF00BF09A340F20F3230A1AA
:10C2800016A0FAF785F800BF00BF701CC6B23C4686
:10C2900000E0002400BF002C9ED1304698E700004B
:10C2A0002E2E2F4D6964646C6577617265732F540F
:10C2B000686972645F50617274792F4C7749502FAE
:10C2C0007372632F636F72652F706275662E6300E1
:10C2D0007020213D204E554C4C0000004173736589
:10C2E0007274696F6E2022257322206661696C6505
:10C2F00064206174206C696E6520256420696E205D
:10C3000025730A00706275665F667265653A207013
:10C310002D3E726566203E203000000070632D3E89
:10C32000637573746F6D5F667265655F66756E6366
:10C3300074696F6E20213D204E554C4C000000006A
:10C34000696E76616C6964207062756620747970BC
:10C350006500000070B50446254629460748FEF7EB
:10C36000DBF907480078012806D10020044908704D
:10C3700004480068FFF75AF970BD0000EC6D010831
:10C38000300000203400002070B500BF01F008F834
:10C390000546002009490870284601F00DF800BF45
:10C3A0000748046806E0606F18B1204602F00CFBF5
:10C3B00070BDE468002CF6D100BFF9E73D01002014
:10C3C0005001002010B50446FFF7DEFF10BD70B528
:10C3D00004460D4601222946204600F001F870BDB2
:10C3E00070B505460C461646002C04DA6142284614
:10C3F00000F040F970BD324621462846FFF7CCF9DF
:10C40000F8E770B5DDE90445002606604160028169
:10C41000438104734573012686730026C67370BD7D
:10C4200070B500F0BDFF05460C48047801200B49AB
:10C430000870284600F0C0FF7CB900BF0021084802
:10C4400008F00CFD40B100F0ABFF054600200349A9
:10C450000870284600F0B0FF00BF70BD3D0100200D
:10C46000C5C300082DE9F04106460F4600BF002E67
:10C4700008D100BF2CA34FF4CC7237A13CA0F9F730
:10C4800087FF00BF00BF3089B84201DCBDE8F08102
:10C490003089C01B1FFA80F83D46344613E060899E
:10C4A000281A85B22089A0EB08002081246800BFEB
:10C4B00044B900BF1CA340F2AF1237A12CA0F9F77A
:10C4C00067FF00BF00BF6089A842E8DB207B00F067
:10C4D0000F0000281BD16089A84218D0607B00F0B3
:10C4E0000200002813D1A088001B284481B22046F6
:10C4F000FDF792FF044600BF44B900BF0AA340F213
:10C50000BD122BA11AA0F9F743FF00BF00BF658140
:10C5100060892081206810B12068FFF747FE002065
:10C52000206000BFB2E700002E2E2F4D6964646CBE
:10C530006577617265732F54686972645F506172C8
:10C5400074792F4C7749502F7372632F636F726524
:10C550002F706275662E6300706275665F7265612A
:10C560006C6C6F633A207020213D204E554C4C007E
:10C57000417373657274696F6E2022257322206681
:10C5800061696C6564206174206C696E6520256446
:10C5900020696E2025730A00706275665F7265619E
:10C5A0006C6C6F633A207120213D204E554C4C003D
:10C5B0006D656D5F7472696D2072657475726E65FC
:10C5C000642071203D3D204E554C4C0070B5044612
:10C5D000002C18D000BF00F0E3FE0546A07B401CF5
:10C5E000A073284600F0E8FE00BF00BFA07B002833
:10C5F00008DC00BF04A340F242320FA113A0F9F7F8
:10C60000C7FE00BF00BF70BD2E2E2F4D6964646C45
:10C610006577617265732F54686972645F506172E7
:10C6200074792F4C7749502F7372632F636F726543
:10C630002F706275662E6300706275662072656683
:10C64000206F766572666C6F7700000041737365CA
:10C650007274696F6E2022257322206661696C6591
:10C6600064206174206C696E6520256420696E20E9
:10C6700025730A002DE9F04104460D4600BF44B978
:10C6800000BF18A340F24B2222A125A0F9F780FE9B
:10C6900000BF00BF14B1B5F5803F02D30120BDE853
:10C6A000F0810DB90020FAE7AEB200BF6089B04258
:10C6B0000ADA00BF0BA340F2552223A118A0F9F714
:10C6C00067FE00BF0120EAE700BF67686068284492
:10C6D00060606089801B60812089801B2081002030
:10C6E000DDE700002E2E2F4D6964646C6577617262
:10C6F00065732F54686972645F50617274792F4C4E
:10C700007749502F7372632F636F72652F70627554
:10C71000662E63007020213D204E554C4C000000D9
:10C72000417373657274696F6E20222573222066CF
:10C7300061696C6564206174206C696E6520256494
:10C7400020696E2025730A00696E6372656D656EDF
:10C75000745F6D61676E6974756465203C3D20701F
:10C760002D3E6C656E0000002DE9F041044600BFCF
:10C770003B480068844208D200BF3AA340F2DF126F
:10C7800044A14AA0F9F704FE00BF00BF00BF514812
:10C790000068844208D300BF32A34FF4F0724EA168
:10C7A00042A0F9F7F5FD00BF00BF00BF20790028C7
:10C7B00008D000BF2BA340F2E1124EA13BA0F9F735
:10C7C000E7FD00BF00BF00BF2088B0F5C86F08D9E3
:10C7D00000BF24A34FF4F2724DA134A0F9F7D8FDA5
:10C7E00000BF00BF208800F0F3FB0546AC4219D023
:10C7F0002879B8B937480068854213D04F48006897
:10C80000A84201D14D480460288820802888B0F5CE
:10C81000C86F07D02046FDF7F7FD0746288800F0CF
:10C82000D7FB4780608800F0D3FB0646A64215D0B0
:10C83000307998B941480068A04201D13F4806606C
:10C84000208830802088B0F5C86F07D03046FDF7CB
:10C85000DBFD0746208800F0BBFB4780BDE8F08188
:10C86000F00000202E2E2F4D6964646C6577617294
:10C8700065732F54686972645F50617274792F4CCC
:10C880007749502F7372632F636F72652F6D656DDB
:10C890002E630000706C75675F686F6C65733A207B
:10C8A0006D656D203E3D2072616D000041737365C2
:10C8B0007274696F6E2022257322206661696C652F
:10C8C00064206174206C696E6520256420696E2087
:10C8D00025730A00F4000020706C75675F686F6C48
:10C8E00065733A206D656D203C2072616D5F656EE9
:10C8F00064000000706C75675F686F6C65733A2048
:10C900006D656D2D3E75736564203D3D20300000E2
:10C91000706C75675F686F6C65733A206D656D2D1F
:10C920003E6E657874203C3D204D454D5F53495A1D
:10C93000455F414C49474E4544000000FC00002043
:10C940002DE9F04105460E461C4807681C48006862
:10C95000001D08F075FD50B91948006890F82C10BA
:10C960000120884017490968814316480160681C06
:10C9700038B936B112480168091D134808F0AAFDFC
:10C980001AE07C190E4800684460BC4207D20C488B
:10C990000168091D0D48006808F082FD0CE0084898
:10C9A0000168091D0A48006808F07AFD0948006816
:10C9B000844201D207480460BDE8F0818C00002069
:10C9C00078000020900000209C8200208000002041
:10C9D0007C000020A800002010B5044608F086FD69
:10C9E00023480068401C224908602248006840B97A
:10C9F000204804600846006801280DD100F0BEF907
:10CA00000AE01D48006838B91A480068C06AE16A3F
:10CA1000884201D81748046018480068401C17492C
:10CA2000086094F82C1001208840154909680843D3
:10CA300013490860E16A01EB8101124A02EB8100AF
:10CA4000211D08F047FD08F07BFD0B48006868B128
:10CA500008480068C06AE16A884207D24FF08050F7
:10CA600009490860BFF34F8FBFF36F8F10BD0000FF
:10CA7000880000207800002094000020A4000020FE
:10CA800090000020CC7F002004ED00E010B516E0FF
:10CA900008F02CFD0C48C068C468201D08F0D0FCCC
:10CAA0000A480068401E0949086009480068401E9D
:10CAB0000749086008F044FD204600F05FF804488C
:10CAC00000680028E4D110BD888200208800002082
:10CAD0008400002070B504460D46206C70B1216CB6
:10CAE000E0680144E160D4E90210884201D3216882
:10CAF000E1602846226CE168F3F708FC70BD2DE97F
:10CB0000F04104460F4615464FF00008A66B206C16
:10CB100048B9206800282CD1A06809F01DFF804684
:10CB20000020A06025E07DB93946226C6068F3F7EB
:10CB3000EDFB216C606808446060D4E90101884223
:10CB400017D32068606014E03946226CE068F3F780
:10CB5000DDFB216CE068411AE1602168E0688842F1
:10CB600003D2216CA068411AE160022D01D106B107
:10CB7000761E701CA0634046BDE8F08110B50446E7
:10CB800094F8590030B9206B08F0F8FC204608F002
:10CB9000F5FC1AE094F85900012803D1204608F06A
:10CBA000EDFC12E094F85900022801D1012000E0C8
:10CBB000002050B900BF502080F31188BFF34F8F81
:10CBC000BFF36F8F00BF00BFFEE710BD01464A6A8A
:10CBD00022B10A6B1268C2F1200000E00020704709
:10CBE00030B54FF47053174800F007042CB1C01D46
:10CBF00020F00700134C041B1B1B0246124C226042
:10CC00000024114D6C60D018083820F007000F4C3C
:10CC1000206000240D4D2D686C600C4D2D682C603B
:10CC20001146441A4C60094C24680C60084D4C684D
:10CC30002C60084D4C682C604FF00044064D2C6071
:10CC400030BD0000B0820020B4000020BC000020F5
:10CC5000C4000020C0000020D000002000BFFFF76B
:10CC600015FF064800680128F9D94FF080500449A3
:10CC70000860BFF34F8FBFF36F8FF0E7CC7F0020CA
:10CC800004ED00E010B5044654B10020A06020601F
:10CC90000021E16000231A461946204609F00AF9EE
:10CCA00010BD2DE9F04106460D4617469846069CF4
:10CCB0000DB9246000E02760E66325640121204669
:10CCC00009F0ACF8BDE8F0812DE9FF5F81460E4622
:10CCD0009246DDE90E7B109CAAF10100216B01EB6D
:10CCE000800828F0070808F0070008B9012000E0D4
:10CCF000002050B900BF502080F31188BFF34F8F40
:10CD0000BFF36F8F00BF00BFFEE786B1002507E0CD
:10CD1000715D04F134004155705D00B902E06D1C95
:10CD2000182DF5D300BF00214B20015502E0002053
:10CD300084F83400202F00D31F27E762E764002027
:10CD40002065201D08F0A9FB04F1180008F0A5FBE0
:10CD50002461C7F12000A06164620020606584F84E
:10CD6000580049464046039A00F0F0F92060BBF1B4
:10CD7000000F01D0CBF80040BDE8FF9F10B50024A4
:10CD800007E004EB84010F4A02EB810008F078FB16
:10CD9000641C202CF5D30C4808F072FB0B4808F0FB
:10CDA0006FFB0B4808F06CFB0A4808F069FB0A4867
:10CDB00008F066FB0448094908600448084908600F
:10CDC00010BD0000CC7F00204C820020608200203B
:10CDD00074820020888200209C8200207C00002039
:10CDE0008000002010B50146164800E00068036886
:10CDF0008B42FBD30246436813448B4204D1436801
:10CE00004C682344436001460A464B681344046857
:10CE1000A34211D10C4C03682468A34208D04B688C
:10CE20000468646823444B6003681B680B6005E07A
:10CE3000054B1B680B6001E003680B60884200D063
:10CE4000016010BDB4000020BC00002070B5054694
:10CE500008F04CFBA86B08B9012400E0002408F09E
:10CE60006FFB204670BD70B5054608F03FFBA86B10
:10CE7000E96B884201D1012400E0002408F060FB46
:10CE8000204670BD0A490968096809B9012100E016
:10CE9000002121B14FF0FF31064A116006E004493C
:10CEA0000968C968C868034A416811607047000092
:10CEB0007C000020A80000200E480068401C08B933
:10CEC000012000E0002050B900BF502080F31188FD
:10CED000BFF34F8FBFF36F8F00BF00BFFEE700BFF0
:10CEE000502080F31188BFF34F8FBFF36F8F00BFC7
:10CEF00000BFFEE7D400002010B502460020114616
:10CF000052B900BF502383F31188BFF34F8FBFF393
:10CF10006F8F00BF00BFFEE70B4C4B69A34201D1EE
:10CF2000012300E0002373B1084C8B6AA34201D1B6
:10CF3000012300E0002333B98B6A0BB9012300E021
:10CF4000002303B1012010BD9C82002074820020C8
:10CF500070B5044608F0CAFA94F9455010E0606ACA
:10CF600008B9012000E0002038B904F1240009F0DC
:10CF7000B3FD18B108F0DEFB00E003E0681E45B227
:10CF8000002DECDC00BFFF2084F8450008F0D8FA43
:10CF900008F0ACFA94F9445010E0206908B9012077
:10CFA00000E0002048B904F1100009F095FD08B137
:10CFB00008F0C0FB681E45B200E001E0002DECDC8B
:10CFC00000BFFF2084F8440008F0BAFA70BD0000EA
:10CFD000014602480068084470470000F000002045
:10CFE0002DE9F04104464FF0000808F051FD494892
:10CFF000006808B9FFF7F4FD4748006820400028A2
:10D0000070D1D4B1083404F00700B0B104F00700C7
:10D01000C0F10800044404F0070008B9012000E052
:10D02000002050B900BF502080F31188BFF34F8F0C
:10D03000BFF36F8F00BF00BFFEE7002C52D0374810
:10D04000006884424ED8364E3046056801E02E46D0
:10D050002D686868A04202D228680028F7D12D48C0
:10D06000006885423ED0306800F1080828683060CA
:10D070006868001B102819D92F1907F0070008B994
:10D08000012000E0002050B900BF502080F311883B
:10D09000BFF34F8FBFF36F8F00BF00BFFEE768681D
:10D0A000001B78606C603846FFF79CFE1B4968687F
:10D0B0000968081A1949086008460068194909688A
:10D0C000884203D21548006816490860124968680A
:10D0D0000968084368600020286013480068401C05
:10D0E0001149086009F044FD08F0070008B9012063
:10D0F00000E0002050B900BF502080F31188BFF33A
:10D100004F8FBFF36F8F00BF00BFFEE74046BDE803
:10D11000F0810000BC000020D0000020C0000020F2
:10D12000B4000020C4000020C800002006480068A9
:10D1300030B10549096801F15000096D491C0160D1
:10D14000014800687047000078000020001F4FF081
:10D1500080730360001F21F001030360001F054B73
:10D16000036014380260001F6FF002030360203870
:10D1700070470000B9CE0008F8B506460C461546C3
:10D180004FF47A702B46084A214600903046F5F756
:10D1900031FF10B14FF0FF30F8BD2A46024920465A
:10D1A000F3F7B4F80020F7E708F70020F9F74CFB95
:10D1B00000BF0C480068FEF7DFFA002400BF04E05F
:10D1C0002046F9F729FA601CC4B20A2CF8DBF9F7FB
:10D1D00055FC04480068FEF7B5FA0A2008F070FA1A
:10D1E000E7E700001C000020F9F7C2FC00BF0E4872
:10D1F0000068FEF7C1FA0D48D0ED000AB0EE600AF3
:10D200000120F9F7CFFC0948D0ED010AB0EE600A21
:10D210000220F9F7C7FC04480068FEF793FA64207F
:10D2200008F04EFAE3E70000200000200000002094
:10D2300000BFFCF74DFB07F04BFF07F071FE0A2023
:10D2400008F03EFAF5E700BF08F064F8642008F043
:10D2500037FAF9E700BF04210448F5F741F907F070
:10D26000AFFF4FF4FA7008F02BFAF4E70004024025
:10D2700008B5F7F72FFF00F0EFFF07F0DDFE00BF66
:10D28000002000906B46012200212348F4F7C6FCE1
:10D290000098C0F3800090BB2048FDF75DFF1F4859
:10D2A000FDF7E2FE1E480078012806D11D480068FF
:10D2B00000F09AFB00201A4908701B4800780128EA
:10D2C00006D11A48006800F08FFB0020164908704C
:10D2D00017480078012806D11648006800F084FB42
:10D2E0000020134908701448007801280ED1134813
:10D2F000006800F079FB00200F49087006E0FFE7A6
:10D300000648FDF799FF0548FEF70AF84FF47A70D2
:10D3100008F0D6F9B4E700006C7E0020747F00208E
:10D3200008000020A801002009000020AC01002016
:10D330000B000020B40100200C000020B8010020E8
:10D34000F0B587B004460D461646FEF768F8074666
:10D35000AEB1324601A82168FEF780F801A807C8DF
:10D3600004AB07C30498102806D105982860FEF77F
:10D3700056F8C01B07B0F0BD4FF0FF30FAE74FF092
:10D38000FF3201A82168FEF769F801A807C804ABBD
:10D3900007C305982860FEF742F8C01BEAE70000C3
:10D3A00010B54FF0FF3103480068FEF70BF901207C
:10D3B00010BD0000A401002010B50446024800681A
:10D3C000FEF7D8F810BD0000A40100202DE9F041BF
:10D3D00000F07EF8074600BF0F4804680CB9BDE8AE
:10D3E000F0816068381AB0F1004F01D3012000E0ED
:10D3F000002000B1F3E7084920680860A568E668E6
:10D4000006496068086021460920FDF72DF90DB135
:10D410003046A847E0E70000880100208C0100208A
:10D4200010B50348FEF798F80249086010BD0000E7
:10D43000906F0108A40100207FB504460D46094BFA
:10D440000FCB8DE80F00009500216846FDF7F1FF36
:10D450002060206818B94FF0FF3004B070BD002084
:10D46000FBE70000986F010870B505460E460022E4
:10D4700031462868FEF740F808B9002401E04FF073
:10D48000FF34204670BD0146086808B90020704787
:10D490000120FCE710B504464FF0FF312068FEF78D
:10D4A00091F810BD1CB5044600200090019068461C
:10D4B000FEF752F82060206810B94FF0FF301CBD15
:10D4C0000020FCE710B504462068FEF753F810BDB5
:10D4D00010B5F5F715F810BD2DE9F04188B00446F8
:10D4E0000D4616461F46DDF838801C2101A8F2F7CC
:10D4F00034FF019402950FFA88F0ADF80C000597FF
:10D50000314601A8FEF7EEF808B0BDE8F081000052
:10D510002DE9F04104460E46174600BFB4F1804F96
:10D5200008D300BF09A340F2291215A122A0F8F7E1
:10D530002FFF00BF00BFFFF7CBFF05193A4631466A
:10D54000284600F04DF8BDE8F08100002E2E2F4D4A
:10D550006964646C6577617265732F54686972647D
:10D560005F50617274792F4C7749502F7372632F1B
:10D57000636F72652F74696D656F7574732E6300C8
:10D5800054696D656F75742074696D6520746F6F73
:10D59000206C6F6E672C206D6178206973204C576A
:10D5A00049505F55494E5433325F4D41582F342016
:10D5B0006D73656373000000417373657274696F06
:10D5C0006E2022257322206661696C656420617477
:10D5D000206C696E6520256420696E2025730A0021
:10D5E0002DE9F04106460F4690460920FDF70AF95D
:10D5F0000446002C0CD100BF07D100BF20A3BE22DF
:10D600002CA13CA0F8F7C4FE00BF00BFBDE8F0812C
:10D6100000202060A760C4F80C8066603F48006866
:10D6200010B93E480460F1E73C4960680968496800
:10D63000401AB0F1004F01D3012000E0002028B1D2
:10D640003648006820603548046017E033480568B4
:10D6500011E0286850B1606829684968401AB0F143
:10D66000004F01D3012000E0002018B1286820609D
:10D670002C6002E02D68002DEBD100BF00BFC5E794
:10D680002E2E2F4D6964646C6577617265732F541B
:10D69000686972645F50617274792F4C7749502FBA
:10D6A0007372632F636F72652F74696D656F757424
:10D6B000732E63007379735F74696D656F75743A67
:10D6C0002074696D656F757420213D204E554C4C5A
:10D6D0002C20706F6F6C204D454D505F5359535F38
:10D6E00054494D454F555420697320656D707479C8
:10D6F00000000000417373657274696F6E2022250B
:10D700007322206661696C6564206174206C696EA7
:10D710006520256420696E2025730A008801002099
:10D7200010B5012408E0064901EBC40251F83400A9
:10D730000449FFF7EDFE641C032CF4D310BD000078
:10D740006C6F0108FD9B000870B51548006810B9A2
:10D750004FF0FF3070BDFFF7BBFE04461048006875
:10D760004068001BB0F1004F01D3012000E0002011
:10D7700008B10020EEE70A4800684068051B00BFBA
:10D78000B5F1004F08D300BF06A34FF4DC7212A11D
:10D7900016A0F8F7FDFD00BF00BF2846DAE700003D
:10D7A000880100202E2E2F4D6964646C65776172AC
:10D7B00065732F54686972645F50617274792F4C7D
:10D7C0007749502F7372632F636F72652F74696D81
:10D7D000656F7574732E6300696E76616C69642081
:10D7E000736C65657074696D6500000041737365E5
:10D7F0007274696F6E2022257322206661696C65E0
:10D8000064206174206C696E6520256420696E2037
:10D8100025730A002DE9FF5F04460E4600BF002C69
:10D820000AD100BF42A340F23D224DA153A0F8F718
:10D83000AFFD00BFBDE8FF9F00BF00BF207D0128F6
:10D8400008D100BF3AA34FF4107256A14BA0F8F7CD
:10D850009FFD00BF00BF207D0A2807D121465E48FA
:10D8600003F0B8F9204600F069FF5FE04FF0000ACE
:10D87000D346276DD4F82480D4F89050D4F8109073
:10D88000207DE8B9E08A38B300BF54480068A04260
:10D8900005D152480068C068504908600DE04F4902
:10D8A000086806E0C168A14202D1E168C16002E0F7
:10D8B000C0680028F6D100BF00BF0020E0600BE088
:10D8C000B246B4F816B000BF2146454803F082F9CD
:10D8D00001204449087000BF206F10B1206F05F08F
:10D8E000CEF9E06E10B1E06E05F0C9F9606F10B1CD
:10D8F000606F05F0C4F9BAF1000F0AD0208B211D2A
:10D9000023464246CDE9001B02903946204605F0E9
:10D91000BBF8207D0390204600F010FF00BF1DB132
:10D920006FF00C014846A84700BF00BF00BF81E769
:10D930002E2E2F4D6964646C6577617265732F5468
:10D94000686972645F50617274792F4C7749502F07
:10D950007372632F636F72652F7463702E630000A0
:10D960007463705F6162616E646F6E3A20696E7697
:10D97000616C69642070636200000000417373652C
:10D980007274696F6E2022257322206661696C654E
:10D9900064206174206C696E6520256420696E20A6
:10D9A00025730A00646F6E27742063616C6C2074A9
:10D9B00063705F61626F72742F7463705F61626124
:10D9C0006E646F6E20666F72206C697374656E2D65
:10D9D00070636273000000005401002048010020C1
:10D9E000500100205801002010B5044601212046B6
:10D9F000FFF710FF10BD28B1027D012A02D10246B7
:10DA0000916100BF7047000070B505460C46164690
:10DA100000BF002C08D100BF07A340F20F3212A1B3
:10DA200019A0F8F7B5FC00BF00BF2046FFF7DCFFE8
:10DA30006FF00C0070BD00002E2E2F4D6964646CD9
:10DA40006577617265732F54686972645F506172A3
:10DA500074792F4C7749502F7372632F636F7265FF
:10DA60002F7463702E6300007463705F616363657D
:10DA700070745F6E756C6C3A20696E76616C696467
:10DA80002070636200000000417373657274696FF7
:10DA90006E2022257322206661696C6564206174A2
:10DAA000206C696E6520256420696E2025730A004C
:10DAB00070B505460020FCF7A5FE04461CBB00F02F
:10DAC000B1FF01F05FFD0020FCF79CFE0446CCB9DD
:10DAD000092001F0EFFC0020FCF794FE044684B915
:10DAE000082001F0E7FC0020FCF78CFE04463CB95E
:10DAF000284601F0ABFC0020FCF784FE044600BF82
:10DB000000BF00BF00BF44B39C212046F2F725FCB4
:10DB10000C3465724FF48660A4F858004000E0832E
:10DB2000A083FF2004F8010C4FF40670E084062067
:10DB3000A0866086C01FA0840120A08708480068D6
:10DB4000606108480078A0744FF48660E08706485A
:10DB5000A0670648C4F888000C3C204670BD000051
:10DB6000440100205A0100204D23010800DD6D0012
:10DB70002DE9F04705460C4617464FF0040904B955
:10DB80002E4C00BF002D0CD100BF2DA340F2A922C6
:10DB900037A13DA0F8F7FCFB00BF6FF00F00BDE818
:10DBA000F08700BF00BF287D00280BD000BF24A352
:10DBB00040F2AB223EA134A0F8F7EAFB00BF6FF0C1
:10DBC0000500ECE700BF37B901F0DEFF07460FBBE9
:10DBD0006FF00100E3E74FF0000819E03E4850F80D
:10DBE0002800066810E0F08AB8420CD146B13068CF
:10DBF00030B12CB1206818B130682168884202D158
:10DC00006FF00700CBE7F668002EECD108F10108B1
:10DC1000C845E3DB34B1206820B10CB9002000E036
:10DC200020682860EF8200BF2C480068E8602B481D
:10DC3000056005F043FE00BF0020B0E7886F0108D3
:10DC40002E2E2F4D6964646C6577617265732F5455
:10DC5000686972645F50617274792F4C7749502FF4
:10DC60007372632F636F72652F7463702E6300008D
:10DC70007463705F62696E643A20696E76616C6984
:10DC80006420706362000000417373657274696F91
:10DC90006E2022257322206661696C6564206174A0
:10DCA000206C696E6520256420696E2025730A004A
:10DCB0007463705F62696E643A2063616E206F6E98
:10DCC0006C792062696E6420696E2073746174657A
:10DCD00020434C4F534544005C6F0108480100202D
:10DCE00010B5044600BF002C0BD100BF0CA34FF4AD
:10DCF000F47217A11CA0F8F74BFB00BF6FF00F00E8
:10DD000010BD00BF207D012805D000BF608B40F012
:10DD10001000608300BF0121204600F039F8EFE7D2
:10DD20002E2E2F4D6964646C6577617265732F5474
:10DD3000686972645F50617274792F4C7749502F13
:10DD40007372632F636F72652F7463702E630000AC
:10DD50007463705F636C6F73653A20696E76616C93
:10DD60006964207063620000417373657274696F47
:10DD70006E2022257322206661696C6564206174BF
:10DD8000206C696E6520256420696E2025730A0069
:10DD90003EB504460D4600BF002C08D100BF55A378
:10DDA0004FF4AF725FA167A0F8F7F2FA00BF00BFAF
:10DDB000002D56D0207D042802D0207D072850D188
:10DDC000A06F18B9208DB0F5066F4AD000BFA07EB5
:10DDD00000F0100040B900BF46A34FF4B27263A137
:10DDE00058A0F8F7D5FA00BF00BF208BE18A221DAA
:10DDF000CDE90021029023462046626A216D04F09D
:10DE000043FE204602F078FE00BF00BF5E48006877
:10DE1000A04205D15C480068C0685B4908600DE01D
:10DE20005949086806E0C168A14202D1E168C160B1
:10DE300002E0C0680028F6D100BF00BF0020E0600B
:10DE400000BF01205149087000BF51480068A0423E
:10DE500002D105F003FE02E0204600F06FFC002036
:10DE60003EBD207D20B1012824D002283AD12CE0EB
:10DE7000E08AD8B100BF47480068A04205D14548B4
:10DE80000068C068434908600DE04249086806E040
:10DE9000C168A14202D1E168C16002E0C068002807
:10DEA000F6D100BF00BF0020E06000BF204600F0B8
:10DEB00045FC1BE0204601F083FB2146364802F07A
:10DEC00089FE204600F032FD10E000BF21462E48BA
:10DED00002F080FE01202D49087000BF204600F0AE
:10DEE0002DFC03E0204600F059F8B9E700BF002000
:10DEF000B6E700002E2E2F4D6964646C6577617261
:10DF000065732F54686972645F50617274792F4C25
:10DF10007749502F7372632F636F72652F7463702C
:10DF20002E6300007463705F636C6F73655F73686A
:10DF30007574646F776E3A20696E76616C696420DF
:10DF400070636200417373657274696F6E2022257D
:10DF50007322206661696C6564206174206C696E4F
:10DF60006520256420696E2025730A007063622D88
:10DF70003E666C61677320262054465F5258434CBE
:10DF80004F5345440000000050010020580100207C
:10DF900084010020480100204C01002070B5054696
:10DFA00000BF45B900BF1EA34FF4CE7228A12BA01D
:10DFB000F8F7EEF900BF00BF287D032804D004283D
:10DFC0000AD0072818D10FE0284604F005FF0446C0
:10DFD0000CB90520287511E0284604F0FDFE044622
:10DFE0000CB90520287509E0284604F0F5FE044622
:10DFF0000CB90920287501E0002070BD00BF1CB9D4
:10E00000284601F0E3FE09E0601C38B900BF688BC8
:10E0100040F00800688300BF0020EEE72046ECE7F0
:10E020002E2E2F4D6964646C6577617265732F5471
:10E03000686972645F50617274792F4C7749502F10
:10E040007372632F636F72652F7463702E630000A9
:10E0500070636220213D204E554C4C004173736526
:10E060007274696F6E2022257322206661696C6567
:10E0700064206174206C696E6520256420696E20BF
:10E0800025730A002DE9F05F80460D4691469A46B9
:10E090000A9F00BFB8F1000F07D100BF40A3A32221
:10E0A0004CA154A0F8F774F900BF00BF00BF002DC9
:10E0B00007D100BF3AA3A42258A14EA0F8F768F9EF
:10E0C00000BF00BF07F0010008B1042000E00020FD
:10E0D00007F0020109B1002100E00021084407F027
:10E0E000080109B1002100E00021084407F01001F7
:10E0F00009B1002100E0002146180220FCF782FB54
:10E10000041E05D12846FEF751F80020BDE8F09F17
:10E11000A77200202060656000BF2889B04207DA3E
:10E1200000BF1FA3B02246A132A0F8F731F900BF0B
:10E1300000BF2889801B208114212846FDF723FB7E
:10E1400020B1204604F08EFD0020DFE760684068C3
:10E15000E060B8F81600FBF786FDE1680880B8F8C3
:10E160001800FBF780FDE16848805046FBF76EFD24
:10E17000E1684860B346F11706EB91718910491DBB
:10E180004FF6FF7202EA013141EA0900FBF76BFD2D
:10E19000E16888810020E16848822046B6E70000F7
:10E1A0002E2E2F4D6964646C6577617265732F54F0
:10E1B000686972645F50617274792F4C7749502F8F
:10E1C0007372632F636F72652F7463705F6F757402
:10E1D0002E6300007463705F6372656174655F73C2
:10E1E00065676D656E743A20696E76616C6964204E
:10E1F00070636200417373657274696F6E202225CB
:10E200007322206661696C6564206174206C696E9C
:10E210006520256420696E2025730A007463705F91
:10E220006372656174655F7365676D656E743A20CE
:10E23000696E76616C69642070627566000000002A
:10E24000702D3E746F745F6C656E203E3D206F7064
:10E25000746C656E000000002DE9F041002400257B
:10E260000026002701F08AFC044641F28932224947
:10E270002046FFF77DFCFF21204601F005FB044608
:10E280001E492046FFF7B7FB01F078FC054641F236
:10E290008A3219492846FFF76BFCFF21284601F016
:10E2A000F3FA054616492846FFF7A5FB01F066FC80
:10E2B000064641F2717210493046FFF759FCFF21C2
:10E2C000304601F0E1FA06460E493046FFF793FB6F
:10E2D00001F054FC074641F28B3207493846FFF7FC
:10E2E00047FCFF21384601F0CFFA07460649384679
:10E2F000FFF781FBBDE8F081886F0108194701082D
:10E300003D470108D1460108F54601082DE9F041D5
:10E3100006460D46174600BF002F08D100BF10A3C8
:10E3200040F6C5021AA124A0F8F732F800BF00BFDA
:10E3300015B93046BDE8F0812C8D74B12820844297
:10E3400002DD211A89B200E000218846464501DA43
:10E35000314600E041460E4600BF3046EAE7000085
:10E360002E2E2F4D6964646C6577617265732F542E
:10E37000686972645F50617274792F4C7749502FCD
:10E380007372632F636F72652F7463702E63000066
:10E390007463705F6566665F73656E645F6D7373EB
:10E3A0005F6E657469663A20696E76616C69642097
:10E3B0006473745F69700000417373657274696F90
:10E3C0006E2022257322206661696C656420617469
:10E3D000206C696E6520256420696E2025730A0013
:10E3E0002DE9F84304460D460027B94600BF05F065
:10E3F000030040B900BF60A340F211426B496CA01A
:10E40000F7F7C6FF00BF00BF00BF002C08D100BF58
:10E4100059A340F2134270A165A0F7F7B9FF00BFFE
:10E4200000BF05F0020000B1012707F0010008B1AC
:10E43000042000E0002007F0020109B1002100E003
:10E440000021084407F0080109B1002100E0002183
:10E45000084407F0100109B1002100E0002100EBA1
:10E4600001094FF4207249463620FDF709FAB0F150
:10E47000000809D100BF608B40F08000608300BFBE
:10E480004FF0FF30BDE8F88300BFB8F80A004845F8
:10E4900008DA00BF38A340F2394257A144A0F7F789
:10E4A00077FF00BF00BF00972A4641462046E36D34
:10E4B000FFF7E8FD061E07D100BF608B40F080002B
:10E4C000608300BF701EDDE700BF307B00F00300FB
:10E4D00040B100BF28A340F2424256A134A0F7F752
:10E4E00057FF00BF00BF00BF308940B100BF22A36B
:10E4F00040F2434255A12EA0F7F74AFF00BF00BFEC
:10E50000E06E08B9E66607E0E06E00E000680168CA
:10E510000029FBD1066000BF0020A4F8680005F0C8
:10E52000020010B905F0010010B1E06D401CE0657B
:10E5300005F0010028B100BF608B40F0200060832F
:10E5400000BF7068FDF71CFC34F8661F084420808B
:10E5500034F8660970B100BF206F50B9E06E40B961
:10E5600000BF05A340F2654243A111A0F7F710FFD9
:10E5700000BF00BF002085E72E2E2F4D6964646C1C
:10E580006577617265732F54686972645F50617258
:10E5900074792F4C7749502F7372632F636F7265B4
:10E5A0002F7463705F6F75742E630000C070010874
:10E5B000417373657274696F6E2022257322206621
:10E5C00061696C6564206174206C696E65202564E6
:10E5D00020696E2025730A007463705F656E717523
:10E5E0006575655F666C6167733A20696E76616C0C
:10E5F00069642070636200007463705F656E71759A
:10E600006575655F666C6167733A20636865636B07
:10E610002074686174206669727374207062756614
:10E620002063616E20686F6C64206F70746C656E1F
:10E63000000000007365672D3E746370686472208B
:10E640006E6F7420616C69676E6564007463705FDF
:10E65000656E71756575655F666C6167733A206993
:10E660006E76616C6964207365676D656E74206C8D
:10E67000656E6774680000007463705F656E717525
:10E680006575655F666C6167733A20696E76616C6B
:10E690006964207175657565206C656E67746800C6
:10E6A00070B523480078401C2149087000BF2148FC
:10E6B000046839E0A07F1E490978884233D01C489D
:10E6C0000078A077A07E00F0010078B100BF608BD9
:10E6D00040F00200608300BF204601F077FB00BFDE
:10E6E000608B4FF6FC710840608300BFA07E00F095
:10E6F000080048B100BF608B4FF6F7710840608397
:10E7000000BF2046FFF74AFCE568A06F48B1002033
:10E7100009490870204602F0EBFE0748007800B176
:10E72000C5E72C4600E0E468002CC3D170BD0000B2
:10E730005A010020500100205801002010B5044665
:10E7400000BF207D012807D100BF06A3D42211A15C
:10E7500015A0F7F71DFE00BF00BF21460020FBF704
:10E7600083FF10BD2E2E2F4D6964646C6577617236
:10E7700065732F54686972645F50617274792F4CAD
:10E780007749502F7372632F636F72652F746370B4
:10E790002E6300007463705F667265653A204C49B1
:10E7A0005354454E00000000417373657274696FE5
:10E7B0006E2022257322206661696C656420617475
:10E7C000206C696E6520256420696E2025730A001F
:10E7D0002DE9F04705460C469146984635E0264619
:10E7E00024687068FDF7CCFA074600BFB5F86600EC
:10E7F000B84208DA00BF22A340F257422DA137A049
:10E80000F7F7C6FD00BF00BF35F8660FC01B2880B4
:10E8100030893C49098808443A490880304604F068
:10E8200021FA35F8660900280FD000BF002C0BD163
:10E83000B8F1000F08D100BF11A340F2614232A12C
:10E8400026A0F7F7A5FD00BF00BFB4B1E168486896
:10E85000FBF7FCF98246E1688889FBF704FA00F0CF
:10E86000030008B1012000E0002021890844504441
:10E870002D490968401A0028B1DD2046BDE8F0871F
:10E880002E2E2F4D6964646C6577617265732F5409
:10E89000686972645F50617274792F4C7749502FA8
:10E8A0007372632F636F72652F7463705F696E2E6E
:10E8B000630000007063622D3E736E645F71756566
:10E8C00075656C656E203E3D20706275665F636C99
:10E8D000656E286E6578742D3E70290041737365EE
:10E8E0007274696F6E2022257322206661696C65DF
:10E8F00064206174206C696E6520256420696E2037
:10E9000025730A00780100207463705F7265636587
:10E910006976653A2076616C696420717565756504
:10E92000206C656E677468007401002010B50446A1
:10E9300000BF207D012807D100BF06A3DF2211A15F
:10E9400017A0F7F725FD00BF00BF21460120FBF708
:10E950008BFE10BD2E2E2F4D6964646C657761723D
:10E9600065732F54686972645F50617274792F4CBB
:10E970007749502F7372632F636F72652F746370C2
:10E980002E6300007463705F667265655F6C697307
:10E9900074656E3A20214C495354454E00000000E6
:10E9A000417373657274696F6E202225732220662D
:10E9B00061696C6564206174206C696E65202564F2
:10E9C00020696E2025730A0010B50446606F20B1DF
:10E9D000606F04F054F90020606710BD0D48018895
:10E9E0000088401C0B4A10800B48006818B10B4887
:10E9F0000088814205DA0A48006800F11402505C80
:10EA0000704706480078081AC2B203480068805C64
:10EA1000F6E700006C01002068010020660100207C
:10EA20006001002070B50B48046810E0E568A07E26
:10EA300000F0080048B100BF608B4FF6F771084046
:10EA4000608300BF2046FFF7A9FA2C4600BF002CC8
:10EA5000ECD170BD5001002010B5F1F745FCC0F3BA
:10EA60000D0000F540400149088010BD4001002024
:10EA70002DE9FE4F05468B4600BF002D07D100BF94
:10EA8000E2A38322EEA1F4A0F7F782FC00BF00BF4F
:10EA9000FB49686808606889142800DAC8E3F94A05
:10EAA00011685069F9F785FD28B9F648007D00F036
:10EAB000F000E02800D1BBE3F14909688889FBF741
:10EAC000D2F800138700142F02DB2889B84200DA3D
:10EAD000AEE3A7F11400EC4908800020EB49086080
:10EAE0006889B84208DBE8480088E9490880394667
:10EAF0002846FDF7BFFD4AE000BF286838B900BFCF
:10EB0000C2A3C222E3A1D4A0F7F742FC00BF00BF1A
:10EB100014212846FDF7AEFD6889DD490880DA48F2
:10EB200000880988401A1FFA80FAD94801882846C7
:10EB3000FDF7A0FD28684089504500DA78E3286891
:10EB40004068D249086051462868FDF793FD28893E
:10EB5000A0EB0A00288100BF688938B100BFABA3D1
:10EB6000DF22D0A1BCA0F7F713FC00BF00BF00BF9D
:10EB7000288929680989884207D000BFA3A3E02219
:10EB8000CBA1B5A0F7F704FC00BF00BF00BFBC4994
:10EB900009680888FBF767F8B94909680880B84927
:10EBA00009684888FBF75FF8B54909684880B449A7
:10EBB00009684868FBF74AF8B14909684860C449E0
:10EBC0000860AF4909688868FBF740F8AC490968F4
:10EBD0008860C0490860AA490968C889FBF743F8FA
:10EBE000A7490968C881A64909688889FBF73BF8E5
:10EBF00000F03F00B84908702889B8490880B64835
:10EC0000007800F0030040B108460088401C0880EE
:10EC100028890988884200DD0AE34FF00009B048DE
:10EC2000046873E000BF207D38B900BF77A3FB22E2
:10EC3000ACA189A0F7F7ACFB00BF00BF00BF207DEF
:10EC40000A2807D100BF71A3FC22B0A182A0F7F768
:10EC50009FFB00BF00BF00BF207D012807D100BF80
:10EC60006AA3FD22B4A17CA0F7F792FB00BF00BF0E
:10EC7000207A50B1217A8348406890F83400401CD3
:10EC8000C0B2814201D0A1463FE0208B7C49096897
:10EC90000988884237D1E08A7949096849888842D9
:10ECA00031D178496068096988422CD1754920685A
:10ECB0004969884227D100BFE068A04208D100BF5F
:10ECC00052A340F20D12A6A163A0F7F761FB00BFAB
:10ECD00000BFB9F1000F07D0E068C9F80C00804808
:10ECE0000068E0607E48046000BFE068A04208D190
:10ECF00000BF46A340F21512A4A157A0F7F748FBA6
:10ED000000BF00BF04E0A14600BFE468002C89D129
:10ED100000BF002C78D1A848046839E000BF207DEE
:10ED20000A2808D000BF39A340F21F12A3A14AA0AD
:10ED3000F7F72EFB00BF00BF207A48B1217A514877
:10ED4000406890F83400401CC0B2814200D01EE000
:10ED5000208B4B4909680988884217D1E08A4849C5
:10ED600009684988884211D1464960680969884222
:10ED70000CD1444920684969884207D1204604F0F3
:10ED8000B9FD2846FDF712FABDE8FE8F00BFE46822
:10ED9000002CC3D1A146954806681FE0307A50B1D7
:10EDA000317A3848406890F83400401CC0B2814243
:10EDB00001D0B14611E0F08A31490968498888429A
:10EDC00009D1304930684969884200D108E00EB164
:10EDD000306800B904E0B14600BFF668002EDDD10E
:10EDE00000BF8EB1B9F1000F07D0F068C9F80C0070
:10EDF0007E480068F0607D480660304600F04AFCBE
:10EE00002846FDF7D3F9BFE7F2E000002E2E2F4D84
:10EE10006964646C6577617265732F5468697264A4
:10EE20005F50617274792F4C7749502F7372632F42
:10EE3000636F72652F7463705F696E2E63000000EC
:10EE40007463705F696E7075743A20696E76616C78
:10EE50006964207062756600417373657274696FCE
:10EE60006E2022257322206661696C6564206174BE
:10EE7000206C696E6520256420696E2025730A0068
:10EE800060010020B0BE0020640100206801002065
:10EE900066010020702D3E6E65787420213D204E65
:10EEA000554C4C00702D3E6C656E203D3D20300071
:10EEB000702D3E746F745F6C656E203D3D20702D2B
:10EEC0003E6E6578742D3E746F745F6C656E0000E5
:10EED00070010020740100207C0100207A010020D4
:10EEE000500100207463705F696E7075743A206120
:10EEF0006374697665207063622D3E737461746516
:10EF000020213D20434C4F53454400007463705F03
:10EF1000696E7075743A20616374697665207063F8
:10EF2000622D3E737461746520213D2054494D4526
:10EF30002D574149540000007463705F696E70750D
:10EF4000743A20616374697665207063622D3E7344
:10EF50007461746520213D204C495354454E000096
:10EF60007463705F696E7075743A207063622D3ED1
:10EF70006E65787420213D2070636220286265668A
:10EF80006F72652063616368652900007463705F58
:10EF9000696E7075743A207063622D3E6E65787488
:10EFA00020213D20706362202861667465722063B1
:10EFB0006163686529000000540100207463705F7C
:10EFC000696E7075743A2054494D452D5741495426
:10EFD000207063622D3E7374617465203D3D205442
:10EFE000494D452D57414954000000004C01002077
:10EFF000002C73D0002091490860288908810846B8
:10F0000045608F480068C86000208E4908608E49BE
:10F0100008708E4908808E48007800F0080018B10A
:10F02000687B40F001006873A06F80B1204602F059
:10F030005FFA0D3028B1A06F48B1864800880028DB
:10F0400005DD608D10B9204603F026FEBCE0824845
:10F050000460204601F0AAFE804608F10D00002859
:10F0600016D07948007800F0080090B100BFD4F8BD
:10F07000900028B16FF00D01D4F8902020699047DE
:10F0800000BF2146754801F0A5FD2046FFF756FB5D
:10F0900099E04FF000086D480088002819DD6B48A2
:10F0A000B0F800A000BFD4F8800038B15246214625
:10F0B000D4F8803020699847804601E04FF000087E
:10F0C00000BF08F10D0000B97EE000205F49088014
:10F0D00000BF204600F0D8F808B175E084E0594838
:10F0E0000068A8B300BFA06F50B100BFAFF2E42327
:10F0F0004FF4F3725AA1AFF2A020F7F749F900BF1D
:10F1000000BFA07E00F0100038B14E480068FDF747
:10F110004DF82046FEF768FC56E000BFD4F88400A6
:10F1200048B100234749D4F884C020690A682146C1
:10F13000E047804607E0002342482146026818461F
:10F1400003F004F9804600BF08F10D0008B93BE068
:10F1500005E0B8F1000F02D03A480068A0673A48CD
:10F16000007800F0200018B3A06F30B1A06F407B92
:10F1700040F02000A16F48731AE0208DB0F5066FB3
:10F1800002D0208D401C208500BFD4F8840040B1FF
:10F1900000231A462146D4F884C02069E0478046FF
:10F1A00001E04FF0000800BF08F10D0000B90BE0CE
:10F1B000002029490860204600F066F800B103E00D
:10F1C000204600F003FE00BF0020234908601D49CF
:10F1D00008601A48406840B318494868FCF7E6FFE1
:10F1E00000201649486020E0154909688889FAF727
:10F1F0003AFD00F00400A8B91148006800881049E1
:10F20000096849881D4ACDE9002102901C48006820
:10F21000104909884218194B1B1D1A480168002023
:10F2200003F032FC2846FCF7C1FF00BF00BFABE58E
:10F230002846FCF7BBFF00BFA6E5000024F5002030
:10F2400060010020800100207D0100207801002065
:10F250007C0100207A010020840100205001002060
:10F260007063622D3E726566757365645F64617478
:10F2700061203D3D204E554C4C000000C0BE00209A
:10F28000700100207401002010B5044600BF002C5E
:10F2900008D100BF13A340F25A221FA128A0F7F7FC
:10F2A00077F800BF00BF3048007800F01000B8B118
:10F2B000A07E00F0100050B900BFD4F8900028B133
:10F2C0006FF00E01D4F890202069904700BF2146CE
:10F2D000264801F07FFC2046FFF730FA012010BDE0
:10F2E0000020FCE72E2E2F4D6964646C65776172F7
:10F2F00065732F54686972645F50617274792F4C22
:10F300007749502F7372632F636F72652F74637028
:10F310005F696E2E630000007463705F696E7075C4
:10F32000745F64656C617965645F636C6F73653A83
:10F3300020696E76616C6964207063620000000071
:10F34000417373657274696F6E2022257322206683
:10F3500061696C6564206174206C696E6520256448
:10F3600020696E2025730A007D01002050010020D5
:10F370002DE9F0410446002600BF002C08D100BF53
:10F3800014A340F6240220A126A0F7F701F800BF3D
:10F3900000BF216D481EFAF759FC80464346002203
:10F3A0003146204600F0C4FE05461DB94FF0FF303F
:10F3B000BDE8F081334600222946204601F036F8A8
:10F3C000231D22462946204600F0B2FF0746384654
:10F3D000EEE700002E2E2F4D6964646C6577617234
:10F3E00065732F54686972645F50617274792F4C31
:10F3F0007749502F7372632F636F72652F74637038
:10F400005F6F75742E6300007463705F6B65657069
:10F41000616C6976653A20696E76616C696420700A
:10F4200063620000417373657274696F6E202225F8
:10F430007322206661696C6564206174206C696E5A
:10F440006520256420696E2025730A002DE9F041AE
:10F4500007467F2F01DD7F2000E0384606460EB9C3
:10F46000BDE8F081701EC6B24FF0000800250F48BD
:10F47000046813E0607DB04208DB607DB0420CD1CF
:10F480000B49206A0968081A404506D30849206AD2
:10F490000968A1EB00082546667DE468002CE9D1E7
:10F4A00015B12846FEF7A0FA00BFD9E750010020A9
:10F4B000440100202DE9F041054600BF082D0AD087
:10F4C000092D08D000BF13A340F2DD621DA121A0C9
:10F4D000F6F75EFF00BF00BF00270026274804683C
:10F4E0000EE0207DA8420AD12549206A0968081A41
:10F4F000B84204D32249206A09680F1A2646E468F4
:10F50000002CEED11EB100213046FEF783F9BDE894
:10F51000F08100002E2E2F4D6964646C6577617256
:10F5200065732F54686972645F50617274792F4CEF
:10F530007749502F7372632F636F72652F746370F6
:10F540002E630000696E76616C6964207374617467
:10F5500065000000417373657274696F6E20222527
:10F560007322206661696C6564206174206C696E29
:10F570006520256420696E2025730A005001002053
:10F580004401002070B5002600250B4804680BE0FC
:10F590000A49206A0968081AB04204D30749206A58
:10F5A00009680E1A2546E468002CF1D115B12846E9
:10F5B000FEF71AFA70BD000054010020440100203B
:10F5C00070B5044600BF44B900BF12A340F2111247
:10F5D0001CA11FA0F6F7DCFE00BF00BF00BF207D0E
:10F5E000012808D000BF0BA34FF4897222A118A0F4
:10F5F000F6F7CEFE00BF00BF012507E0244951F811
:10F6000025100868214602F091FF6D1C042DF5D3EA
:10F6100070BD00002E2E2F4D6964646C6577617299
:10F6200065732F54686972645F50617274792F4CEE
:10F630007749502F7372632F636F72652F746370F5
:10F640002E63000070636220213D204E554C4C001B
:10F65000417373657274696F6E2022257322206670
:10F6600061696C6564206174206C696E6520256435
:10F6700020696E2025730A007063622D3E737461E9
:10F680007465203D3D204C495354454E0000000018
:10F690005C6F01082DE9FE4305465448007800F0F0
:10F6A000040008B1BDE8FE8300BF002D08D100BFF3
:10F6B0004FA340F281225BA162A0F6F769FE00BF72
:10F6C00000BF4A48007800F01000B0B167480068F9
:10F6D0000088664909684988654ACDE90021029099
:10F6E00064480068644909884218614B1B1D6348DF
:10F6F0000168284603F0C8F975E03C48007800F03E
:10F70000020000286FD0687DFEF7D2F9044674B974
:10F7100000BFA86938B14FF0FF320021AB692869FA
:10F720009847804601E06FF00F0800BFBAE75048E5
:10F730001038406920604E48103800696060E88ADF
:10F74000E0824A48006800882083032020754948E9
:10F750000068401C6062606AE062204600F048FA7F
:10F760000646A66526656664E66542480068401E52
:10F77000606528692061E567687A00F00C006072B6
:10F78000287A207200BF00BF3D480068E0603C4816
:10F79000046004F093F800BF01203A49087000BFEC
:10F7A000204601F055F831480068C08924F8600F00
:10F7B00020886080603C201DF9F7D0FB8046608E79
:10F7C000221D4146FEF7A2FD608612212046FEF76B
:10F7D00007FE074627B100212046FEF71BF861E728
:10F7E000204600F0F3FA00BF5CE700007C01002037
:10F7F0002E2E2F4D6964646C6577617265732F548A
:10F80000686972645F50617274792F4C7749502F28
:10F810007372632F636F72652F7463705F696E2EEE
:10F82000630000007463705F6C697374656E5F6978
:10F830006E7075743A20696E76616C6964207063CD
:10F8400062000000417373657274696F6E20222537
:10F850007322206661696C6564206174206C696E36
:10F860006520256420696E2025730A006001002050
:10F87000C0BE0020700100207A0100207401002029
:10F88000500100205801002070B504460D460022AA
:10F890002946204600F002F870BD00002DE9F04135
:10F8A000044688461746002500BF002C0BD100BF38
:10F8B00038A340F2593243A14EA0F6F769FD00BFCC
:10F8C0006FF00F0660E000BF00BF207D00280BD066
:10F8D00000BF30A340F25A3250A146A0F6F758FDBF
:10F8E00000BF6FF00E064FE000BF207D012803D15E
:10F8F00025466FF0080647E00120FAF783FF05462A
:10F9000015B94FF0FF363FE020692861E08AE882B0
:10F9100001202875607D6875607A68720020287201
:10F92000E07AE872A07AA87220682860E08AD8B1EC
:10F9300000BF48480068A04205D146480068C0683A
:10F94000444908600DE04349086806E0C168A142E7
:10F9500002D1E168C16002E0C0680028F6D100BFB2
:10F9600000BF0020E06000BF2046FEF7E7FE3A48F7
:10F97000A86100BF39480068E8603848056003F0B6
:10F980009DFF00BF002600BF07B13E702846BDE8BE
:10F99000F08100002E2E2F4D6964646C65776172D2
:10F9A00065732F54686972645F50617274792F4C6B
:10F9B0007749502F7372632F636F72652F74637072
:10F9C0002E6300007463705F6C697374656E5F779B
:10F9D0006974685F6261636B6C6F675F616E645FBF
:10F9E0006572723A20696E76616C69642070636238
:10F9F00000000000417373657274696F6E202225E8
:10FA00007322206661696C6564206174206C696E84
:10FA10006520256420696E2025730A007463705F79
:10FA20006C697374656E5F776974685F6261636B3C
:10FA30006C6F675F616E645F6572723A20706362BB
:10FA400020616C726561647920636F6E6E656374AA
:10FA5000656400004801002009DA00084C0100201C
:10FA600070B506460D46D6B13068C0B10C48016885
:10FA7000304600F01BF80B480168304600F016F8DD
:10FA80006DB1286858B10848046806E020683168FC
:10FA9000884201D128682060E468002CF6D170BD4E
:10FAA00050010020480100204C0100202DE9F041C8
:10FAB00005460E46344600BF002D08D100BF0CA3FA
:10FAC0004FF4106216A123A0F6F762FC00BF00BF3E
:10FAD0000AE020682968884205D1E7682046FDF7DA
:10FAE00083FF3C4600E0E468002CF2D1BDE8F081E1
:10FAF0002E2E2F4D6964646C6577617265732F5487
:10FB0000686972645F50617274792F4C7749502F25
:10FB10007372632F636F72652F7463702E630000BE
:10FB20007463705F6E657469665F69705F61646459
:10FB3000725F6368616E6765645F7063626C69734E
:10FB4000743A20696E76616C6964206F6C645F61E1
:10FB500064647200417373657274696F6E2022254C
:10FB60007322206661696C6564206174206C696E23
:10FB70006520256420696E2025730A0010B5402099
:10FB8000FDF796FF10BD000010B5002300BF16481A
:10FB90000088401C144C2080204600884FF6FF74DB
:10FBA000A04203D14FF440400F4C2080002116E0CA
:10FBB0000E4850F8210002680DE0D08A0A4C2488D3
:10FBC000A04207D1581C83B2B3F5804F01DB00205F
:10FBD00010BDDCE7D268002AEFD1481CC1B204296D
:10FBE000E6DB01480088F3E7400100205C6F010874
:10FBF00010B5044600BF002C08D100BF09A340F691
:10FC0000AF0214A11AA0F6F7C3FB00BF00BF224841
:10FC100000682249096808441F49086008460068CE
:10FC200010BD00002E2E2F4D6964646C65776172E3
:10FC300065732F54686972645F50617274792F4CD8
:10FC40007749502F7372632F636F72652F746370DF
:10FC50002E6300007463705F6E6578745F69737300
:10FC60003A20696E76616C696420706362000000FE
:10FC7000417373657274696F6E202225732220664A
:10FC800061696C6564206174206C696E652025640F
:10FC900020696E2025730A005C01002044010020C9
:10FCA00070B505460C4600BF002D08D100BF25A346
:10FCB00040F21F4230A13AA0F6F76AFB00BF00BF36
:10FCC000E9688889F9F7CFFF00F0010020B12046EC
:10FCD00002F0D5FF002433E013E0E1688889F9F7EA
:10FCE000C2FF00F0010038B10120F9F7BCFFE9685C
:10FCF00089890843E968888126462468304602F0ED
:10FD0000B1FF4CB1E06840682189084429892E4A36
:10FD100012681144081AE0D594B128892A49096863
:10FD20000844E1684968401A002809DDE0688088D5
:10FD300025490988401A288129896868FCF792FBBF
:10FD40002C6070BD2E2E2F4D6964646C65776172D6
:10FD500065732F54686972645F50617274792F4CB7
:10FD60007749502F7372632F636F72652F746370BE
:10FD70005F696E2E630000007463705F6F6F735F66
:10FD8000696E736572745F7365676D656E743A2032
:10FD9000696E76616C6964206373656700000000BA
:10FDA000417373657274696F6E2022257322206619
:10FDB00061696C6564206174206C696E65202564DE
:10FDC00020696E2025730A00700100202DE9F84F8C
:10FDD000044600BF002C08D100BFA7A340F2E142B7
:10FDE000B2A1B8A0F6F7D4FA00BF00BF00BF207DD3
:10FDF000012808D100BFA0A340F2E342BBA1B1A0FB
:10FE0000F6F7C6FA00BF00BFC2480068A04202D1A0
:10FE10000020BDE8F88FB4F86000B4F848108842BC
:10FE200002DAB4F8600001E0B4F848008146E56EFB
:10FE300045B9A07E00F0020018B1204602F02CFF68
:10FE4000E7E710E1221D2146204602F00DFE07469D
:10FE500017B96FF00300DCE70CB1206858B90FB197
:10FE6000381D00E00020014611B96FF00300D0E713
:10FE70000868206000BFE9684868F9F7E7FE616C30
:10FE8000401A29890844484519D9B4F86000484502
:10FE90000CD1206F50B994F8990038B9002004F8BB
:10FEA000980F012060700020A070983CA07E00F0A8
:10FEB000020018B1204602F0EFFEAAE7D3E00020CE
:10FEC00084F89900266F26B100E036683068002873
:10FED000FBD1B5E000BFE9688889F9F7C4FE00F0FE
:10FEE000040040B100BF64A340F236528AA175A05D
:10FEF000F6F74EFA00BF00BF206FA0B1A07E00F061
:10FF0000440080B9E06E38B1E06E006858B9E06E28
:10FF10000089618E884206DAB4F8640018B1B4F83A
:10FF20006600092801DB012000E0002020B9A07E46
:10FF300000F0A00000B98FE0207D022807D010203B
:10FF4000F9F791FEE96889890843E96888813A46AA
:10FF50002146284600F0FCFA0090009838B100BF16
:10FF6000608B40F08000608300BF009851E72868F4
:10FF7000E066207D022806D000BF608B4FF6FC7142
:10FF80000840608300BFE9684868F9F75FFE804673
:10FF9000E9688889F9F767FE00F0030008B10120DD
:10FFA00000E000202989084408EB000A206DB0EB2E
:10FFB0000A0001D5C4F850A0E9688889F9F753FE12
:10FFC00000F0030008B1012000E000202989084466
:10FFD00088B300202860206F10B925672E462EE0D8
:10FFE000E9684868F9F732FE8046F1684868F9F731
:10FFF0002DFEB8EB00001BD504F1700801E0D8F825
:020000040801F1
:100000000080D8F8000068B1D8F80010C9684868C6
:10001000F9F71CFE8346E9684868F9F717FEBBEB61
:100020000000ECD4D8F800002860C8F8005006E0C2
:100030003560366803E0FFE7284602F013FEE56E00
:1000400055B1E9684868F9F701FE616C401A2989E1
:10005000084448457FF63EAF00BFE06E10B900206F
:10006000A4F8680000BF00BF608B4FF67F710840A6
:10007000608300BF0020CCE62E2E2F4D6964646C97
:100080006577617265732F54686972645F5061723D
:1000900074792F4C7749502F7372632F636F726599
:1000A0002F7463705F6F75742E6300007463705FEC
:1000B0006F75747075743A20696E76616C6964202E
:1000C00070636200417373657274696F6E202225DC
:1000D0007322206661696C6564206174206C696EAE
:1000E0006520256420696E2025730A00646F6E27E1
:1000F000742063616C6C207463705F6F75747075CD
:100100007420666F72206C697374656E2D70636203
:100110007300000084010020525354206E6F74203D
:100120006578706563746564206865726521000098
:100130002DE9FF4104460E461746984600BF002CA5
:1001400008D100BF10A340F242721CA125A0F6F70F
:100150001FF900BF00BF608D1023218BE28ACDE91B
:1001600001130092039043463A463146606A00F01C
:100170004DF805461DB1618D606A0844E06228466D
:1001800004B0BDE8F08100002E2E2F4D6964646C30
:100190006577617265732F54686972645F5061722C
:1001A00074792F4C7749502F7372632F636F726588
:1001B0002F7463705F6F75742E6300007463705FDB
:1001C0006F75747075745F616C6C6F635F68656187
:1001D0006465723A20696E76616C6964207063624E
:1001E00000000000417373657274696F6E202225F0
:1001F0007322206661696C6564206174206C696E8D
:100200006520256420696E2025730A002DE9F05FC2
:1002100082460D4617469846DDF830B005F11400C9
:10022000384481B24FF420722220FBF729FB0646A6
:10023000002E34D000BF718905F11400814208DA24
:1002400000BF18A340F2237223A12FA0F6F7A0F855
:1002500000BF00BF74680A98F9F705FD20800B986D
:10026000F9F701FD6080C4F804805046F9F7EEFC10
:10027000A060A946E91705EB91718910491D4FF659
:10028000FF7202EA013141EA0B00F9F7ECFCA081B0
:100290000D98F9F7E8FCE08100202082608230466A
:1002A000BDE8F09F2E2E2F4D6964646C65776172F6
:1002B00065732F54686972645F50617274792F4C52
:1002C0007749502F7372632F636F72652F74637059
:1002D0005F6F75742E630000636865636B207468DC
:1002E0006174206669727374207062756620636140
:1002F0006E20686F6C64207374727563742074630D
:10030000705F686472000000417373657274696F96
:100310006E2022257322206661696C6564206174F9
:10032000206C696E6520256420696E2025730A00A3
:100330002DE9FE4F04460E4692469B4600BF002E16
:1003400008D100BF17A340F2877223A12DA0F6F7B2
:100350001FF800BF00BF5A465146204602F084FBFA
:10036000054615B96FF0030715E024B194F80B802A
:1003700094F80A9003E04FF0FF084FF000090620C0
:1003800043465A465146CDE9009002953046F8F76B
:100390007DFB074600BF3046FBF708FF3846BDE847
:1003A000FE8F00002E2E2F4D6964646C657761729C
:1003B00065732F54686972645F50617274792F4C51
:1003C0007749502F7372632F636F72652F74637058
:1003D0005F6F75742E6300007463705F6F75747067
:1003E00075745F636F6E74726F6C5F7365676D6554
:1003F0006E743A20696E76616C696420706275660D
:1004000000000000417373657274696F6E202225CD
:100410007322206661696C6564206174206C696E6A
:100420006520256420696E2025730A002DE9F047B8
:1004300081460D4614469A464FF0000800BF002D35
:1004400008D100BF1CA340F2567228A131A0F5F7D5
:100450009FFF00BF00BF6E6806F1140700BF38465B
:1004600000EB880004F0010109B1042100E0002143
:10047000084404F0020109B1002100E00021084411
:1004800004F0080109B1002100E00021084404F053
:10049000100109B1002100E000210844B84208D051
:1004A00000BF05A340F2757224A11AA0F5F770FFF2
:1004B00000BF00BFBDE8F0872E2E2F4D6964646C2D
:1004C0006577617265732F54686972645F506172F9
:1004D00074792F4C7749502F7372632F636F726555
:1004E0002F7463705F6F75742E6300007463705FA8
:1004F0006F75747075745F66696C6C5F6F7074692A
:100500006F6E733A20696E76616C696420706275F3
:1005100066000000417373657274696F6E20222556
:100520007322206661696C6564206174206C696E59
:100530006520256420696E2025730A006F70746938
:100540006F6E73206E6F742066696C6C656400005A
:100550002DE9FE4F04460D46164600BF002C08D17B
:1005600000BF58A34FF4B76263A16BA0F5F710FF6B
:1005700000BF00BF00BF002D08D100BF51A340F253
:10058000B9526FA164A0F5F703FF00BF00BF00BF21
:10059000002E08D100BF4BA340F2BA5270A15EA05A
:1005A000F5F7F6FE00BF00BF204600F0F7F810B1E7
:1005B0000020BDE8FE8F686AF9F748FBE1688860B3
:1005C000688DF9F750FBE168C881698D686A084455
:1005D000E862E06800F11407A07A00F0010068B159
:1005E0002A1D31464FF40670FDF790FE82464AF010
:1005F0000170F9F72BFB38603F1D00BFB5F93000E3
:10060000002801DA00202886686B38B95D48006848
:100610006863E1684868F9F719FBA863A089616815
:100620008988401A1FFA80F860684089A0EB0800AA
:100630006168488160680089A0EB080061680881F2
:100640006168E06848600020E168088200BFE068F7
:100650001430A17A01F0010109B1042100E0002168
:100660000844A17A01F0020109B1002100E0002153
:100670000844A17A01F0080109B1002100E000213D
:100680000844A17A01F0100109B1002100E0002125
:100690000844B84208D000BF0AA340F21C623AA145
:1006A0001DA0F5F775FE00BF00BF0621A87A8DE8F2
:1006B0004300EB7A2A1D29466068F8F7E7F981467E
:1006C000484676E72E2E2F4D6964646C657761721B
:1006D00065732F54686972645F50617274792F4C2E
:1006E0007749502F7372632F636F72652F74637035
:1006F0005F6F75742E6300007463705F6F75747044
:1007000075745F7365676D656E743A20696E7661A6
:100710006C69642073656700417373657274696FF7
:100720006E2022257322206661696C6564206174E5
:10073000206C696E6520256420696E2025730A008F
:100740007463705F6F75747075745F7365676D65E2
:100750006E743A20696E76616C6964207063620021
:100760007463705F6F75747075745F7365676D65C2
:100770006E743A20696E76616C6964206E65746986
:1007800066000000440100206F7074696F6E732072
:100790006E6F742066696C6C6564000010B5044669
:1007A00000BF002C08D100BF08A340F29A5214A148
:1007B0001DA0F5F7EDFD00BF00BF6068807B01283C
:1007C00001D0012010BD0020FCE700002E2E2F4D8F
:1007D0006964646C6577617265732F5468697264CB
:1007E0005F50617274792F4C7749502F7372632F69
:1007F000636F72652F7463705F6F75742E63000092
:100800007463705F6F75747075745F7365676D6521
:100810006E745F627573793A20696E76616C696493
:100820002073656700000000417373657274696F1F
:100830006E2022257322206661696C6564206174D4
:10084000206C696E6520256420696E2025730A007E
:100850002DE9F041054600BF002D08D100BF28A3B7
:1008600040F27D7233A13AA0F5F792FD00BF00BFC0
:1008700041480088002840D000204049088036E0E8
:10088000FEF7ACF8074627B1012F04D0022F1FD185
:1008900002E0BDE8F08128E0FEF7A0F8042806D1C8
:1008A00036480088801C34490988884200DDF0E71A
:1008B000FEF794F80602FEF791F80643B6F5067FB8
:1008C00000DC16B94FF4067000E0304668860CE094
:1008D000FEF784F80446022C00DADAE7A01E274966
:1008E000098808442549088000BF00BF00BF23488D
:1008F0000088214909888842C2DB00BFC9E700009F
:100900002E2E2F4D6964646C6577617265732F5468
:10091000686972645F50617274792F4C7749502F07
:100920007372632F636F72652F7463705F696E2ECD
:10093000630000007463705F70617273656F707440
:100940003A20696E76616C69642070636200000011
:10095000417373657274696F6E202225732220665D
:1009600061696C6564206174206C696E6520256422
:1009700020696E2025730A00640100206C010020AC
:100980002DE9F84F81460C4617469846DDE90BAB3A
:100990000A9E009400BFB8F1000F07D100BF29A341
:1009A000E82235A13DA0F5F7F3FC00BF00BF00BF72
:1009B000002E07D100BF23A3E92242A137A0F5F7FB
:1009C000E7FC00BF00BFBC421BDA0AF0020050B9CE
:1009D000B07E00F04000A0B9BBF1000F03D0F06E74
:1009E00008B9306F68B104F21B2020F00300B84250
:1009F00001D9384603E004F21B2020F0030080B246
:100A000000904FF4207248460099FAF739FF0546E6
:100A100015B90020BDE8F88F00BF286840B100BFBD
:100A200008A340F20B122FA11CA0F5F7B1FC00BFE8
:100A300000BF6889001BA8F800002C816C81284643
:100A4000E8E700002E2E2F4D6964646C65776172B3
:100A500065732F54686972645F50617274792F4CAA
:100A60007749502F7372632F636F72652F746370B1
:100A70005F6F75742E6300007463705F70627566DB
:100A80005F707265616C6C6F633A20696E76616C41
:100A90006964206F76657273697A65004173736566
:100AA0007274696F6E2022257322206661696C65FD
:100AB00064206174206C696E6520256420696E2055
:100AC00025730A007463705F706275665F7072658B
:100AD000616C6C6F633A20696E76616C696420703A
:100AE000636200006E65656420756E636861696E9F
:100AF000656420706275660010B5044600BF002C66
:100B000009D100BF16A340F6510221A127A0F5F795
:100B10003FFC00BF10BD00BF207DF8B1207D0A283A
:100B20001CD0207D012819D0A06F20B1A06FFBF749
:100B30003DFB0020A067606F10B12046FDF744FF29
:100B40004FF0FF302086E06E02F099F8206F02F03F
:100B500096F80020E0662067A4F8680000BFD9E797
:100B60002E2E2F4D6964646C6577617265732F5406
:100B7000686972645F50617274792F4C7749502FA5
:100B80007372632F636F72652F7463702E6300003E
:100B90007463705F7063625F70757267653A206935
:100BA0006E76616C696420706362000041737365E6
:100BB0007274696F6E2022257322206661696C65EC
:100BC00064206174206C696E6520256420696E2044
:100BD00025730A0070B505460C4600BF002C08D1ED
:100BE00000BF3AA340F6830244A14BA0F5F7D0FB27
:100BF00000BF00BF00BF002D08D100BF33A340F6E7
:100C000084024FA144A0F5F7C3FB00BF00BF00BFA3
:100C10002868A04203D12868C06828600CE02868D2
:100C200006E0C168A14202D1E168C16002E0C0688B
:100C30000028F6D100BF00BF0020E06000BF2046C2
:100C4000FFF75AFF207D0A280FD0207D01280CD005
:100C5000A07E00F0010040B100BF608B40F00200B8
:100C6000608300BF2046FFF7B1F8207D012826D021
:100C700000BFE06E40B100BF14A340F6930238A15C
:100C800025A0F5F785FB00BF00BF00BF206F40B176
:100C900000BF0EA340F6940237A11FA0F5F778FB22
:100CA00000BF00BF00BF606F40B100BF07A340F6A8
:100CB000960238A118A0F5F76BFB00BF00BF00201B
:100CC0002075E08200BF00BF70BD00002E2E2F4DAA
:100CD0006964646C6577617265732F5468697264C6
:100CE0005F50617274792F4C7749502F7372632F64
:100CF000636F72652F7463702E6300007463705F9E
:100D00007063625F72656D6F76653A20696E7661B9
:100D10006C69642070636200417373657274696FFB
:100D20006E2022257322206661696C6564206174DF
:100D3000206C696E6520256420696E2025730A0089
:100D40007463705F7063625F72656D6F76653A2081
:100D5000696E76616C6964207063626C697374009B
:100D6000756E73656E74207365676D656E74732040
:100D70006C65616B696E6700756E61636B6564209D
:100D80007365676D656E7473206C65616B696E6702
:100D9000000000006F6F736571207365676D656E8D
:100DA0007473206C65616B696E6700002DE9FE430A
:100DB00004460027002600BF002C08D100BFE5A391
:100DC0004FF44772F0A1F7A0F5F7E2FA00BF00BFB9
:100DD000FE48007800F00400002845D0207D02285D
:100DE00006D1FB49206D096888421BD1012719E013
:100DF000F849606A0968884201D1012712E0F54983
:100E0000606A0968081A0DD4218D606A0844F149A6
:100E10000968081A002805DC00BF608B40F002005A
:100E2000608300BF002F1DD000BF207D40B900BFF0
:100E3000C8A34FF44E72E8A1DAA0F5F7A9FA00BFF3
:100E400000BFED48007840F00800EB49087000BF93
:100E5000608B4FF6FE710840608300BF6FF00D009D
:100E6000BDE8FE830020FBE7D848007800F00200D0
:100E700068B1207D02280AD0207D032807D000BF5A
:100E8000608B40F00200608300BF0020E8E7A07E96
:100E900000F0100010B9D94800682062002084F8E2
:100EA0009B0084F89A002046FFF7D2FC207D801E2C
:100EB000082875D2DFE800F004CDF4F3F2F1F0EF8A
:100EC000C248007800F0100000286AD0BF480078BF
:100ED00000F002000028F8D0606C401CBC49096892
:100EE00088425ED1BB480068401C6062606AE06274
:100EF000B74800686064C2480068C089A4F8600010
:100F0000B4F86000A4F86200B2480068401E606552
:100F100004202075201DF8F721F88046608E221DE0
:100F20004146FDF7F3F96086608E8100400041F292
:100F30001C12904202D9608E400001E041F21C1068
:100F4000814202D2608E80000AE0608E400041F251
:100F50001C11884202D9608E400001E041F21C1051
:100F6000A4F8480000BFB4F86600002808DC00BF01
:100F700078A34FF45B72A3A18AA0F5F709FA00BF2A
:100F800000BFB4F86600401EA4F86600256F95B94E
:100F9000E56E00BF5DB900BF6EA34FF45D7201E066
:100FA0008DE231E09DA17FA0F5F7F2F900BF00BF0F
:100FB0002868E06601E028682067284601F052FEB4
:100FC000206F18B94FF0FF30208603E00020208604
:100FD00084F8420000BFD4F8880038B100222146CE
:100FE000D4F8883020699847064600E0002600BF04
:100FF00006F10D0010B96FF00C0031E700BF608BF7
:1010000040F00200608323E07048007800F0100098
:10101000F0B17B4800680088794909684988844AAA
:10102000CDE9002102906B48006882490988421886
:101030007F4B1B1D66480168204601F025FD94F892
:101040004200062804DA00202086204601F0D0FB6A
:1010500036E25E48007800F01000002876D0606C20
:10106000401C5B490968081A71D45949206D096808
:10107000081A00286BDC04202075E06F10B96FF0AF
:10108000050623E000BFE06F806978B900BF31A397
:101090004FF46A7205E0FCE1BCE107E17CE117E195
:1010A00005E165A13FA0F5F773F900BF00BF00BFE0
:1010B000E06F806938B1E16F206900228B692146B9
:1010C0009847064601E06FF00F0600BF46B106F1F3
:1010D0000D0010B12046FCF787FC6FF00C00BFE656
:1010E000204600F09FFA5C48008820B15A480088EA
:1010F000401E59490880608E8100400041F21C1258
:10110000904202D9608E400001E041F21C10814201
:1011100002D2608E80000AE0608E400041F21C1115
:10112000884202D9608E400001E041F21C10A4F810
:1011300048003148007800F0200048B100BF608BC3
:1011400040F00200608300BF072087E09FE087E057
:10115000ABE000002E2E2F4D6964646C65776172E0
:1011600065732F54686972645F50617274792F4C93
:101170007749502F7372632F636F72652F7463709A
:101180005F696E2E630000007463705F70726F633E
:101190006573733A20696E76616C6964207063626E
:1011A00000000000417373657274696F6E20222520
:1011B0007322206661696C6564206174206C696EBD
:1011C0006520256420696E2025730A007C010020BB
:1011D00074010020700100207463705F696E707587
:1011E000743A207063622D3E737461746520213DF2
:1011F00020434C4F534544007D0100204401002012
:10120000600100207063622D3E736E645F717565CE
:1012100075656C656E203E20300000006E6F207397
:1012200065676D656E7420746F2066726565000079
:10123000C0BE00207A0100207063622D3E6C69738D
:1012400074656E65722D3E61636365707420213D27
:10125000204E554C4C00000078010020207524E001
:10126000994800680188984800684088974ACDE905
:101270000020029196480068964909884218934BCD
:101280001B1D95480168204601F0FEFB0DE09348C8
:10129000007800F0020040B1606A401E8C49096885
:1012A000884202D1204601F09BF909E100BF2046A7
:1012B00000F0B8F98A48007800F0200038B100BF8B
:1012C000608B40F00200608300BF07202075F7E0CC
:1012D000204600F0A7F98248007800F02000E8B32B
:1012E0007E48007800F01000C8B37B49206D096883
:1012F000884239D1E06E90BB00BF608B40F00200A5
:10130000608300BF2046FFF7F7FB00BF00BF7548B2
:101310000068A04205D173480068C0687149086040
:101320000DE07049086806E0C168A14202D1E16899
:10133000C16002E0C0680028F6D100BF00BF0020F5
:10134000E06000BF01206849087000BF0A202075D6
:1013500000BF66480068E060644801E00DE003E01B
:10136000046002F0ABFA16E000BF608B40F00200B0
:10137000608300BF082020750DE05848007800F019
:10138000100040B15449206D0968884203D1E06ED5
:1013900008B90620207593E0204600F043F9504834
:1013A000007800F02000A0B300BF608B40F0020086
:1013B000608300BF2046FFF79FFB00BF00BF494886
:1013C0000068A04205D147480068C06845490860E8
:1013D0000DE04449086806E0C168A14202D1E16815
:1013E000C16002E0C0680028F6D100BF00BF002045
:1013F000E06000BF01203C49087000BF0A20207552
:1014000000BF3A480068E0603848046002F056FACD
:1014100000BF55E0204600F005F93048007800F0A4
:101420001000A8B32C49206D0968884230D1E06EC5
:1014300070BB2046FFF760FB00BF00BF2948006873
:10144000A04205D127480068C068264908600DE021
:101450002449086806E0C168A14202D1E168C16080
:1014600002E0C0680028F6D100BF00BF0020E060A5
:1014700000BF01201C49087000BF0A20207500BF72
:101480001A480068E0601948046002F017FA00BFCB
:1014900016E0204600F0C6F81048007800F0100072
:1014A00060B10D49206D0968884207D1E06E28B906
:1014B0000B48007840F010000949087000E000BFB8
:1014C00000BF0020CCE4000060010020C0BE00206E
:1014D000700100207A010020740100207C010020AE
:1014E0007D010020500100205801002054010020FF
:1014F0002DE9F041044600BF002C0CD100BF29A308
:1015000040F2096233A13DA0F4F742FF00BF6FF043
:101510000F00BDE8F08100BFA06F477BA66F0020E1
:10152000A06700BFD4F8840040B1002332462146B2
:10153000D4F884C02069E047054606E0002332461F
:101540002146184600F002FF054600BFF5B907F036
:10155000200028B3208DB0F5066F02D0208D401CEE
:10156000208500BFD4F8840040B100231A462146EC
:10157000D4F884C02069E047054600E0002500BF9C
:1015800005F10D0060B96FF00C00C2E705F10D0028
:1015900010B96FF00C00BCE7A6676FF00400B8E765
:1015A0000020B6E72E2E2F4D6964646C657761725A
:1015B00065732F54686972645F50617274792F4C3F
:1015C0007749502F7372632F636F72652F74637046
:1015D0002E6300007463705F70726F636573735F76
:1015E000726566757365645F646174613A20696EE3
:1015F00076616C69642070636200000041737365FA
:101600007274696F6E2022257322206661696C6591
:1016100064206174206C696E6520256420696E20E9
:1016200025730A002DE9F05F04464FF0000900BF62
:10163000002C08D100BFE5A340F27B42F0A1F7A047
:10164000F4F7A6FE00BF00BF00BF207D042808DA23
:1016500000BFDEA340F27C42FAA1F0A0F4F798FEAE
:1016600000BF00BFFE48007800F01000002870D0D6
:10167000B4F86000A16D00EB0108FA49606D0968DB
:10168000401A15D4F749606D0968884204D1F649BB
:10169000A06D0968401A0BD4F349A06D096888420F
:1016A0001AD1F2480068C089B4F86010884213D992
:1016B000EE480068C08924F8600F608834F860192B
:1016C000884203DAB4F86000A4F86200E5480068D4
:1016D0006065E5480068A065E349606C0968081A20
:1016E00000284ADCE248008890BBB4F86010A06D86
:1016F000084440453AD1B4F93000002836DBDA49D5
:10170000606C0968884231D14FF0010994F84300B8
:10171000401CC0B294F84310884204DD94F84300A2
:10172000401C84F8430094F84300032817DD00BFF1
:10173000B4F84800618E084480B2B4F8481088427A
:1017400008DBB4F84800618E0844A4F8480005E0BE
:101750000CE02AE14FF6FF70A4F8480000BF94F8AF
:101760004300032802DB204600F0BCFFB9F1000F64
:1017700002D1002084F84300EBE0606C401CBA49C1
:101780000968081A7ED4B849206D0968081A00282B
:1017900078DCA07E00F0040060B100BF608B4FF6E3
:1017A000FB710840608300BF4834608820800020BF
:1017B0006084483C00202434A077608BB4F9181072
:1017C00000EBE10000B2A083208CA7490988081A29
:1017D00085B20020E077A4480068206214F8100C5D
:1017E000243C042865DBB4F84800B4F84A10884269
:1017F00027DA628B02F400620AB1012200E00222C1
:101800001146628E4A4392B2AA4201DD2A4602E0A4
:10181000628E4A4392B2104600BFB4F84820024498
:1018200092B2B4F848309A4205DBB4F8482002443A
:10183000A4F8482003E04FF6FF72A4F8482000BF48
:1018400037E000BFB4F86A00284480B2B4F86A10E8
:10185000884205DBB4F86A002844A4F86A0003E073
:101860004FF6FF70A4F86A0000BFB4F86A00B4F83D
:10187000481088421DDB4834608C2188401A6084FF
:10188000483C00E062E000BFB4F84800618E0844C4
:1018900080B2B4F84810884206DBB4F84800618E84
:1018A0000844A4F8480003E04FF6FF70A4F848008D
:1018B00000BF70A22046D4E91B31FCF789FF2067E6
:1018C0006EA22046D4E91B13FCF782FFE066206F6E
:1018D00018B94FF0FF30208601E00020208600205C
:1018E0002077E06E10B90020A4F86800B4F8640016
:1018F000644909880844A4F86400608B00F400601F
:1019000018B3206F88B9E06E40B1E16EC9684868CD
:10191000F8F79CF9E16C081A002816DC00BF608B10
:101920004FF2FF71084060830FE0216FC96848687B
:10193000F8F78CF9E16C081A002806DC00BF608B10
:101940004FF2FF710840608300BF02E0204601F0C3
:10195000A3F9606B48B34449A06B0968401A24D5C9
:10196000A08E49490988081A07B2B4F93C00A7EBD0
:10197000E00007B2A08F384400B2A087002F01DA40
:10198000784207B2B4F93E00A7EBA00007B2E08F9F
:10199000384400B2E087E08FB4F93C1000EBE1007E
:1019A00000B2A4F84000002060633148008800289D
:1019B0006CDD207D072869DA2A48616A0068401CCE
:1019C000081A7CD42748616A006860E02E2E2F4DEB
:1019D0006964646C6577617265732F5468697264B9
:1019E0005F50617274792F4C7749502F7372632F57
:1019F000636F72652F7463705F696E2E6300000001
:101A00007463705F726563656976653A20696E76A6
:101A1000616C69642070636200000000417373654B
:101A20007274696F6E2022257322206661696C656D
:101A300064206174206C696E6520256420696E20C5
:101A400025730A007463705F726563656976653A31
:101A50002077726F6E6720737461746500000000F8
:101A60007C01002070010020740100206001002032
:101A70007A010020756E61636B656400756E736535
:101A80006E7400007801002044010020D4E3F74A7E
:101A900012881044401E081A00285FDCF44846688B
:101AA000F449606A0968A0EB010A00BFF048406889
:101AB00060B900BFAFF2EC0340F2945200E04DE099
:101AC000EDA1AFF2A800F4F763FC00BF00BF00BFB8
:101AD0004FF6FF7082450AD300BFAFF2101340F2F9
:101AE0009552E9A1AFF2CC00F4F752FC00BF00BF61
:101AF0001FFA8AF500BFDE4840680089A8420ADA6A
:101B000000BFAFF2381340F29752E3A1AFF2F400F6
:101B1000F4F73EFC00BF00BFD5480089401BD44904
:101B20000881084640680089401B1FFA80FB07E0D7
:101B30007089281A85B2A6F808B00020708136682E
:101B40007089A842F4DB29463046FAF793FDC9496B
:101B5000606A0860C649C96848600AE0C549606AA9
:101B60000968081A05D500BF608B40F00200608349
:101B700000BFC049606A0968081A7DD4218D606A77
:101B80000844401EBB490968081A002874DCB9499A
:101B9000606A0968884270D1B549C9688889F8F7D0
:101BA00062F800F0030008B1012000E00020B04915
:101BB00009890844AD490880208D0988884256DA91
:101BC000AB49C9688889F8F74EF800F0010098B170
:101BD000A749C9688889F8F746F800F03E05284605
:101BE000F8F741F8A249C96889894CF2FF0211400F
:101BF00008439F49C9688881208D9D490881C9682B
